:040000000C94880CC8
:100004000C9400000C9400000C9400000C9400006C
:100014000C9400000C9400000C949A610C94000061
:100024000C9400000C9475140C9400000C940000C3
:100034000C9400000C9400000C9400000C94231405
:100044000C9400000C943E5E0C9400000C947A5EB8
:100054000C9400000C9400000C9400000C9400001C
:100064000C9400000C9400000C9400000C9400000C
:100074000C9400000C94F55F0C9400000C9438610F
:100084000C9400000C9400006B65696E204B726543
:100094006469740054696D656F757400504C552023
:1000A400000000000100020004000800100020000D
:1000B400400080000001000200040008001000203D
:1000C40000400080000102040810204080002C043D
:1000D400C10B801000003004C10B821F00003A04E1
:1000E400C10B810300004204C10B010403004C0452
:1000F400C20B010605005604C40B01800000620413
:10010400CB0B020F00006A04C50B020F000072043F
:10011400C70B020FD0127A04C90B0110000084042B
:10012400190C011000008E04CA0B00010000960493
:10013400CD0B01080100A004CE0B03080100AE049E
:10014400CF0B03070000B604E50B017F3F00C0049A
:10015400E40B0106000096051C0C01040300CA040C
:10016400D00B03040000D204E30B01641E00DE0480
:10017400D10B00010000EA04D20B00010000F604D8
:10018400E20B010200000205D30B00010000100580
:10019400D40B020F00001C05D60B020FE703260543
:1001A400180C0163000084051A0C011000008E0570
:1001B4001B0C010202003205D80B030801003805AC
:1001C400D90B030800003E05DA0B030800004405C0
:1001D400DB0B030800004A05DC0B03080000500594
:1001E400DD0B030800005605DE0B030800005C0568
:1001F400E60B040A2E006405F00B040A2E006C05BD
:10020400FA0B040A2E007405040C040A2E007C0563
:100214000E0C040A2E0000000000FF0000005370C2
:100224006172746520200000A4050002AC0504047A
:10023400B2050807B8050C05B8058C06BE0580098B
:10024400C605100BCE05500CD8054003E005140A72
:10025400EA051808F2051C010000000254657374D5
:100264000000546F74616C2000006A6100006E65C8
:10027400696E0000580043616C6962726174696F51
:100284006E004F4B00004B653A00496E3A005469CA
:100294006E79200062616400454550524F4D200044
:1002A400446174612000496E6974000053746F7076
:1002B4000000567320312E354100310B312041426C
:1002C4004300320B322044454600330B3320474869
:1002D40049004D0A4D0000000000340B34204A4B05
:1002E4004C00350B35204D4E4F00360B3620505107
:1002F40052002B0A2B0000000000370B3720535408
:100304005500380B382056575800390B3920595AA4
:100314002F002D0A2D0000000000430C43000000B4
:100324000000300B3020202E2C002C0A2C00000062
:1003340000003D0A435200000000210C58002D0B20
:100344002D002B0B2B004D0A4D0028006000980057
:10035400D0000801400180818283840000218889C3
:100364008A8B8C8D8E8F00004A014600320021005A
:10037400004B004A01460032004D000096004A013D
:1003840046003200540000E1004A01460032003DBC
:100394000000F0000000320050002D0000F000507A
:1003A4000032005000470000F000A000320050006E
:1003B4004B0000F000F000320050002B0000B400AD
:1003C400040038003800217802008700C800640067
:1003D40032003D6E02000800C80064003200217241
:1003E40002004B004A01460032004D0000000100AB
:1003F4000100E60063004D0000000000A0001B00A7
:10040400007105D700A0001A020071056900000000
:10041400180400730569001E011906007305507263
:100424006F64756B742000005F4944005F5273323F
:100434003332494400005F526F74617465005F5445
:10044400617374656E5800005F54617374656E590E
:1004540000005F44656661756C744B6579002A43DE
:100464006F64653000002A436F64653100002A43DD
:100474006F64653200002A4D61784D6F64756C00BD
:100484005F4572774D6F64756C002A5469736368B5
:1004940045005F4D795465726D4E72005F4D617316
:1004A4007465725465726D7300005F454D6F6465C9
:1004B40000005F4543726564577472005F52733085
:1004C4004D6F646500005F5634756E6435005F508F
:1004D400756C736554696D6500005F41736B43729D
:1004E4006564697400005F53656E64446562697491
:1004F40000005F4372656469744D6F6465005F4317
:1005040072656469744D6173746572002A54616222
:100514006C655374617274002A5461626C65456E33
:1005240064002A4669727374426F6E5000002A4A4E
:100534006F6231002A4A6F6232002A4A6F623300C6
:100544002A4A6F6234002A4A6F6235002A4A6F626F
:1005540036002A4A6F6237005F4572726F7231004B
:100564005F4572726F7232005F4572726F72330050
:100574005F4572726F7234005F4572726F7235003C
:100584005F4672656967616265005F4B6F6D6D619F
:1005940000005F52733042617564726174650000DB
:1005A40054617374657200004C69745A00004C65A0
:1005B4006974540050756C73000054617374203076
:1005C400000073657269656C6C0073657269656CB3
:1005D400203200005461737420320000546173743B
:1005E400207061720000466F6C6765540000537799
:1005F400697463680000706F7274696F6E69657204
:10060400656E00002E666F6C67650000506F727433
:10061400696F6E656E207369636865726E006661EA
:100624006C73636865722054697363682000206783
:100634006573706572727400546973636820766FB1
:100644006E204B2000004665686C6572200056657C
:100654006E74696C20616B746976000043534920A1
:100664004E722000436F64652000546973636820F0
:100674000000436865662D4D656E75004B206C69FE
:100684007374656E00004B206C6F65736368656EF0
:1006940000004B20647275636B656E0054206C69B6
:1006A4007374656E000054206C6F65736368656EC7
:1006B40000005420647275636B656E005379737423
:1006C400656D0000506F7274696F6E004B726564E3
:1006D400697465004B7265642E436C7200006D6131
:1006E4006E2E506F7274696F6E00506172616D6529
:1006F4007465720050726F64756B746500004B65AD
:100704006C6C6E65720056656E74696C650045723A
:10071400726F72004F70742E0000496D70756C73A7
:1007240000004162726563686E756E6700004D6F0C
:1007340064756C20000073656300496D700050722D
:1007440031005072320046756E6374005479700043
:100754003A20563A2020302B203000003A20544FC3
:100764003A2000003A2050733A20000053703A00B7
:10077400730049004B204D6F6465204A6F62204A24
:100784006F62466C616773004B2000004D6F6465B7
:1007940020004A6F622000005620202045727220FB
:1007A40050676C20496D7020544F000020563A0069
:1007B4005061757365002E202C304142433144450D
:1007C4004632474849334A4B4C344D4E4F355051CD
:1007D40052365354553756575838595A2F3930765C
:1007E40006318006328A0633960634A00635AA06F8
:1007F40036B60646C00641C80643D00644D8064A63
:10080400E2060000000030C00637600239EE063808
:10081400F806420207450A07000000001207300CE0
:10082400000500001807330C000300001E07310CFC
:10083400000500009800320C001400000500C111EE
:1008440000000300D90B00000300C1110300170EC0
:100854000300D90B00000500E00800000A00C111E4
:100864000A00170E0A00D90B0A00C1110A00170E5C
:100874002800D90B00000000000000000000000068
:100884000000000000000000000000000000070C51
:10089400182022204D994D40114048914720222094
:1008A40018C007000000070C1F3FEE3F7277727FED
:1008B400FF7F777F783FEE3F1FC0070000000000F6
:1008C40000000C183DEE3F3FEE3F1FC80F0700022B
:1008D40000000000000000000000000207080F1FD5
:1008E400CE3F1FC80F0700020000000000000000F8
:1008F4000007080F0F880F376F7F7FFF7F32600775
:100904000F800000000000000002000207080F1F13
:10091400CE3F3FEE3F1AC0070F80000000000000EA
:100924000000000000000006000F0F000600000099
:10093400000000000000FFFFFFFFFFFFFFFFFFF9C3
:10094400FFF0F0FFF9FFFFFFFFFFFFFFFFFF0000D5
:100954000000000006000910881010881009000625
:10096400000000000000FFFFFFFFFFFFF9FFF6EFAC
:1009740077EFEF77EFF6FFF9FFFFFFFFFFFF0000D0
:1009840000000E01006A1E33286161886133001E75
:10099400000000000000000000078C0C1866181806
:1009A4006C0C078003030C0F03000300000002001B
:1009B40003038C0302CC0202800202000E1E001EFE
:1009C4000C00000000000C000E0B08090CC40E0BF8
:1009D4004C0938C478784C3103CC03018000000002
:1009E400020202271FCC18306770306C181FC22710
:1009F4000200020000000000001000181C001E1F6E
:100A0400081F1F001E1C001810000000000000003A
:100A1400000088010388070F881F0F8807038801D7
:100A240000800000000000000207080F1FC002023F
:100A340000020200021FC80F0700020000000008A5
:100A44001919881919881919881919881919800008
:100A5400198819000000000E1F36CC6666CC663675
:100A6400CC1E06CC0606CC0606CC06000000000808
:100A74001F30C03030081F30CC301F8C0000CC3009
:100A84001F800000000000000000000000000000C3
:100A94000000000000000E1F1FEE1F0000000200F7
:100AA400070F8C1F0200020200020200021FC80F7F
:100AB4000700021FC00000000207080F1FC0020247
:100AC4000002020002020002020002000000000014
:100AD400020200020200020200020200021FC80F0A
:100AE40007000200000000000000000001080101EE
:100AF400CE3F01C80101000000000000000000001A
:100B04000000000004000C1C0E3F1C000C0400003C
:100B140000000000000000000000000000000000D1
:100B24000000400040400040400E7F0000000000F4
:100B340000000000088C1838EF7F38EC180880009B
:100B44000000000000000000000000000000020798
:100B5400080F1FCE3F7FF0000000000000000000DF
:100B640000000000000F7F3FEC1F0F800702000011
:100B74000000000000000000000000000000000071
:100B8400000000000000000000000000000006005B
:100B9400060F000F0F000F0F0006060006000000EE
:100BA40006000600000000000019881919881900C1
:100BB400000000000000000000000000000000062B
:100BC400060666063FFC0C0CC819198C7F330033EB
:100BD4003300000000000600061F8C3F3600363F3D
:100BE4008C1F06CC063FC81F06000600000000004C
:100BF40000001338387E3801C80307000E1C0E3875
:100C040070EE600000000000070D881919801B0EAB
:100C1400001E3E063333C8313BC61E0000000E00E2
:100C24000E0E000606000C0000000000000000008C
:100C34000000000000000380060E000C1C001C1CB9
:100C4400001C1C001C0C000E0608030000001C0005
:100C540006070003038803038803038803030007CC
:100C640006001C000000000000000C3636C81F0FF0
:100C74000C3F0F081F36CC360000000000000000B7
:100C840000000000060006060C3F3FC006060006F2
:100C94000000000000000000000000000000000050
:100CA400000000000000000E0E000E06000C000004
:100CB40000000000000000000C3F3FC000000000E6
:100CC4000000000000000000000000000000000020
:100CD400000000000000000E0E000E0000000001E5
:100CE4000000370000EC010380070E001C38007080
:100CF4006000000000000F8E3F30676060FB61639E
:100D040033666C33787036303FE80F000000030020
:100D1400071F001F03000303000303000303000372
:100D24001FEE1F0000001FCE3F707360607E000145
:100D3400C80307000E1C00387FFF7F0000001FCE91
:100D44003F7073600037000FEC0F00630060377072
:100D54003FEC1F00000001CC0307CC0E1CCC387004
:100D6400CC607FFF7F00CC0000CC000000007FFF40
:100D74007F600060600C7F3FE700003300603770E5
:100D84003FEC1F00000003CC070E001C3800307F2E
:100D9400CE7F7073606037703FEC1F0000007FFFF0
:100DA4007F00660000CC00018801030003060006F2
:100DB4000C000C0000000F8C1F38E630306E381F1A
:100DC400CE3F7073606037703FEC1F0000001FCE91
:100DD4003F7073606037703FFF1F006E0001C803EF
:100DE4001F001E0000000000000000000E000E0E98
:100DF40000000000000E000E0E00000000000000C5
:100E0400000000000E000E0E00000000000E000E98
:100E14000E000606000C00CC010380070E001C38EF
:100E240000381C000E07080301CC0000000000007D
:100E340000000000000E3F3FE000000E3F3FE000D6
:100E44000000000000003000381C000E07080301F9
:100E5400CC010380070E001C3800300000001F8CFA
:100E64003F70E66060EC01038007060006060000A0
:100E74000600060000001FCE3F306B676FBB6D6D30
:100E8400BB6D6DBE6F67C0703FCC0F0000000600E5
:100E9400060F000F0F081919881930CC3F3FC660A0
:100EA4006066600000007F087F61CC6060CC617F79
:100EB4008C7F60E660606E607FC87F0000000F8CEE
:100EC4001F38E630600060600060600060306E389B
:100ED4001FC80F0000007F087F61CC6060666060FF
:100EE400666060666060CC617F807F0000007FEE9A
:100EF4007F6000606000607F887F600060600060E9
:100F04007FEE7F0000007FEE7F6000606000607F06
:100F1400887F6000606000606000600000000FCEA9
:100F24001F38603060006063EE636066603066386E
:100F34001FEE0F0000006066606066606066607FA0
:100F4400EE7F6066606066606066600000001F8817
:100F54001F06000606000606000606000606000632
:100F64001F881F0000000066000066000066000085
:100F74006600006660606C703FC81F000000606E11
:100F84006061C86367006E7C007C6E0067638C617F
:100F940060E6600000006000606000606000606007
:100FA40000606000606000607FEE7F000000606EA3
:100FB4007070EE7979E66F6F66666666606066608B
:100FC4006066600000006066707066786C666C66CF
:100FD400666663666361EE6060E6600000000F08A9
:100FE4001F39CC3060666060666060666030CC3902
:100FF4001F800F0000007F8C7F60E6606066606089
:10100400EC7F7F80606000606000600000000F087B
:101014001F39CC3060666060666060666333CC39CB
:101024001FE60F0000007F8C7F60E66060666060F2
:10103400EC7F7F8067638C6160E6600000001F8C3A
:101044003F70E6606000703F8C1F00E600606E70C9
:101054003FC81F0000003FCC3F06000606000606FE
:10106400000606000606000606000600000060668C
:1010740060606660606660606660606660606C3078
:101084003FC81F000000606660606C3030CC3019CF
:10109400881919800F0F000F060006000000606613
:1010A4006060666060666060666666666F79EE7052
:1010B40070E66000000060666030CC3019800F0676
:1010C40000060F081930CC306066600000006066CE
:1010D4006030CC301988190F000F06000606000690
:1010E4000600060000007FEE7F00CC0001800306AE
:1010F40000060C00183000307FEE7F0000001F88CF
:101104001F180018180018180018180018180018CC
:101114001F881F00000000004060007038001C0E93
:101124000007038C0100E7000030000000001F8866
:101134001F018801018801018801018801018801DA
:101144001F881F0000000200070F8C1D38E7706025
:10115400300000000000000000000000000000005B
:10116400000000000000000000000000000000007B
:101174000000007FFF7F000007070007060006034A
:10118400000000000000000000000000000000005B
:1011940000000000000C1F3FE6001FEE3F60666089
:1011A4007FEE3F00000060006060006060086F7FB9
:1011B400CE70606660606E607FC87F0000000000D3
:1011C4000000000000081F3FC670600060600670E9
:1011D4003FC81F00000000660000660000661F3F55
:1011E400EE716066606066703FEE1F0000000000F4
:1011F4000000000000081F3FC6707FEC7F60007095
:101204003FC81F00000007880F1C00181800187F33
:10121400007F1800181800181800180000000000BB
:1012240000000000000E1F3FE670606E703FE61F76
:10123400006E003FC83F60006060006060006F7F28
:101244008C7160CC6060CC6060CC600000000000F9
:101254000006000600000E0E000606000606000644
:101264001F881F000000000000018801000803031C
:1012740088010188010188010188191F800F30004D
:10128400303000303008313380373E003E37083389
:1012940031CC300000000E000E06000606000606E3
:1012A40000060600060600061F881F000000000056
:1012B400000000000008597FCE7F66666666666699
:1012C40066666600000000000000000000083F3F62
:1012D400CE303066303066303066300000000000BA
:1012E4000000000000081F3FCE70606660606E70F2
:1012F4003FC81F00000000000000000000087F7FBE
:10130400CE6060666070EC7F6F806060006000009B
:1013140000000000000E1F3FE67060666070EE3F44
:101324001F6600006600000000000000000C373F4C
:10133400E63830003030003030003000000000006B
:101344000000000000003F7F80607F083F018801AB
:101354007F803F00000000001818001818007F7FED
:1013640000181800181800181F880F00000000004B
:1013740000000000000660606660606660606E7079
:101384003FE61F000000000000000000000660604F
:101394006C3030C81919800F0F00060000000000DF
:1013A400000000000006666666666666666F6C3F4F
:1013B40039C810000000000000000000000C60713B
:1013C400C83B1F000E1F083B71CC600000000000EA
:1013D40000000000000C3030C81919800F0F0006FF
:1013E40006000C0C0018000000000000000C7F7FB9
:1013F400800306000C1800307FCC7F00000003CC73
:10140400070E000C0C000C1C00381C000C0C000C0B
:101414000E0C0703C00006000606000606000600C0
:1014240000060600060600060600060000003C0052
:101434003E070003030003038C010380030300033E
:1014440007003E3C00000000001C6C366380000076
:101454000000000000000000000000000000000088
:101464000000000006000F198C306066607FEE7F7C
:1014740000000000000000001E0060077E0700F06E
:101484001EF060F77EF7FBDE1F00E007FF0700F8A1
:101494001FF8E0FFFFFF00000F00E002EF020078FA
:1014A4000F78E07AEF7AF7BD1F00E007FF0700F836
:1014B4001FF8E0FFFFFF23000002000010000005FA
:1014C4000000FE0500182800FE0400182400F90F8F
:1014D40000F80F0070001F71802372802A731115A9
:1014E40074111C75151B76151A77181C78152105AF
:1014F4000100FF000000013F2B0200100721000043
:101504000100072300100000FD30000733001130F4
:1015140068FF0000E50080000100010001020004F2
:101524000330100400000802020900000A00000C45
:1015340000000D00000F0000100000110700120051
:1015440000130000FD500010B01B110700FD5000F7
:10155400121E01FD500013001F291F00FD50002022
:101564000000210000FE01002B0C00FE00002B20D7
:10157400003000003106033200023507013604044E
:101584003706063805013907073C00063D070850B1
:10159400000051EF00520000533F01FE01006000C3
:1015A400A7FE00006000276101006A0000800000BF
:1015B4008100008200008300008400008500009008
:1015C4001000920007930700953F039700009800CE
:1015D40000070100FD5000072100072300FD500013
:1015E400077301FF0000000000000000F800000085
:1015F400FF000000FF0000007F80001E0F80007FBE
:10160400E7C0007FFFE0003FFFE00007FFC00001EC
:10161400FFC00001FF800001FF0003FFFE0007FF81
:10162400FC0007FFF00003FFF00003FFFE00001FB3
:10163400FFC001FFFFF001FFFFF801FFFFF8007F8B
:10164400FFF80007FE00003FFF00007FFF80007FDF
:10165400FF80007FC100001FE000001FF000001F9A
:10166400F000000FE0000007C0000007C000000702
:10167400C000000780000003000000030000000217
:10168400000000000000000000000000E000000076
:1016940000000003900000000000000E180000008D
:1016A4000000003808000000000000C0180000001E
:1016B400000003807000000000000C01C000000165
:1016C4008006300700000003C00F401C0000000625
:1016D400E01DC0700000000C3039C1C000000018CB
:1016E4001871C7180000001C0CE1DC7C0000000E1F
:1016F40007C3F1C4000000070386070600000003C7
:10170400800E1C0200000001C01C30030000000019
:10171400E03818010080000070700FC183C0000021
:1017240038E003E08E6006001DC00020FC200F009E
:101734000F8000307030198007000010003030C076
:101744000000001800E060600000000803806030C2
:101754000000000C0E003018000000043800180CC3
:1017640000000006E0000C060000000380000603F1
:101774000000000000000301800000000000018060
:10178400C000C0C060C030C030C030C030C030C045
:1017940030C030C030C030C030E030703018300C51
:1017A40030043FFC3FFC2564002B003E3E004944CE
:1017B4003D00202047433D002D2D2D2D00204C00C1
:1017C400533F000058313939313030004D42005018
:1017D40053004D31004F31005350004350004459E1
:1017E4000062757379004D50002564002020004389
:1017F4003F003A20004D49004D42004D43004D50FA
:10180400004D4C004F4E0000253032580025303436
:101814005800253664002533642E253032640025B3
:101824003564002564002532640025336400444493
:1018340000004B230042530042210042460054233F
:1018440000544F004952004D5A0042510042520088
:10185400435300565300564300494C00426600006F
:101864004B230054230042450043450042410044B9
:10187400530043420023502241534349492D492FE9
:101884004F222C22312E3030222C323030382D3061
:10189400312D30313B0023482245636F222C223105
:1018A4002E3030222C323030382D30312D30313B37
:1018B4000023532245636F222C22312E3030222CF8
:1018C400323030382D30312D30313B00504F005004
:1018D4004632333B5055002564002B302B303B00FF
:1018E40025640025303258002E3030004F4E000061
:1018F4006D696B726F746F756368000001002D4E23
:10190400414E00000100E40E00190000F894EE2797
:10191400ECBBF1E0F5BFE5BFE0936C00F8E1F1BD8D
:10192400E1BD8DE0A2E0BB27ED938A95E9F780E065
:1019340090E1A0E0B1E0ED930197E9F7E8E0F9E187
:1019440085919591009761F0A591B59105901590B9
:10195400BF01F00105900D920197E1F7FB01F0CF73
:10196400EFEFEDBFE0E1EEBFC0E0D3E00C94F01583
:101974000A9902C0E1E00895E0E00895A0913F0CC7
:10198400A13031F40E94856C0E94CC670E94966C51
:101994000895A0913F0CA13031F40E94856C0E94FF
:1019A400A06C0E94966C0895E881E03011F01C9AB6
:1019B40001C01C9832C00E94A46C0E94A46C0E94B6
:1019C400A96CEFE3F0E00E94AE6C08951A93A09125
:1019D4000403A43081F4E0910F04E093100410E0B8
:1019E400183048F4ABE01A9FF001E659FC4F0E940E
:1019F400B46C1F5FF5CF3FC0A0910403A43039F449
:101A0400E881E0931004E0E0E0930F0406C0E8816D
:101A1400E0930F04E0E0E0931004219608951A93F4
:101A2400A0910403A43019F110E0143000F50E94D1
:101A3400B86C3196E491EA93DFDFE0E0E0931004C0
:101A44000E94C16CEBE0F1E00E94CB6C0E94CB6C75
:101A5400FA93EA930E94B86CE491EA930E94B86CFA
:101A640032960E94D06C0E94F6431F5FDECF0E9424
:101A7400D36C0E94D86C199108952A970E94B47D62
:101A840030E010E000E047ED50E028E0E091190C70
:101A9400E03019F020E149E650E0321710F00C94E0
:101AA400920D0E94DC6CE130A0F10E94DC6CE03805
:101AB40070F0EEE00E94E26CEAEAF7E1FA93EA934E
:101AC4000E94DC6CEF70EF5F0E94EA6C09C0ECE0EE
:101AD400EA9392DFE8E7F2E004900E82E0E0EF831D
:101AE4000E94C16CA02FB0E0E7E3F0E00E942E7BDF
:101AF400E40FF51F0E94CB6CFA93EA93EDE2F0E059
:101B0400FA93EA930E94DC6CEA930E94A46C0E940C
:101B1400F46C1F5F143011F410E00F5F3F5FBDCF12
:101B24000E94D36C0E9486490E94BB7D61960895F1
:101B34000E94FA6CECE0EA935FDFE2ECF3E00E94CF
:101B4400B46CEBE0EA9358DF0E94FE6C0E94036DD4
:101B5400EAEAF0E00E94086DE0913C0CF0913D0C43
:101B6400E491EA93E0913C0CF0913D0C31960E9493
:101B74000F6D0E94F64301E00E94126D0E94156DE4
:101B840011F00F5FF9CF0E94236D031718F4E0E002
:101B9400E093C0050E94236D11E00E942A6D0E940B
:101BA400156D11F0153008F021C00E94FE6C0E94E2
:101BB4002D6DE0E4F0E00E942E7B3496FA93EA93D4
:101BC400E2EEF0E00E94086D0E942A6D0E94306DE2
:101BD400E491EA930E942A6D0E94306D31960E942E
:101BE4000F6D0E94F6433F5F1F5FD7CF0E94D86CF2
:101BF4000E94BD7D30C427970E94B47D22E354E047
:101C0400A0910403A43011F426E453E010E014304E
:101C140010F00C94580E00E0051710F00C94560EBA
:101C2400E12FEE0FEE0FE00F3E2F0E942A6D0E946F
:101C34003C6D3196E4910E94E26C0E942A6D0E94F0
:101C44003C6D3296FA93EA930E949B69ED85E030ED
:101C540039F4AF81A13210F4E0E0EF83E0E0E887EB
:101C6400A02FBB27E22FE85FF0E00E942E7B38967E
:101C7400FA93EA930E942D6DEAE3F0E00E942E7B32
:101C8400E55BFF4F0E94416D0E94CB6CFA93EA938F
:101C94000E942A6D0E943C6DE491EA930E94A46C18
:101CA4000E94F46C0F5FB8CF1F5FB1CF0E94D86C55
:101CB4000E94BB7D2E96089522970E94466DA13006
:101CC40059F40E944B6DABE2B1E00E94597B2E2F78
:101CD40057E1E2ECF0E008C00E944B6D0E944F6DAA
:101CE4002E2F53E0E7EEF0E0EE83FF830E94546D65
:101CF400A0911908A13081F4E9ECF0E00E946B6D29
:101D04000E94726D0E94776DEBE2EA93EDEAF7E1CF
:101D14000E94D06C0E94F643E3E0F0E00E946B6DF9
:101D24000E947D6D0E94776D0E94826D0E94866D77
:101D34003F5FE091C10BAFEE0E94387BF0E0EE8391
:101D4400FF8311E0E091C20B1E17C0F500E0E091A3
:101D5400C10B0E1788F50E948C6D59F10E94936D8A
:101D6400E09310040E94126DAE81BF810E942E7B0D
:101D740033960E94416D0E942D6D0E942E7BDF01DF
:101D84000E949D6D0E94A06DEA85FB853497FA93AD
:101D9400EA930E94776D0E94826D0E94866D3A9349
:101DA4000E94C720EF3F29F0ADE05A9FF0010E9446
:101DB400A56D3F5F0F5FCBCF1F5FC4CF0E94D36C75
:101DC4000E94D86CCAC022970E94B47DE2E5F7E075
:101DD400EE83FF8340E0443190F4AE81BF811196DD
:101DE4000E94AD6D1396EFEFEC93AE81BF81EC933F
:101DF400EE81FF813496EE83FF834F5FECCFE09159
:101E0400C10BA0EF0E94387B2E2F0E944B6DA0E4E3
:101E1400B1E00E94597B5E2F0E94546D21FE23C0C5
:101E24000E94B26D0E94B26DEFEAF0E0FA93EA9379
:101E34000E94B76D0E94826D0E94866D0E94BD6DE6
:101E4400E6EBF0E0FA93EA930E94B26D0E94726DA1
:101E54000E94B76DEFE7EA93EFEAF7E1FA93EA93AA
:101E6400E0E0F0E011C00E94B26D0E94B26DE8EEB5
:101E7400F0E0FA93EA93E52F0E94C46DFA93EA9393
:101E84000E94826DEAE8FBE0FA93EA930E94F6432B
:101E94003F5F11E0E091C20B1E1710F00C94A90FE4
:101EA40000E0E091C10B0E1710F00C94A70F0E94F4
:101EB4008C6D11F40C94A40FA0919A0BE0E8EA2322
:101EC400E03821F0A091E20BA23019F40E94936D46
:101ED4000AC00E94C76DE03011F4E0E001C0E8E000
:101EE400E0930F04E7E0E0931004A02FBB27E22F58
:101EF400F0E00E942E7B3396FA93EA930E949D6D44
:101F04000E942D6D0E942E7B3396FA93EA930E94D1
:101F1400776D0E94B76D0E94826D0E94866D4E2F70
:101F2400A0911E08E32F0E94CC6DEA0FFB1F438390
:101F34003A930E94C720EF3F29F0ADE04A9FF00199
:101F44000E94A56D3F5F0F5FACCF1F5FA3CF0E94C0
:101F5400D36C0E94D86C0E9408360E94BB7D2896E0
:101F64000895E1E0E0930D04E2E0E0930E04E0E084
:101F7400E0931004ECE0E0930F04EAEDF3E00E9438
:101F8400B46CEAE0E0930F04EEECF3E00E94B46C6E
:101F94000E94864908951A93A981A43029F4A0E0E7
:101FA40021FCA1E0A03009F426C0E9810E94D36D90
:101FB4000490E9810E94D96DE491A02DAE1BA2503A
:101FC4001A2F0E94BD6DE4EBF0E0FA93EA93EB81E3
:101FD4000E94D96D0E94E17B3296FA93EA93EAE378
:101FE400F0E00E94E16DEFE7EA93EFEAF7E10E9487
:101FF400D06C0E94F6431881229608951A930A938E
:102004000E94E86D0E9477180E94C76D0E2FEEE4BF
:10201400F3E00E94E17B33971E2F0E94A46C0E9480
:10202400A46C0E94A96C0E94ED6D0A930E946D4BF2
:10203400ECE3F0E00E94F26D0E94F246E2E0E093ED
:102044000E04E091980BEF70E09310040E94F96D78
:10205400EFE0E0931004AA81A13051F40E94016ED4
:102064000E94036D0E94D746ECE8F0E00E94066EE1
:1020740021FE0DC0E4E0EA938EDFE6E5F3E00E9482
:102084000A6EE8E5F3E00E940A6E0E94A1499EDC14
:1020940080C0E8810E94D96D0E940A6EEA810E9484
:1020A400D36D0E940A6E0E942F47E881EA9373DF82
:1020B400C0C11A930A93EC81EA93EBDF1AEEEC8128
:1020C4000E94D36D0490EC810E94D96DE491A02DFF
:1020D400AE1BA2500A2FAC81A43029F4A0E021FC4D
:1020E400A1E0A03009F409C01EEAAA81BB811B96B5
:1020F400E0E0EC93EC81EA934EDF0E94936DE09371
:102104001004EC810E940F6EFF93EF930E94B26D56
:10211400EE810E94D96D0E94E17B31960E94E16DAF
:102124000E94126DFA93EA93EC85E058EA930E94B8
:10213400A46C0E94156E0E94F643AF91BF91EC937C
:10214400EC810E94D96D0E940A6EEE810E94D36DCB
:102154000E940A6E0E94A14919810881259608955A
:102164000E941A6E0E944F6D8F010E94A46C0E94FF
:10217400A46C0E94A96C0E941D6E0E94016E0E94B4
:10218400D746EA81EA930E9477180E94F96D0E946B
:10219400246E19810881239608950E941A6E0E9464
:1021A4004F6D8F010E94A46C0E94A46C0E94A96CC4
:1021B4000E941D6E0E94016E0E94D746EC81FD8133
:1021C4000E94066EAA81BB810E94AA7D24F4A030DD
:1021D400E0E1BE070CF006C0EA81FB81FA93EA93C2
:1021E4000E949241AA81BB81A130E0E1BE0724F0A4
:1021F400A030E1E1BE070CF00AC0A6EEBBE0EA8124
:10220400FB81E150F0410E942E6E0E94366E0E94C6
:10221400246E19810881269608950E941A6E0E94E0
:102224004F6D8F010E94A46C1A930A930E94A149D6
:10223400E0E0E0933E0C099119910895E881EA9356
:102244000E9477180E94951FE03051F10E943C6E65
:102254000E94A46C0E94406E0E94F96D0E94446E1C
:10226400E881EA930E941521E8830E94486E3B9717
:1022740034F00E94486E0E94536EE9E40BC0A3EE52
:10228400B6E00E94576E0E945A6E0E945F6E0E94D2
:10229400646EE3E7EA930E947146E2E0E0930E0481
:1022A400C8C00E940C69E0E0E0930F04A09104030D
:1022B400A43019F4E6EEF3E002C0E2EFF3E0FA939F
:1022C400EA930E94D64308950E94FE460E940C6938
:1022D4000E945F69E1E0E0930D040E943C6EE6E039
:1022E400F0E00E94686EE6EBF2E00E94066E0E9447
:1022F400A46CE7E0F0E00E94686EE2EBF7E10E9474
:10230400066E0E946C6EEA930E949F41E6EBF7E131
:102314000E94066EE0910403EA930E949F4108958F
:102324002A971A930A930E94A46C0E94A46C0E9498
:10233400A96CE4E6F0E00E94AE6C00E010E0153019
:10234400B0F4053020F40E94716EE03009F40DC041
:102354000E94A46C0E94126D0E94686E0E94786EA6
:102364000E94716E0E947D6E0F5F1F5FE8CF0E9416
:102374007F6E0E94D746EAE8F2E00E94066EE09182
:10238400430CEA930E949F41E091420CEA930E941D
:10239400A5410E94FE6C0E94016E0E94D746EEE8A1
:1023A400F2E00E94066EE0912606EA93E5E0EA93E5
:1023B4000E945541E091190CE03079F10E94FE6CC5
:1023C400E2E0F0E00E94686EE09128060E94826ECE
:1023D4000E94B26D0E94D746E0912806E295EF7004
:1023E400E695E695AE2FE0912906EE0FEE0FEA0F83
:1023F4000E94826E0E94036D0E94D746E0912906D6
:10240400E295EF70AE2FE0912A06E295E07FEA0FA5
:10241400EA93E6E0EA930E945541198108817DC15F
:10242400E881E064E7B9369A349BFECF349AE4B18C
:10243400F5B121960895E881F981AA81BB81AE178F
:10244400BF071CF4EA1BFB0B06C0A881B981EA8113
:10245400FB81EA1BFB0B2496089528970E94B67D06
:10246400EFE0E0936100E1E00E94886EE5E00E9405
:102474008F6E0E94966EE0936F05F0937005E09165
:102484007B05F0917C05E0936D05F0936E05E1E02A
:10249400EA93C6DFE0937B05F0937C05EFE0E093DD
:1024A4006100E8E00E94886EEAE00E948F6E0E945C
:1024B4009B6EE0936B05F0936C05E0917905F091C8
:1024C4007A05E0936905F0936A05E0E0EA93A8DFF2
:1024D400E0937905F0937A050E949B6EA0916B05B9
:1024E400B0916C05EA0FFB1FA0917905B0917A05B4
:1024F4000E94A06E8F010E94966EA0916F05B0910C
:102504007005EA0FFB1FA0917B05B0917C050E942A
:10251400A06E9F01E0916B05F0916C050E94A76E7F
:10252400FF93EF930E949B6E0E94A76EAF91BF91A1
:10253400EA0FFB1FFF93EF93E0917905F0917A0581
:102544000E94A76EAF91BF91EA0FFB1FE093750540
:10255400F0937605E0916F05F09170050E94AD6EE1
:10256400FF93EF930E94966E0E94AD6EAF91BF9160
:10257400EA0FFB1FFF93EF93E0917B05F0917C053D
:102584000E94AD6EAF91BF91EA0FFB1FE0937705F8
:10259400F0937805A0917505B0917605E4E1F0E03B
:1025A4000E94007B0E2EA0917705B0917805E4E19E
:1025B400F0E00E94007BE02919F00E94A645ABC020
:1025C400009371051093720520937305309374057D
:1025D400A0916405A63428F4E0916405EF5FE093CC
:1025E40064050E94B36E989724F40E94B86E98977D
:1025F4000CF00EC0A0916405AA3019F4E1E0E09358
:102604006105A0916405A83219F4E2E0E093610544
:102614000E94B36E999724F00E94B86E99970CF4B7
:102624007AC0E0916705EF5FE09367050E94BD6E95
:102634000E94B36E0E94C26E0E94C96E0E94CE6E4A
:102644000E94337B7F936F93FF93EF93A2E0B0E0FC
:102654000E94FC7B0F010E94BD6EDF01F001EA1BAA
:10266400FB0BAF91BF918F919F910E94D76E0E94F7
:10267400C96E0E94DC6E0E94B86E0E94C26E0E94F7
:10268400E16EAC81BD818E819F81EFE3F1E060E07A
:1026940070E00E94337B7F936F93FF93EF93A6E0E8
:1026A400B0E00E94FC7B0F010E94DC6EDF01F001B0
:1026B400EA1BFB0BAF91BF918F919F910E94D76E44
:1026C4000E94E16EE0911204E03049F4E885F98556
:1026D400E0935905F0935A05EC81FD810AC0EC8121
:1026E400FD81E0935905F0935A050E94CE6E0E9435
:1026F400C87AE0935B05F0935C05E0915905F0918D
:102704005A05FA93EA93E0915B05F0915C05FA931C
:10271400EA930E942E450E94BD7D2C9608951A933B
:102724000E94FE46E2E0E0930E04E2E3F0E00E9441
:10273400CB6C0E94E66EEAE7F2E00E94066EE4E1EA
:10274400EA930E94FE40E0E9F1E00E94EA6EE4E1CF
:10275400EA930E94FE40A0916705A13010F0A8956D
:10276400FACF10E0143010F00C941214E2E0E0936D
:102774000D040E94EE6EDF010E940A6EFD01329686
:102784000E940A6E0E94F2460E94EE6E3496E49114
:10279400EA930E947146E1E0E0930D04A09167057D
:1027A400AF3110F4A895FACFEAE0EA930E94FE4014
:1027B4000E94EE6EDF0135960E94E17BBF01FD01B0
:1027C4000E94F46EDB010E940C7C0E94FB6E0E944E
:1027D4002D6DE8E2F0E00E942E7BE65AFF4F0E9446
:1027E400E66E0E94EE6E0E94F46E0E94536EA091FB
:1027F4006705AE3110F0A895FACF0E94EE6EDF01A6
:102804000E940A6EFD0132960E940A6EE8E1F0E031
:10281400FA93EA93E8E2F0E00E94AE6C1F5FA2CF65
:102824000E94FB6EEAEFF0E00E94E66EE6E8F2E05A
:102834000E94066EE0EDF7E00E94EA6E0E94FE46FA
:1028440067C10E94006F0A93E4E6E2BF78940E9495
:10285400F04403DEE6B3AFEFEA27E093430CE091E4
:10286400420CE03009F002C0E091430CE0933008E0
:10287400A2E6BBE00E940F6FE091620BE77031F4B7
:10288400A0910A04E0E4EA27E0930A04E091620BD1
:10289400EF7131F4A0910A04E3E8EA27E0930A0413
:1028A4000E9490660E94B421E0913108E030C1F0AA
:1028B400E2B3EF700E2EA0911408B0911508EFE06A
:1028C400F0E0AE27BF27EA23FB230E94E17AE02948
:1028D400E2BBE0911408E07111F41D9A01C01D9847
:1028E4000991199115C00E94006FE6E0E4BDE0B1C2
:1028F400E295EF70AE2FE0916300E071EA2BE06E99
:102904001E2F0E94ED6D0E948B210E946A66199110
:10291400E991EFBFF991E991B991A99199918991BF
:1029240079916991F9901990099018950E94906590
:102934000E941A660E9410510E94D31E08951A9391
:10294400A8950E940443E13011F00C940115E09124
:10295400C605E1501E2FA091C505A13021F40E94A7
:10296400156FE03009F40CC0ADE01A9FF001E15F8F
:10297400FC4FBF01E081E260DB01EC930E941C6F1D
:10298400A091C505A23011F0A43089F40E94156FFE
:10299400E093DB050E94216F31F0FD01E15FFC4F04
:1029A400E081E27009F403C01A930E942A6FA09197
:1029B400C505A33019F41A930E94BB27A091C5053D
:1029C400A53029F4E091C605EA930E94E827A09176
:1029D400C505A730A1F4E0E0EA93E091C605EA93C7
:1029E4000E944A181E2F1F3F51F0E0E0EA930E9414
:1029F400FE4010932E06E12FE058E0932D06E0915F
:102A04000A04E07841F1E0910A04EF77E0930A04C4
:102A14000E94CA49E0910A04E07131F0E0910A048D
:102A2400E270EA930E94D845E0913108E03021F049
:102A3400E4EEEA930E94F266A0913F0CA13021F4E7
:102A4400A0911908A43009F406C0E0EBEA930E94AF
:102A5400F266E093420CA0913E0CA13039F4E0916F
:102A6400400CF091410C0E942E6F09F401C0D5DB9B
:102A74005DDF4EC01A930E94FE46E1E0F0E00E9442
:102A8400D06C0E94D74610E00E94386F0E94A46C5C
:102A94000E94ED6D0E94D746E0912008E03049F491
:102AA400E6E6F2E00E94066E0E943E6F0E94646EAB
:102AB4001E5FA0912008A130F0F0E0912008E150C1
:102AC400EA930E94A618A091B30BAD3229F40E9498
:102AD400476F0E94A67D79F0E3EBFBE00E94366E1F
:102AE400E6E0F0E0FA93EA930E94546F0E94476F85
:102AF4000E94646E1E5FE0912008EF5FE09320085F
:102B04001C3020F4A0912008AB3008F001C0BECFE7
:102B1400199108951A930E94FE46E981E03019F450
:102B2400E0E0E0931E08A981A230A9F410E0A0918E
:102B34001E08A13010F01C3008F00DC0E0911E08F2
:102B4400E150E0931E080E94586F19F40E94666FCA
:102B540009F01F5FECCF0E94386F10E00E94A46C54
:102B64000E94ED6D0E94D746A0911E08A03408F57E
:102B74000E94586F19F40E94666FD1F0E0911E080C
:102B8400EA930E9477180E94F96D0E94A46C0E9437
:102B9400546F0E94716F0E94536EE8E7EA930E949B
:102BA40071460E94446E0E94766F0E94646E1E5F9E
:102BB40005C0ECEBF7E10E94066E1E5FE0911E0873
:102BC400EF5FE0931E081C3020F4A0911E08A1348E
:102BD40008F001C0C3CF188122960895E0E0E5BF54
:102BE400E0936D00E0936C00EBBBEFEFEABBE0E039
:102BF400E8BBE7BBE5BBEFEFE4BBE0EFE2BBE1BB67
:102C0400E0E2E3B9ECEBE2B9E0E0E0936200E093E8
:102C14006100EFE0E0936500E0936400E0E0E0BF72
:102C2400E7E0E3BFE4E6E2BFE0E0E1BFEFBDEEBD15
:102C3400EDBDECBDE7BDE6BDEBBDEABDE9BDE8BD5C
:102C4400E0937900E0937800E3E0E5BDE6E0E4BDDD
:102C5400E0E0E3BDE0938B00EAE0E0938A00E0E08B
:102C6400E0938900E0938800E0938100E093800082
:102C7400E2E1E0938700E4E3E0938600E0E0E093A0
:102C84008500E0938400E0938300E0938200E09366
:102C94006A00E0E3EABFE0E4E9BFE8BFE1E4E7BFDC
:102CA400E0E0E0937D00EBB9E8EDEAB9E6E0E0931B
:102CB4009500E0E0E0939000E7E6E9B9E0E0E09316
:102CC4009B00E8EDE0939A00E6E0E0939D00E0E0ED
:102CD400E0939800E3E3E0939900E0E8E8B9E0E0EA
:102CE400E0BDE0E4E7B9E7E8E6B9E0B5EF7EE0BDD2
:102CF400E0E2E0937000E0E0E0937200E4E4E0934B
:102D04007400EFE1E1BDEFE0E1BD0E941B5E0E94B3
:102D1400094B0E94C9457894E1E0EA930E94D60CDD
:102D24000E946C6EE53128F0A9E0B0E0E0E00E947A
:102D3400147CCADA21E030E0E0EEEA930E94F26605
:102D4400E09331080E947F6F3F5FA0913108A43562
:102D540011F03A3008F001C0EFCF30E0E0EBEA9335
:102D64000E94F266EF3F19F0E1E0E0933F0C0E940D
:102D74007F6F3F5FA0913F0CA03011F43A3008F010
:102D840001C0ECCF0E94016E0E94FE6C0E94D746E7
:102D9400E2E9F2E00E94066EA0913108A43551F4F4
:102DA400E2EEEA930E94F266E0933108EA930E940D
:102DB40071460DC0E0E0E0933108E8E9F2E00E94DA
:102DC400066EE0E0E0939800E7E6E0939900A091B6
:102DD4003F0CA13021F4E1ECF7E10E94066E9FD094
:102DE400E03079F40E94016EE9E0F0E00E94686E40
:102DF400ECE9F2E00E94066EE8E9F2E00E94066E59
:102E040020E00E94BD6E0F01A2E0B0E00E94FC7BB6
:102E14000E161F0654F40E94DC6E0F01A6E0B0E00B
:102E24000E94FC7B0E161F060CF079DC203071F436
:102E34000E94016EEAE0F0E00E94686EE0EBF2E0CE
:102E44000E94066EA8950E94826FFCCF0E94EF3606
:102E54000E94016EE9E0F0E00E94686EE4EAF2E0AC
:102E64000E94066E0E94251BE03019F0EAEAF2E0A7
:102E740002C0E6E8F2E0FA93EA930E948846E09101
:102E84003B0CEA930E94A541EBE4EA930E9471464D
:102E94000E94A266E1E0EA930E94FE4000E010E096
:102EA4000436E0E01E0724F40E941A66E03009F0BC
:102EB40005C00E947F6F0F5F1F4FF2CF0436E0E022
:102EC4001E072CF0A0916705AF3108F028DC37DD30
:102ED4000E9462320E94571DFACFFFCF0E94856F75
:102EE40017FD02C0103011F4E0E060C3E12F5EC3AF
:102EF4000E94856F17FD10E01A3008F41F5F0E94CE
:102F0400926F54C30E94856F17FD02C0103011F4F4
:102F1400E0E04CC311500E94926FE1E047C31A9362
:102F24000A9310E0E4E6F0E00E94EA6EA8950E949D
:102F34000C67E03021F4E0EA0E949D6F09F002C0C2
:102F440001E001C000E00E941D671F5F003011F422
:102F5400153008F001C0E6CFE02F099119910895CA
:102F64000E94A26F4AC40E94A26F0E94AF6F08958C
:102F7400A881B9810E94AA7D24F4A83EE3E0BE079B
:102F84000CF005C00E94B26F0E947F6710C3E0E09E
:102F94000EC3EA81E03011F4EFEFEA83A881B9812E
:102FA4000E94AA7D24F4A83EE3E0BE070CF006C00C
:102FB4000E94B26FED81EA930E94AB675AC10E94EE
:102FC400B67D20E030E0283EE3E03E077CF4A8959F
:102FD4003A932A93CDDF1E2F1F3F29F0EFEFEA9398
:102FE4003A932A93D6DF2F5F3F4FEDCF0E94BD7DEA
:102FF4004DC01A930A93E0E0F0E0E093440CF093A0
:10300400450CAA81A03458F40E94BB6FE55FFB4FC6
:103014008F010E94C26FE4E4FCE00E94CB6FE09158
:10302400440CF091450C23C11A931FEF1F5F1A93B0
:10303400E0DFA981BA81EA17FB0711F0113408F027
:1030440001C0F4CFE12F188114C11A930A93A091FF
:10305400C10BE091C20BEA9FF001A0911E08EA0F98
:103064000E2F013408F00FE310911E08101758F4C6
:103074001A93BFDFAA81BB81EA17FB0711F4E12F82
:1030840003C01F5FF3CFEFEF1981088124960895E1
:103094000E94B47D10E0103418F50E942D6DE8E212
:1030A400F0E00E942E7BE050FC4FAF01E0EAEA938F
:1030B400FA0170960E94CF6FEC713E2FE0EAEA931A
:1030C400FA013F960E94CF6F0E2FEF81E31719F498
:1030D400EE81E01709F002C0E12F03C01F5FDBCFD0
:1030E400EFEF0E94BB7D289608951A930A93E0910E
:1030F400890BAA81EA17C1F0A03468F40E94BB6F5F
:10310400E050FC4F8F010E94D36F0E94CB6FEA8185
:10311400E093890B09C0EFEFE093890B0E94DE6F07
:103124000E94E36FE093940BA2C01A930A930E9447
:10313400BB6FE050FC4F8F01AA81A03420F40E94A1
:10314400D36F0E94AF6F93C01A930A93E091B20BAE
:10315400AA81EA17A1F00E94ED6F40F40E94F96F72
:103164000E94CB6FEA81E093B20B09C0EFEFE093CA
:10317400B20B0E9404700E94E36FE093BD0B77C012
:103184001A930A930E94ED6F20F40E94F96F0E9433
:10319400AF6F6DC01A930A93E091340CAA81EA17B9
:1031A40051F10E94097008F50E94C26FE5E3FCE04A
:1031B4000E94CB6FEA81E093340CE0E0E0932B06AD
:1031C400A091360CA13020F0A091360CA83008F064
:1031D4000BC0A8EDBBE0E091360C0E941370AE0F5B
:1031E400BF1FEC91E0932B0606C0EFEFE093340C85
:1031F400E0E0E093350C3BC01A930A930E940970F7
:1032040030F40E94C26FE5E3FCE00E94AF6F2FC070
:103214001A930A93E0912F0CAA81EA17C1F00E9435
:10322400167070F4E0EAEA930E94036D1A930A930D
:10323400E0E3FCE00E94CB6FEA81E0932F0C07C02F
:10324400EFEFE0932F0C0E9420700E9470690FC072
:103254001A930A930E94167050F4E0EAEA930E94CB
:10326400036D1A930A93E0E3FCE00E94AF6F1981A7
:103274000881239608950E9420700E947069E88155
:10328400EF5FE093310C99C224970E94B47D0E94B1
:1032940027700E947069AA85A03490F5AB85A1308F
:1032A40020F0E0913B0CEA1708F407C0EB850E947C
:1032B40013700E942E700E944170EB85E03001F57E
:1032C400E0E0EE83EF83E887E98740E050E020E028
:1032D40030E0E0913B0C0E94467084F4F9010E94B6
:1032E4002E700E9441700E94716F4E0F5F1F0E94EA
:1032F400766F0E944B702F5F3F4FEBCF0E9456704A
:103304003DC11A930A93AB81A13020F0E0913B0CAC
:10331400EA1708F41CC0EB810E9413700E94E57A3E
:103324000E94E17ADF01EA810E946770E8E0F0E040
:103334000E942E7BE050FA4E8F01E0EAEA930E944D
:10334400FE6C1A930A93EDE1FCE00E94AF6F1981C1
:1033540008810C949E1E0E94B67DEC810E946B70C5
:10336400E83119F40E94BD7D15C20E947070309737
:1033740029F00E9470700E947570EC830E94891F6E
:103384000E2F10E0101710F00C940B1A0E94797095
:103394007BDFAFE1BCE00E940F6FA091210CB091E4
:1033A400220C8091230C9091240C0E947E700E9428
:1033B400C37AE093210CF093220C6093230C709356
:1033C400240C0E9479709DDFE0EAEA93EE810E946A
:1033D4001370EE0FFF1FE050F04F0E94CF6FE270AA
:1033E400B1F4ED81E093250C0E947070309729F4BC
:1033F400EC81F0E0EF5EF84D02C00E947070E09343
:10340400260CF093270C0E9485700E948A701F5F1F
:10341400B9CF0E94BD7DBEC11A930A930E949070D9
:10342400ECE2F0E00E9497700E949B700E94A070F2
:1034340010E01034D8F41A9358DEE0912108EA938E
:103444001A9322DF0E94A970EA0FFB1F0F010E944A
:10345400A9700E94B170DF01CB010E94766F0E94B7
:10346400C37AD0010E94DC7B1F5FE3CFA0911908CF
:10347400A330B9F500E00031A0F50E94126D0E945E
:10348400B67069F510E01A3050F5E02FE05DEA936C
:10349400E4ECF7E10E94BB70E12FE05D0E94C27092
:1034A400E1F40E94C7700E94CE70EA0FFB1FFF93E5
:1034B400EF930E94CE700E94B1707F936F93FF933D
:1034C400EF930E947862AF91BF918F919F910E9478
:1034D400C37AAF91BF910E94DC7B1F5FD4CF0F5F93
:1034E400CACF10E01A3090F40E94CE700E94B170DE
:1034F400A0912808B091290880912A0890912B085E
:103504000E94C37A0E94A0701F5FECCF0C94171F17
:1035140024970E94B47DEA85EA936BDD9F01022E15
:10352400032A39F13A932A937FDD1E2F40E050E0BD
:10353400E0E0EE83EF83E887E987AA851A17B1F400
:10354400012F003498F40A9354DD2E173F0761F4D9
:10355400EB85EA930A9398DE0E94716F4E0F5F1F0A
:103564000E94766F0E944B700F5FEBCF0E945670E3
:1035740005C0EB85EA93EB85EA9386DE0E94BB7D6A
:103584002C9608951A93A895E0913B0CA981EA170B
:1035940068F00E9427700E94706910E0103430F4C3
:1035A400E981EA931A93ADDE1F5FF8CF1881229662
:1035B40008951A9311E0E0913B0CE11720F01A935F
:1035C400E1DF1F5FF8CF72C3E1E0E093350CE093D5
:1035D400360CF3C0A8950E940470E2E2F2E0FA937C
:1035E400EA930E94FE6C0E9460690E94D570E09389
:1035F400BB0B0E94DC70E093BC0BE0E0E093BD0BDE
:10360400DCC0A895E9E8FBE00E94E370E9E2F0E0A1
:103614000E9497700E94DE6FE2E2F4E0FA93EA936C
:103624000E94FE6C0E946069E881EF5FE8830E945B
:10363400D570E093920B0E94DC70E093930BE0EB67
:10364400E093980BBAC00E94B47D9CD30E94E870AA
:10365400E03228F0AAE0B0E0E0E00E94147C00E050
:103664007FDCA091BE0BB091BF0BA633E2E1BE0795
:1036740041F110E01A3030F41A93ACDF1A9380DD74
:103684001F5FF8CF10E0103430F41A93BADF1A93A6
:103694004CDD1F5FF8CF10E0103830F41A9394DF3C
:1036A4001A93AADD1F5FF8CF84DFA9E0B0E0E0E061
:1036B4000E94147CE6E3F2E1E093BE0BF093BF0BAF
:1036C40001E010E0193210F00C94B91B0E94ED7067
:1036D4009F010E94ED70AF010E94F7703496E4914F
:1036E400E03011F0E13069F4D901AC910E94F77037
:1036F4003596E491EA1720F40E94F7700E94FE7058
:1037040034C0E23091F4DA010E94D27BE031A7E2C6
:10371400FA0714F4FF2342F40E94F77036960E94CD
:10372400E17BDA01ED93FC9320C0E33049F4D90145
:10373400AC91AF3F21F40E94F7700E94FE7015C057
:10374400E43099F4D901AC91AF3F79F400E00E94E0
:10375400F7703596E4910E1740F40E94F7700E94BA
:10376400FE702F5F3F4F0F5FF2CF1F5FABCFFBDBCE
:1037740010E0153060F41A934BDDA091300CA630A4
:1037840020F01A9378DD1A9363DD1F5FF2CFE02FE8
:103794000E94BB7D26960895E881EF5FE883A881A7
:1037A400A43610F0E0E0E883E88107C00E94576E79
:1037B400A5E0B0E00E942E7B309621960895A0915A
:1037C400380CBB27E091370CA6C0F9DF329774F0B0
:1037D4000E940371E091370C0E940A710E94AF6F3E
:1037E400E091370CEA93D8DFE093370C08950E94F8
:1037F4000371E091380C0E940A71FA93EA930E94D3
:10380400CC670895E5E2FCE00E9412710E94037106
:10381400E091380C0E940A710E94AF6FE091380C5D
:10382400EA93BADFE093380C08950E94B67DE0E095
:10383400E093370CE093380C10E030E0343680F538
:10384400A8950E9403713A93B1DFFA93EA93E5E2F3
:10385400FCE00E94CB6F00E0A091250CA13010F099
:10386400A03808F001C001E0E12FE03041F401305C
:1038740029F43093380C3093370C11E00FC0E13049
:1038840031F4003019F43093370C12E007C0E23001
:1038940029F4013019F43093380C13E03F5FCECF94
:1038A40049C21A93A091CF0BA870B9F010E0E98136
:1038B400FA810E942D6DAE17BF077CF4ED81E09371
:1038C400250CEB81FC81E851FC4F0E941971E0E06A
:1038D400F0E00E948A701F5FEACF18810C941321D4
:1038E400E881EF5FE883A881A43610F0E0E0E88384
:1038F400E8810C942B21E881E150E883A881A43667
:1039040010F0E3E6E883E8810C942B21A0913A0CB3
:10391400BB27E091390CF0E031960E941E71EC59FE
:10392400FF4FDF01E4E6F0E00E948B7B08950E94E4
:10393400576EA5E0B0E00E942E7BE050FE4F0C9441
:103944002B210E942371E881EA93C0D10C942B218E
:103954001A9335DBE1E0E093860BA8C1A89510E04B
:10396400143680F41A93ABD1A0912A0CAF3F31F4F2
:103974000E942671AF3FEFEFBE0711F01A93E1DF0B
:103984001F5FEECF0E942B71689420F88FC10E94B4
:10399400B67D10913A0CAD81AA23CAF5E091390C99
:1039A400E11719F0AD81AA230AF030C01A9387D128
:1039B4000E942671EE81FF81EA17FB0729F4E8854E
:1039C400A0912A0CEA1709F01EC00E943171EC8103
:1039D400FD810E94CD7AEA17FB0744F40E943671F8
:1039E4000E943F71E0E0EC83ED830BC00E943671CE
:1039F400EC83FD83E0E0F0E00E943F71E0E0E093BF
:103A04002A0C1A9363D10E944471C8CF46C0E09136
:103A1400390CE11729F0AC81BD810E94AA7D0CF01C
:103A24001BC01A934CD10E942671EE81FF81EA17C4
:103A3400FB0729F4E885A0912A0CEA1709F009C0CC
:103A44000E9436710E943F711A9340D1E0E0EC83EA
:103A5400ED830E944471DBCFAC81BD810E94AA7DBD
:103A64001CF454DF33970CF418C0E885E0932A0C57
:103A7400EE81FF810E944971EC81FD810E943F71BA
:103A8400E091390CEA9322D1E091390CEA9328DFD2
:103A9400E093390CE0E0EC83ED83689420F8EC814A
:103AA400FD810E94BD7D299608951A93A091460C2C
:103AB400A03059F4E091490CF0914A0CFA93EA933E
:103AC400E8EBFBE00E944E7109F40BC0E1E0E093E7
:103AD400460CE091390CE093480CE091390CE093EA
:103AE400470CA091460CA13011F00C94DA1DE09122
:103AF4003A0CA091480CEA1711F40C94CB1DE091F8
:103B0400480CEA93F8DEE093480CEA93D8D0A091ED
:103B14002A0CA13010F0A03808F034C0E091470C12
:103B2400EA93E9DEE093470CA091480CEA1749F1C7
:103B3400EA93CCD0E091E20BE030E9F410E01530E8
:103B4400D0F4ABE01A9FF001DF01E352FA4FE081B9
:103B5400E03049F0FD01E452FA4FE081AE2FE091EC
:103B6400480CEA1709F005C00E945471A091470C53
:103B7400A0831F5FE4CF0E942371E091480CEA9375
:103B8400A5D006C00E942371E091480CEA939ED010
:103B94000FC0E091470CE0933A0CE0E0E093460C50
:103BA400689420F80E94E668E093490CF0934A0C6C
:103BB4007DC01A93A89510913A0CE091390CE11745
:103BC400C1F00E945A710E94AA7D64F4EB81A09115
:103BD4002A0CEA1739F40E942671E981FA81EA175E
:103BE400FB0709F003C0E12F1881A6C00E944471AD
:103BF400E4CFEFEF1881A0C00E9431710E94AA7D2A
:103C040084F4E0912B06E87031F4E0912E08A09141
:103C14002A0CEA1731F40E945E710E947570E03438
:103C240008F001C08DC10C948921A895E091390C4C
:103C3400A881EA1761F0E8810E94637119F0E881B4
:103C44000C942B21E881EA934BDEE883EFCFEFEF6E
:103C54000C942B211A93A89510913A0CE091390CED
:103C6400E117E1F00E945A710E94AA7D8CF4E09160
:103C74002B06E87031F4E0912E08A0912A0CEA1783
:103C840039F40E942671E981FA81EA17FB0709F0E9
:103C940002C00C9470210E944471E0CFEFEF0C94A9
:103CA40071211A9310913A0C1A93BFDF1991089558
:103CB400E881EA9315DEE883EA93B7DFCAC20E947B
:103CC40003710E946A710E94CB6FC3C20E94037188
:103CD4000E946A710E94AF6FBCC20E94B67D0E94AE
:103CE4002B7110E030E0343628F5A8953A93E7DFDD
:103CF40000E0A0912A0CA03808F401E0E12FE030A4
:103D040041F4013029F430933A0C3093390C11E02A
:103D14000FC0E13031F4003019F43093390C12E063
:103D240007C0E23029F4013019F430933A0C13E05F
:103D34003F5FD9CF0E94BD7D249608950E94B67D31
:103D4400E0EAEA93E2E0FFE0FA93EA93EF81EA9390
:103D54000E94AB67E0EAEA93E2E0FFE00E94CF6FE3
:103D64003E2FE0EAEA93E2E0FFE20E94CF6F2E2FBB
:103D7400EC81E31711F4E21709F402C0E0E474C122
:103D8400E5E072C1E5E5EA93D9DFE0933B0CA0914D
:103D94003B0CA03429F4EAEAEA93D0DFE0933B0C2D
:103DA40008950E947371A43009F43FC010912E0845
:103DB4000091550CE0913008E03059F0E0932E0862
:103DC400689424F80E947871E0E0E0932F08E0E51D
:103DD40020C0E0912F08E03021F0E0932E08E2E5C6
:103DE40018C0E0E0E0932E08E093550CE091C40B7A
:103DF400E03031F0E091C40BE150EA930E94CC181A
:103E0400A091350CA17039F0E091C40BE0932E0819
:103E1400E4E4E093550CA0912E081A1721F4A09124
:103E2400550C0A1711F0689423F809911991089513
:103E34000E947E71EBE0EC93EC81D8011696EC9332
:103E4400EB81D8011796EC93D8011896E0E0F0E0E6
:103E5400ED93FC93D80112960E948B71D8011496AD
:103E64000E948B710E94907101C10E947E71ECE0EE
:103E7400EC930E94907134C21A9318E0113108F542
:103E8400E0911408F0911508A981BA81EA27FB276B
:103E9400BF010E949C71E623F723309781F00E94B2
:103EA4009C71A981BA81EA23FB23309731F01A93DC
:103EB400E0E0EA931A93BCDF02C01A93D6DF1F5FD7
:103EC400DDCF0DC2A0911A0CA93030F0E0915D0C49
:103ED400A0915C0CEA1709F414C0E0915D0CE03089
:103EE40021F4E3E6EA93C1DF08C0E0911A0CEA93F7
:103EF400E0E0EA93E3E6EA939BDFE0915D0CE09374
:103F04005C0C0895A0919A0BECE1EA230895A0912A
:103F14009A0BA07411F0E2E00895A0919A0BA07896
:103F240009F0F5C10DC0A091890BAF3F09F4EFC1B1
:103F3400E9DFE43009F4EBC1E5DFE03109F4E7C17E
:103F4400E1E008950895A881AF3F11F4E0E081C154
:103F5400D9DFE43011F4E1E07CC1E0E07AC1A8816A
:103F6400A23019F4CFDFE83011F0E1E072C1E0E0F3
:103F740070C1A881B981AC91A130A8F0A881B981A0
:103F8400AC91A43180F4A881B981EC910E94A7710D
:103F9400EB5FFC4FE081EF770E2EA881B98112967A
:103FA400EC91E01509F002C0E1E010C1E0E00EC1BF
:103FB400A881A13118F0E881E051E883E8810E94EA
:103FC400AC710E94B671A091D00BA13018F0A881F9
:103FD400A43009F006C0E0EBF0E00E94E17B0E940F
:103FE400B67137C1A881A13010F0A63008F006C020
:103FF400E8810E94C171E15CF94F2AC1E0E029C166
:10400400A881A13010F0A63008F006C0E8810E9413
:10401400C171EC5BF94F1CC1E0E01BC10E94B67D8D
:10402400EC81EA93EDDFEF731E2F1030E1F0EC81A9
:10403400EA93E6DFE0743E2FE12FE150A1E00E9415
:10404400D97AA0912306EA230E2F303011F40030E0
:1040540009F002C0E1E008C0303011F0003009F48A
:1040640002C0E1E001C0E0E00E94BD7D2596089514
:104074000E94B47D00E00530A0F50A930E940A195D
:104084000E94C671A7E10A9FF001EE5CF94F0E94FD
:10409400E370E4E1F0E00E949770E091310CDA0102
:1040A4005096EC93A091300CEFE3EA23AE2FE0910D
:1040B400330CE295E07FEE0FEE0FEA0FDA0155962E
:1040C400EC93E091310CE1503E2F3F3F41F0E09101
:1040D400320C0E94CD71DA015196ED93FC930F5F7F
:1040E400CACF10E01034C0F51A930E9477181A93BF
:1040F4002ADFE13079F5E0919D0BEA9373DFE1501B
:104104000E2F0F3F39F10E94C671E12FDA01139689
:10411400EC93E0919D0BDA011496EC93E091A30BE0
:10412400F091A40BDA011696ED93FC930E947E7035
:10413400A4E6B0E080E090E00E94337BDF01CB0195
:10414400E091A30BF091A40B0E94D76EDA011A96AA
:10415400ED93FC931F5FC6CF0E94BB7D62C0A0910C
:104164001908A23031F0A83021F0A73011F0A530A1
:1041740009F40AC00E949070EFEFF0E00E9497707B
:1041840077DFE0E0E093A20608951A93E981E0580E
:10419400E98310E01530C0F4A3E21A9FF001EB5557
:1041A400F94FE081AE2FE981EA1749F4F001EC55AB
:1041B400F94FE081AE2FE0912E08EA1709F002C012
:1041C400E12F03C01F5FE6CFEFEF18812296089519
:1041D4000E94B67DED81EA93D8DF1E2F1F3FF1F0D8
:1041E400A3E21A9FF001ED55F94F9F01D9011296F0
:1041F400EC91EF77EC93EC81D901EC930E94A771D9
:10420400EF5EFC4FBF01E081EF77DB01EC93EC81C3
:104214000E94A771E15FFC4FA1E0A083E12F0E94FF
:10422400BD7D269608950E94576E0E94D37161F455
:10423400E0914F0CEF5FE0934F0C0E94576EED55E9
:10424400F94FA0914F0CA0830E94576EED55F94F82
:10425400E081219608951A931FEFE091D40BF09119
:10426400D50BA981BA81AE17BF073CF0E091D60BFC
:10427400F091D70BEA17FB070CF412C00E94D87117
:104284000E94BA171E2F103031F01F3F21F0E09129
:104294002E08E11729F4E1E0E0935D0CE0E01FC093
:1042A400E0E0E0935D0C1AC01A930E94D871D3DF4A
:1042B4001E2F103099F01F3F39F4E2E2F6E0FA9332
:1042C400EA93EB81FC8106C0ECE3F6E0FA93EA930F
:1042D4000E94DD71FA93EA930E94CF10E12F1881B6
:1042E40023960895E0916505E03009F00895E09182
:1042F4002C06E03009F008950AC0E0916605E0302C
:1043040009F00895E0912D06E03009F00895E0E009
:1043140008950E94B67DE0912606F0912706AC81AF
:10432400BD81EA27FB279F0110E0153090F4F901C5
:10433400E17049F0A7E11A9FF001EF5CF94FDF014A
:10434400EC91EF5FEC93D9010E94E0719F011F5F34
:10435400ECCFEC81FD81E0932606F09327060E94C2
:10436400BD7D7CC428970E94B47D30912606A0911F
:10437400D00BA47011F40C94F82100917306E09111
:104384004506E31721F4E0915C06E31709F025C024
:104394003F3F51F4013808F00150003820F408E997
:1043A400E0E0E0932D0619C0003809F40AE1013079
:1043B40008F00150003189F4A0911908A23031F0BD
:1043C400A83021F0A13011F0A53039F4EFEFE32744
:1043D400EA93E7E0EA930E942243E0914506E093E2
:1043E4005C0630934506009373063AC010E015301E
:1043F400B8F5A7E11A9FF001EB5BF94F0081E12FBB
:10440400A1E00E94D97A2E2FE22FE32391F0003805
:1044140010F0003C08F001C00F5F003C31F4E22FC3
:10442400A0912306EA2BE0932306003808F400E861
:104434000FC0003408F40F5F003439F4EFEFE227C3
:10444400A0912306EA23E0932306003808F000E055
:10445400A7E11A9FF001EB5BF94F00831F5FC7CF01
:10446400E0E0E0932C06E0E0F0E0E0931608F0933F
:104474001708E0915D0CE03021F0E0911A0CEA930A
:1044840097DDE0911D08EF5FE0931D08E091E30BD9
:10449400A0911D08EA1751F4E091E30BF0E0A0E0CD
:1044A400B1E00E94F57BEA1BE0931D08A091190876
:1044B400A13019F0A93009F096C0A091620BB09117
:1044C400630BE4E1F0E00E948B7B309719F4E1E0A8
:1044D400E0931F0807DFE03019F00FDFE07809F4FC
:1044E40062C00BDFEF775E2F5A930E9477180E9409
:1044F4009D6DED55F94F5081503011F40C94D52237
:1045040012DDE13031F4E0911A08EA9328DDE0305D
:1045140009F449C00E94E5710E946770EC91EC7146
:10452400EC3021F4E0911D08E07851F40E94EA7126
:10453400EC91EA933DDD0E94EF71EC91EA9338DD52
:104544000E94EA71AC91A63070F5A3EEB6E00E9429
:104554009D6D0E945A6E0E940F6F0E94EA71EC9149
:10456400EA9340DD1E2F1130F0F00E94F4710E9496
:10457400F771CF010E94F4710E945A6E6D917C9183
:10458400E12F0E94C171EF5CF94F0E94FC71E60FAC
:10459400F71FDC01ED93FC93E12F0E94C171EF5CE6
:1045A400F94FA0E0A08310E01530E8F40E94FF71F9
:1045B40013965C915F3FA9F05A9335DE5E2F0E94FB
:1045C40009720E94F4710E94F771BF010E94F47194
:1045D4000E945A6E0E940F72AE81BF811296E0E073
:1045E400EC931F5FE1CFA0911908A23039F0A830F5
:1045F40029F0A53019F0A73009F0E2C100E0053038
:1046040010F00C94E224A3E20A9FF001ED55F94F57
:10461400EA87FB87AA85BB85AC91A03019F0A281FB
:10462400A07809F0CBC1AA85BB8513960E94D27BE2
:10463400309771F0AA85BB8513960E941C720E9464
:10464400227229F4AA85BB8513960E948B71B6C188
:1046540054DEE03021F00E94227209F4AFC120E060
:1046640030E0333010F00C948D240E942C72DF0162
:104674000E942A6D0E942E6EE887F987A181A2709C
:1046840021F4A481B581109709F410C1E885F98556
:10469400A181A47011F40C94AF23A181A87021F41A
:1046A4000E94CA33E03009F457C00E943272EBE032
:1046B400EC93A885B9850E943F72A885B9851396A5
:1046C400EC91AC85BD851796EC93EC85FD85389609
:1046D4000F01E885F985A181E1E0EA230E94467291
:1046E400ED93FC93A885B98514960E94D27BAC8582
:1046F400BD851296ED93FC930E944972AC85BD85ED
:104704001496ED93FC93A02FEAE0EA9FF001E30FE7
:10471400EF5F0E944F72E885F985A085B185E2E0DC
:10472400F0E00E942E7BA885B9851896ED93FC9342
:104734000E944972309739F4A885B9851896E8EE35
:10474400F3E0ED93FC93E885F985A181E8E0EA2B99
:10475400A885B9851196EC936EC0E885F985A18189
:10476400A17031F4A885B98514960E941C7243C0C7
:104774000E94587237DCE1501E2F0E94FF7112967E
:10478400EC91E03001F5AE81BF8153960E940F6F2A
:10479400EE81FF81A189B289109751F003881488B2
:1047A400AE81BF8151960E94D27BE015F1050CF0D9
:1047B40009C00E947D6DDDDBE03011F00E945D7266
:1047C4000E9465720EC0E885F98534960E946D7268
:1047D4000E9446720E941E710E94757253960E9436
:1047E4008B71E885F985A581AA232AF4A885B98562
:1047F40014960E948B71A885B985EC91EC71EC300C
:1048040021F4E0911D08E078B1F4E885F985A481EC
:10481400B5815E971CF4A181A07209F404C0E885F7
:10482400F985A28106C00E945872C2DBE885F98529
:10483400A381AA93BDDB0E944972309791F0A885A9
:10484400B98518960E941C720E944972309749F4E7
:104854000E947D6D8EDBE03011F00E945D720E943B
:1048640065720E945872DADBE03001F10E947D6DBE
:1048740080DBE03049F00E945D72AA85BB85EC9133
:104884000E94A7710E94A56DAA85BB851296EC9122
:10489400E058AA85BB851296EC93E3E0E0932406E6
:1048A4000E945872ADDBEF73E0932506A885B985A5
:1048B40014960E94D27B309761F52F5F323048F511
:1048C400A885B98516960E94D27B309789F0E88531
:1048D400F985A681B7810E947C72AA85BB8513964F
:1048E400ED93FC93A885B98516960E948B7111C02F
:1048F4000E942C72DF01E32FEF5FF0E00E942E6E26
:10490400E887F987A181EDEFEA23A885B985119697
:10491400EC933F5FA6CE233011F00C94E0240E9468
:10492400CA33E03069F00E943272E8E0EC93AA8561
:10493400BB850E943F72AA85BB85EC910E944F7291
:104944000E947D6D16DBE03011F00E945D72AA8535
:10495400BB85E0E0EC93EA85FB85A581ECE1EA23E5
:10496400E83061F50E946C6EAE2FEA85FB85E38D1D
:10497400EA1741F4EA85FB85E48DE150EA930E944D
:104984007A171CC00E94CA33E030C1F00E94327210
:10499400E3E0EC93AC85BD85EFEFEC931896EA85E4
:1049A400FB85E38D0E948172AC85BD851296EA85F4
:1049B400FB85E48D0E9481720E9485720F5F1FCE79
:1049C4000E948B7249F4A0911908A23021F0A830FA
:1049D40011F0A53009F401C050C010E0153010F0FA
:1049E4000C943F250E94FF7113965C915F3F11F474
:1049F4000C943D250E940972AE81BF81BD010E94C5
:104A04000F72EE81FF8138960E946D720E9491723E
:104A14000E9475720E94D27BDF010E94AA7DB4F4C9
:104A2400EE81FF81A681B7810E94AA7D7CF4AE81CC
:104A3400BF810D901C90AE81BF8116960E94D27BDF
:104A4400D001AE1BBF0B0E94AA7D0CF014C0AE8136
:104A5400BF81BD010D901C90EE81FF81A681B781BD
:104A6400F001EA1BFB0BDB01ED93FC935A93E5E0A9
:104A7400EA930E9422431F5FB1CFE0911C08E0300B
:104A840041F4E0911608F0911708E0931408F093AC
:104A940015080E94BB7D2E9608950E94B67DA091B4
:104AA400C10BE091C20BE150EA9FF001EF5F1E2FB2
:104AB4002FE330E000911E08A091180CA13080F083
:104AC400E091180CE150A0911E08AE1728F0E09177
:104AD400180CE1503E2F04C0E091180CE2502E2F28
:104AE400EC81E03049F1EF3F51F4A0911E08A11B85
:104AF400A31720F0E0911E08E11B0E2F1DC0EE3F0E
:104B040059F4E12FA0911E08AE0FA21720F4A09132
:104B14001E08EA0F0E2F10C0EC3F49F4A091180CA8
:104B2400A13020F0E091180CE1500E2F05C0AC81AB
:104B3400A1501A9FF0010E2FE0911E08E01751F0CA
:104B44000A930E947718A0918A0BAD3209F4032FBF
:104B540000931E080E94FE46A0911908A83019F47B
:104B64000E94E50E02C00E945E0E0E94BD7D259645
:104B740008950E94B47DC6D9E03111F40C942D2619
:104B840020E030E040E050E010E0133060F50E9497
:104B940095720E945A6E0E94D27B309711F10E9446
:104BA40098720E94AC712E2B3F2B0E949872EA934C
:104BB40035DAE03029F0E3E0E0932406E0E04CC08D
:104BC4000E949F720E94AC712E2B3F2B0E949F72F9
:104BD400EA9324DAE03029F0E3E0E0932406E0E00D
:104BE4003BC01F5FD2CF00E0053058F5A3E20A9F17
:104BF400F0010E94D37119F110E0133000F50E9406
:104C04002C72DF010E94DD710E94A672AE0FBF1FDD
:104C14001296EC910E94AC714E2B5F2B0E942C7269
:104C2400DF010E94DD710E94A672AE0FBF1F1396B2
:104C3400EC910E94AC714E2B5F2B1F5FDECF0F5F98
:104C4400D3CFF901E423F523309729F0E1E0E09391
:104C54002406E0E001C0E1E00E94BB7D26960895B1
:104C64001A93E091530CE03011F40C948726E091F0
:104C7400E40BE13059F4A091530CA13311F4EFE0AB
:104C840001C0E0E0EA930E94B35E3FC0E23059F411
:104C9400A091530CA13311F4E6E001C0E5E1EA93DD
:104CA4000E94B35E32C0E53061F4A091530CA1338D
:104CB40019F4E091990B01C0E0E0EA930E94B35E1D
:104CC40024C0E330B1F410E0173040F40E94DD71E9
:104CD400E15CF64F0E94AD721F5FF6CFA091530CBA
:104CE400A13311F4E1E301C0E0E3EA930E94B35E6F
:104CF4000CC00E94B172E9E4EA930E941B63E09144
:104D0400530C0E94B8720E94BD7288C422970E94FC
:104D1400B47D30E0A0911908A23029F0A83019F030
:104D2400A53009F022C1A985A03410F00C94B6274F
:104D3400E0912E08E03009F418C1E9850E946B70F7
:104D4400E03131F4E1E3E093530C8ADFE1E00DC19B
:104D5400EAD8E03009F409C110E01530A0F4A3E268
:104D64001A9FF001DF010E94D37141F0FD01EB5560
:104D7400F94FE081AE2FE985EA1709F002C0E0E0BF
:104D8400F4C01F5FEACFF5DEE03011F40C94B627CF
:104D940010E0A3E21A9FF001ED55F94FEE83FF8373
:104DA400AE81BF81EC91E03011F00C94AF271396E3
:104DB4000E948B7100E0033010F00C947E27A3E274
:104DC4001A9FF001E855F94FDF010E94126D0E940D
:104DD4002E6EAF01DA0116960E948B710E94C27288
:104DE400DA011296EC930E94C972DA011396EC93DD
:104DF400A0919A0BEEEFEA23DA01EC930E94D072B1
:104E0400DA011196EC937ED8E43139F0FA01A181EC
:104E1400E2E0EA2BDA011196EC930A93A0D8E03091
:104E240011F40C945F27FA01A281AA93DBD8E15014
:104E34002E2F2F3F81F0A7E12A9FF001EF5CF94F5D
:104E4400A0E0A083A7E12A9FF001EE5BF94FA0E068
:104E5400B0E0A083B1830E94D8720E945A6E0E946F
:104E6400D27BDA011496ED93FC93013040F00E945A
:104E7400D8720E945A6E0E94D27B309709F00EC0FD
:104E8400AE81BF811596E02F0E9413700E94A67216
:104E9400AE0FBF1F1196EC91E062EC93AE81BF811F
:104EA4005A96EC91E062EC93023030F40E94DB728B
:104EB400DA0116960E94817204C0DA0114960E94E7
:104EC4008B710E94841FEC3019F4E0E0E0931D081C
:104ED4000E94E2720E94CD71DA011896ED93FC9360
:104EE400FA01A281A63030F0A181E4E0EA2BDA01D4
:104EF4001196EC930F5F5FCFA0911908A23011F0C7
:104F0400A53019F4A885AF3F08F007C0E0912E083A
:104F1400EA93EA85EA930E94AD19E885AE81BF81E0
:104F2400EC93E0912E08AE81BF811196EC93E98554
:104F3400AE81BF811296EC93A885A43138F4E8853C
:104F44000E94A771E15FFC4FA1E0A083AE81BF8105
:104F54001696EC91ED7FEC9331E01F5F303011F445
:104F6400153008F001C015CFE32F0E94BB7D2A96AF
:104F740008950E947371A23021F0A0911908A53000
:104F840021F40E94E9720E942A6FA0911908A830A6
:104F9400C9F40E94E972E1E0EA930E946047E0915B
:104FA400E20BE03069F4EA810E94F472E081EF7769
:104FB4001E2FABE01A9FF001EA51FA4FA0E0A08344
:104FC400689420F8198108812396089564970E94B3
:104FD400466DA23039F4E0912E08EA93EB8DEA9302
:104FE4000E94AD19A0911908A83011F00C945E2804
:104FF4000FEF20E0253050F4A7E12A9FF001EE5C8A
:10500400F94FE081AE2FEA8DEA1709F402C02F5F51
:10501400F1CFA7E12A9FF001E15DF94FAF01DA0179
:1050240015960C910F3F11F40C945E280E94FA72AD
:1050340010810E945A710E94AA7DECF4ADE2BCE09A
:105044000E941C720E9400730E943171A083B1837C
:105054001A930E94681EABE00A9FF001E252FA4FD5
:1050640030810A93FE0137960E9406733A93FE013B
:1050740037960E940A730E941073F1F40E94FA7228
:10508400AFEFA083DA011396EFEFEC93DA011596F4
:10509400EC930E9400730E941673E0E0F0E00E941B
:1050A4003F71E0E0E0932A0C1A930E94681E0A9371
:1050B4000E944B10689420F80E94BB7D6B96089563
:1050C4001A9310E01031B0F4A7E11A9FF001EC5BE1
:1050D400F94FE081EF73AE2FE981EA1729F41A93AF
:1050E4000E941020E03009F403C0E1E01881E0C020
:1050F4001F5FE8CFE0E01881DBC01A93E091560C03
:10510400F091570CFA93EA93E4EFF1E00E944E71A8
:10511400F9F00E941B7310E01530D0F4A0915A0CE2
:10512400AF5FE5E00E94887BE0935A0CEF5FEA935F
:10513400C7DFE03059F0E3E0E0932406E0915A0C35
:10514400F0E0EF5FFF4EE093250668C21F5FE4CFF7
:1051540065C21A93E0912306E093520CE8E7F0E06D
:10516400FA93EA93ECEDF0E0FA93EA930E942F4766
:1051740010E01530D8F4E12FEF5FEA93A1DFE030BF
:1051840099F00E94A46CE12FEA5FF0E00E94686E3F
:10519400EAE4F6E00E94066EA6EEBBE00E94DD7132
:1051A4000E942E6E0E94366E1F5FE3CF37C2A5DFCA
:1051B400E0912406E13029F4E2E5F6E00E9422734E
:1051C4003CC0E23029F4E8E9F0E00E94227335C0E3
:1051D400E33051F4EAE4F6E0FA93EA93E091250629
:1051E400F0E0E050F04F29C0E43019F4E0E6F6E0D6
:1051F4001FC0E53031F4E0912506EA930E94B21015
:1052040020C0E63019F4E8E6F6E012C0E73029F4ED
:10521400ECE8F0E00E94227310C0E83029F4E2E2E6
:10522400F6E00E94227309C0E93059F4ECE3F6E099
:10523400FA93EA93E0912506F0E0FA93EA930E9448
:10524400CF10E0E0E09324060895A881B981119677
:10525400E1E0EC930E945E71A881B9811296ED930E
:10526400FC930E94891FA881B9811796EC930E9430
:105274006C6EA881B98118960E948172E091C6056E
:10528400A881B981EC93E0912A0CA881B981169682
:10529400EC93E091890BA881B9811A96EC93E09183
:1052A400AC0BF091AD0BA881B9811496ED93FC93EE
:1052B4002296089564970E94B67DA091E20BA230D5
:1052C400E1F4EB8DEA930E9477180E94891FADE206
:1052D400BCE00E948172ABE2BCE0EB8D0E94817263
:1052E400E0912E08E0932A0C0E947070309721F010
:1052F4000E9470700E94497114C0AA8DAF3F09F4D6
:10530400CAC0EA8DEA930E94611EAB8DAF3F29F4B7
:105314000E945E710E947570EB8FEB8DEA930E9480
:1053240077180E94891F0E2FA98DAF3F21F00E948C
:10533400951FE03009F001C0AEC00E9431710E9497
:10534400126DAE17BF071CF014DCE13009F0A3C0E6
:10535400A091D10BA03021F4A091E20BA23011F561
:105364000E946C6EE13041F00E94CA33E03021F0BB
:105374000E94E033E03009F002C00E9427730E94CB
:105384006C6EE13021F40E94D033E03009F409C09E
:105394000E943373EE55F84FFA93EA9356DF0E9456
:1053A400397377C0EB8DEA93EA8DEA93AFDC1E2F55
:1053B400113011F00C944B2AA091D30BA13059F465
:1053C400E0912E08EA930E945E71FA93EA93EFEF5C
:1053D400FFEF0E943F730E9431710E94126D0E9480
:1053E4001E710E943F71689420F8A091E20BA030D6
:1053F40019F4A88DAF3F09F437C00E944373EE51EE
:10540400FA4F0E943171A083B183E88D0E940F6E20
:105414003081E88DEA93FE0135960E940673E88D8B
:105424000E940F6EE081EA93FE0135960E940A7392
:105434000E94841FE03131F00E944373EA51FA4F15
:10544400A1E005C00E944373EA51FA4FA2E0A08391
:105454000E944373EC51FA4FFF93EF930E94E66866
:10546400AF91BF91ED93FC930E94107319F4E0E0A7
:10547400E0932A0CEA8DEA930E94681EE0912E08BC
:10548400EA930E9470700E944873FA93EA930E9410
:10549400531CE1E001C0E0E00E94BD7D6C960895DC
:1054A40068DBE13041F40E94CA33E03021F00E940D
:1054B400E033E03009F007C00E9470700E94497127
:1054C4000E94277330C338C30E94B67D0E944B7379
:1054D4001F3F11F40C94B72AE091530CE03011F003
:1054E4000C94B62A1A930E947718E5E0E0932406F8
:1054F40010932506A0911908A23031F40E94547328
:105504000E945621E03009F00EC0A091540CA13342
:1055140031F4E0912E08EA931A930E94AD19E1E365
:10552400E093530C1DC2A0911908A83091F40E9475
:1055340070700E9458730E2F0A930E9442343E2FBB
:105544001A930A93EFEFEA933A93B4DEE03009F04A
:1055540007C2A0911908A53021F4A2DFE03009F0B8
:10556400FFC1E0E3E093530C06C0E0E3E093530C87
:10557400E4E0E0932406F4C1E0913F090E945C73E7
:1055840008951A93E6E0EA930E94B35E0E94B17212
:10559400A0913F09A83539F4E8ECF7E10E9468735B
:1055A400E0E00E94BD72A0913F09A33509F510E027
:1055B400A0911908A83021F0A23011F0A53009F407
:1055C40011E3E3E5EA930E941B631A930E941B63B1
:1055D400E0E8EA930E941B63E0E8EA930E941B63FD
:1055E400E0E80E94B872E093530CE0E00E94BD72C0
:1055F400A0913F09A93491F4A091E40BA43019F4CB
:10560400E0E0E093530C0E946C73E09325060E9443
:105614007673EC91E093540C57DF22DB19910895D3
:105624000E94B67D0E947B73E2E3F0E0E0934D0CB0
:10563400F0934E0CA0913F09A73741F4E3E4F9E05D
:105644000E9482730E9487730E945C73A0913F0939
:10565400A03310F0AA3308F025C020912608309119
:105664002708EFE3F9E00E948273E2E0EA930E94E4
:10567400C2620E2F013090F00E948773E0932506DA
:105684000E9487730E948B730E944B730A931A9330
:105694000E94AD192093260830932708E2E5EA9387
:1056A4000E94B35E5DC1A091E40BA33069F4E09164
:1056B4004B0CF0914C0CFA93EA93E0914D0CF09161
:1056C4004E0C0E944E7109F40FC0E0E0E0933909DA
:1056D400E5E4EA930E94B35E0E947B73E8ECF0E099
:1056E400E0934D0CF0934E0C08950E94E86D0E94D7
:1056F400FD0D0E9490730E94A46C0E94A46C0E94F1
:10570400D746A0911B08A23021F4E0EAF0E00E9401
:10571400066EA0911B08A13021F4E8E6F6E00E9491
:10572400066EE0911B08E03021F4EEE6F6E00E94FC
:10573400066E0E949A730E94D06C0E94D7460E9403
:105744009D730E94A273FA93EA93E0915F05F0912E
:1057540060050E94A8730895E1E003C0E0E001C081
:10576400E2E0E0931B08C1DF08950E94841FEC313E
:1057740009F0E2C1E091990BE33631F4A0911908E4
:10578400A23009F4EBDF17C0E23631F4A091190816
:10579400A23009F4E5DF0FC0A091C505A23011F0D5
:1057A400A63021F4E091990BEA9377D9A091C5052D
:1057B400A43009F4D1DFB7C11A930A93A0E023FC03
:1057C400A1E0A03019F0AA81A03009F014C0E89437
:1057D40023F8E7E0E09318080E941A46A0913008E5
:1057E400A03019F40E94AC7309F405C00E94B1738F
:1057F400A3D7E89424F824FE24C00E94B673EAE5F3
:10580400F0E00E94BD7319F0AA81A130C9F4C0D799
:10581400E030B1F00E94C3730FEF1FEF0E94547386
:105824000E942D21E03021F40091260810912708D0
:10583400EB81EA93E0912E08EA931A930A937CD7BA
:105844000BC00E94B673ECE2F1E00E94BD7321F438
:105854000E94CA73E0932F081981088183C00E94B3
:105864003C6E0E94A46C0E94406E0E94A46C0E9434
:10587400A46C0E94D746EAEFF5E00E94066EE09120
:105884001A080E94CE73E8E0F6E00E94066EE2E099
:10589400E0930E0408950E949070E0ECF0E00E9402
:1058A4009770E881E03009F406C0A0911A08AF5F50
:1058B400E3E00E94887BE0931A08E1E0E0934F0C58
:1058C4000E943A2026C20E94B67D10E0103410F0E7
:1058D4000C94B22C0E94DD71ED55F94F30813F3F9D
:1058E400E9F11A930E94771800E00E94D2730E9493
:1058F4005A6E0E94D27B3B9794F00E94D5730F019D
:105904000E94D2730E945A6E0E94DB730E94E1735C
:105914000E946770EC91EE7FD001EC9301E00E944D
:10592400E6730E945A6E0E94D27B759794F00E948F
:10593400D5730F010E94E6730E945A6E0E94DB73B6
:105944000E94E1730E946770EC91E160D001EC93D6
:1059540001E0013019F41A930E9497181F5FB6CF23
:105964000E94BD7D249608950E947371A93011F49C
:105974000E94E97323FE06C0E7E0E09318080E9442
:10598400B173DAD60E943243E030A1F1E0E00E9424
:10599400F073103838F5113231F4E7E0E093180869
:1059A4000E94B173C9D61D3439F40E94F7730E9462
:1059B4003C64E3E0E09318081B3271F40E94FC732A
:1059C400EAE2EA93E3EDF7E1FA93EA93E0911A0845
:1059D400E05DEA930E943C641F3219F4E1E0EA932B
:1059E4005CD83DDF103830F00E9402741A930E9494
:1059F4001521BBDE0E947F210E2F003810F40C9479
:105A0400432D0F770034E0F5E0911F08E03069F092
:105A14000A930E941521A0911908A13019F40A9340
:105A24000E942011E0E0E0931F08E0915B0CE01776
:105A340039F10A930E9477180E94EA71AC91A83058
:105A440028F40E94EF71AC91A830A8F0E02FEF5F2A
:105A5400E093A2060A930E9415210E94EA71EC9138
:105A6400EA930E94EF71EC91EA93E091A206EA9323
:105A74000E941A1F03C0E0E0E093A20600935B0CAF
:105A84000EC0A0915B0CAF3F51F0E091A206E03054
:105A940019F0EA930E94371FEFEFE0935B0C099132
:105AA40019910895A881A03310F0AA3308F01DC0FD
:105AB4000E9406740E940B74AAE0B0E00E942E7B40
:105AC400DF01E8810E941074EA0FFB1FE0932408B1
:105AD400F0932508E2E0E0930E040E949A730E947A
:105AE400D06C0E94406E0E949D73A881A33451F42F
:105AF4000E9490730E949A730E94D06C0E94406E20
:105B04000E949D7306C1E091C70BF091C80B0E94DF
:105B1400137411F4E2E00895E091C50BF091C60B03
:105B24000E94137411F4E1E00895E091CB0BF0911D
:105B3400CC0B0E94137411F4E0E00895EFEF089584
:105B4400E0E0E0931B08A0911908A23021F40E9420
:105B5400FE460E945E0EA0911908A83009F44BD6A7
:105B6400A0911908A53009F446D10895E2E0EA931A
:105B74000E94FE40E2E0E0930E04E881EA9392DFA3
:105B8400A881AF3721F4E0912B06E37009F403C038
:105B9400E2E0E0931808A881A13239F0A33421F49B
:105BA4000E940674109709F004C0A0911908A2304D
:105BB40009F00FC0A0911B08A33009F4D1DDA09116
:105BC4001B08A23009F4BCDFE0911B08E03009F4A3
:105BD400C5DDA881AD3311F00C94472E0E941A46FE
:105BE400E0911B08E030A1F4E0912408F09125082D
:105BF400FA93EA930E945621E03041F4E09124089C
:105C0400F09125080E948B739BDF01C0A7DD3DC086
:105C1400E13069F478DFEF3F41F0E3E00E9417746C
:105C24000E94F7730E941D7401C08ADF2EC0E23007
:105C3400F1F40E940674A034E0E0BE07B4F4E091ED
:105C44002408EA930E942474E2E0E0930E040E9484
:105C5400A46C0E94A46C0E94D7460E94F96D0E9415
:105C6400B30FE3E0E0931B0801C07ADD0EC0E3301C
:105C740061F4E0912408EA930E947718E0912408E3
:105C8400EA93EEEFEA9342D86BDDA881AD3409F4D0
:105C940063DDA881A43521F4A0911908A23009F08C
:105CA40001C05CDDA881AB3221F4EEEFEA930E94DF
:105CB4004F25A881AD3221F4EFEFEA930E944F25DE
:105CC400A881A73421F4E1E0EA930E944F25A8813A
:105CD400AB3421F4ECEFEA930E944F251AC00E94E2
:105CE400B1200E94FE46E0E0E0931B08A881A130A9
:105CF40039F40E94AC7321F0A091CA0BA03009F4CE
:105D040002C02CDD06C00E945E0E0E9454730E94E5
:105D14002D21219608951A930A930E94E9730E94F3
:105D24002874B9F10E943074A0F10E9402741DDD40
:105D3400E03021F4A091990BA03009F02AC00E9410
:105D440038740E94EA20EF3F09F0F3C40E945473B0
:105D54000E945621E03021F40E94951FE13009F0A1
:105D640018C00E94841FE83119F40E943D7409F0A0
:105D740001C0DFC40E9438740E9488260E2F0130AF
:105D840021F4A091990BA03009F403C01A930E9446
:105D9400B210A0912E06AF3F61F110912E06EFEFE5
:105DA400E0932E061A930E9477180E9454730E945F
:105DB4005621E03021F40E94951FE13009F019C00A
:105DC4000E94841FE83119F40E943D7409F001C057
:105DD400B0C41A93EEEFEA930E9488260E2F013086
:105DE40021F4A091990BA03009F403C01A930E94E6
:105DF400B21059DC9EC40E94B1200E943A20E8945B
:105E040021F8E0E0E0931E080E9444740E94FE46DC
:105E14000E94A46C0E94A46C0E94D746E0913206B2
:105E24000E947D6EE09133060E947D6E0E94A46CF8
:105E34000E94016E0E94D746E0913F060E947D6E4B
:105E4400E0913906F0913A060E94536E08950E943B
:105E5400B67D0E94E973ABD90E943243E03049F029
:105E64000E94307430F00E9402747FDCE03009F448
:105E740017DBE091580CF091590C0E942E6F11F42D
:105E84000C94A42F0E9444740E94A46CE2E0F0E0FD
:105E94000E944B74E0913706F09138060E94536ECD
:105EA400E0913B06F0913C060E94536E00E0053001
:105EB40010F00C94A42FA7E10A9FF001E15DF94FC3
:105EC4009F01F901A381AF3FD9F1D9011A960E942C
:105ED4005F6E7F936F93FF93EF930E944E74AF9125
:105EE400BF918F919F910E94F07A0E94337BDF01D2
:105EF400CB010E945374D9011C96ED93FC93F901D4
:105F040004841584D9011E960E94D27BE015F10504
:105F1400B9F0F90104841584A685B785F001EA1B5C
:105F2400FB0BE093AC0BF093AD0BBADAE13041F428
:105F3400D9011C960E94D27BD9011E96ED93FC9345
:105F44000F5FB5CFB0DB0E94BD7D14C40E94B67D47
:105F54000E94E9730E94287411F40C943B300E944F
:105F640035430E2F0A9302DE003820F0A091C605B7
:105F7400A03808F429C00F770A930E945A740E942B
:105F840058731E2FA091E20BA03011F41F3F09F4A7
:105F940016C030E0353098F4ABE03A9FF001E4529B
:105FA400FA4FE081E11749F43A9FF001E252FA4FC7
:105FB400E081EF5FE093C605232F3F5FEBCF0A93A9
:105FC4000E9438742A9354C0A091E20BA03021F4AB
:105FD400003810F0053808F00AC00F770E94FA72F2
:105FE4001081EFEFEA930E9438740A9363D9A09169
:105FF400E20BA03011F0003808F43BC00F770A938D
:106004000E947718B2DBE030A1F50E945D740E9413
:10601400EA20EF3F19F00E94BD7DACC30E94951F9A
:10602400E13039F50E94891FE03049F40E945D7423
:106034000E948826E03011F00E9462741AC00E9407
:10604400841FE83141F40E943D7421F00E945D7484
:106054000E9488260EC0A0911E08E02F0E94CC6DDD
:10606400AE0FBF1F1C910A930E943874EFEFEA939E
:1060740021D9A0912E06AF3FF9F000912E06EFEF43
:10608400E0932E060A930E945A740E9458731E2F9E
:106094000A931A93EEEFEA93EFEFEA930BD91F3FBB
:1060A40041F4A0919D0BA03021F4A091A00BA0304D
:1060B40009F002C00E94627420FE0AC0E89420F82D
:1060C400E091E20BE03019F4EED33FD501C09ED548
:1060D40030E0353080F5ABE03A9FF001DF01EA5162
:1060E400FA4FE081E03049F0AC51BA4F0E94687435
:1060F400E8EEF3E00E944E7199F4ABE03A9FF001B0
:10610400EA51FA4FE081E23051F43A9FF001EC5148
:10611400FA4FDF010E94D27B0E942E6F09F409C05E
:10612400ABE03A9FF001EA51FA4FA0E0A0836894F3
:1061340020F83F5FCECFB7DA0E94BD7D1BC30E941B
:10614400466DA33011F40C945E32E0913908ED34BD
:1061540011F00C948331E0913A08EA3511F00C9473
:10616400383124FC83C0E0913B08E0532E2FE091AA
:106174003C08E0533E2FEDE3F8E00E9482730E9456
:106184007673AC91AB3429F40E946D740E944E6214
:106194000E2F0E947673AC91A43529F40E946D747D
:1061A4000E944E62AF01E091CD0BE31731F5E0E0C0
:1061B400E093510C0E94C373409326085093270820
:1061C400A0912F080A1759F0E7E0E093180800930C
:1061D4002F082093500CE0E0E0932E080DC0A0910E
:1061E400500C2A1721F0A0912D08A03009F004C00A
:1061F400209318082093500C35C0A0912F08A0308C
:1062040049F4A091CE0B0E942A6DE853FF4FE4910C
:10621400EA2309F40CC0E7E0E09318082093500C3B
:10622400E0E0E0932E08E0913808E093510CE0910F
:106234003808A091510CEA17A9F44093260850930A
:10624400270800932F080E94C373A091500C2A17AB
:1062540021F0A0912D08A03009F004C02093180863
:106264002093500C273011F40E947871E0913A0881
:10627400E93439F4E7E00E9417740E94CA73E0938A
:106284002E08E0913A08E23439F4E4E00E941774ED
:106294000E94CA73E0932E08E0913A08E03519F49D
:1062A400E1E0E0931808E0913A08EC3449F4E4E0C2
:1062B400E0931808E0913B08E053EA930E948C15A0
:1062C400E0913A08E334E9F4A0913B08A13320F0CB
:1062D400A0913B08A93308F014C00E947074E091A7
:1062E4002108EA930E94C41AE0913808EA93E6ED83
:1062F400F7E1FA93EA930E949B700E94E57B0E9467
:106304002F64E0913908E03521F4A0911908A130F7
:1063140009F003C00E94FC73A2DAE0913908EF345B
:1063240059F4E0913A08EE3439F4E0913808EA93EC
:10633400E9EDF7E10E947674E0913908E33579F5E7
:10634400E0913A08EF3359F5A0913B08A03320F0CF
:10635400A0913C08A03308F422C00E947074E0911C
:106364003C08E0531E2FE0913B0CA0912108EA1752
:1063740010F01A3008F013C0103011F40E940E1AF5
:10638400E0913808EA93ECEDF7E1FA93EA930E947E
:10639400CE700E94B1700E94E57B0E942F64E09150
:1063A4003908E33411F00C942632E0913A08EF33C3
:1063B40011F00C942632E0913C08E03319F4EFEF2D
:1063C400E0932208A0913B08A03308F10E94707466
:1063D400E0913B0CA0912108EA17C8F0E091220853
:1063E400EF5FE0932208E0912108EA93E09122080C
:1063F400EA930E948A1AA0911F0CB091200C109766
:1064040021F4A0912208A03408F001C0E7CFE09164
:106414002208EA930E9477180E947C74EFEDF7E15A
:106424000E9468730E94716F0E9481740E94867436
:106434000E94766F0E94E57B0E9486740E94DE6F44
:106444000E94B4630E940164E0913908E434A1F528
:10645400E0913A08E43481F514E0E1E0E09338098E
:10646400103538F40E94DD71E95CF74FE081E032C9
:1064740008F41AC00E94DD71E95CF74FE081E33251
:1064840059F40E94DD71E85CF74FE081E053EA9330
:106494000E94B35E1F5F06C00E94DD71E95CF74F86
:1064A4000E94AD721F5FDCCF0E947C74E2EEF7E1C4
:1064B4000E9468730E9401640E94BB7D2696089521
:1064C4001A930A930E948B7211F40C94D032E0E078
:1064D400E0935D0CE0911808EF770E2F00931808F5
:1064E4000E94FE460E94016E0E94036D0E94D746E0
:1064F400013021F0A0911908A13009F00DC0E0E1AC
:10650400F6E00E94066EDFD9E4EFF1E0FA93EA9335
:106514000E9450430E94FE46073049F40E94B12075
:10652400E0E0E0931B080E9453110E94AB28043062
:1065340031F4E5EEF7E10E94066E0E94110D083079
:1065440019F40E948C7457D1053019F40E948C748C
:1065540052DC013039F40E949974009319087FD9F0
:106564000E945E0E093059F40E9499740E945E0ED6
:106574000A93E1E0EA9320D9E1E0E0935D0C023074
:1065840029F40E948C74E1E0EA93A9DB033011F44E
:106594000E94B040009319080E94641FA09119083A
:1065A400A73011F00C947C33E091560CF091570C09
:1065B4000E942E6F21F0A0911B08A03009F00AC0A0
:1065C4000E941B73E091520CA0912306EA1711F06C
:1065D4000E94AB280E943243E030E9F0E2E00E94DE
:1065E400F0731A935FDA1D3409F4B6D81D3399F4A5
:1065F4000E941A4688DAEF3F41F0E3E0E09318087E
:106604000E94F7730E941D7406C0E7E8E09318081F
:10661400E0E0E0931B08A0912E08A03031F0E09157
:106624002E08A0912D08EA1709F455C0E0912E0810
:10663400E150EA930E94CC18A091350CE1E0EA23E2
:10664400E13021F4E0912B06EF7C09F429C0E0E06D
:10665400E0932D08E091500CE03019F0E093180815
:106664001EC012E0E0912B06EC7009F018E0E091F6
:10667400C40BA0912E08EA1781F0E0912B06E07478
:1066840039F011E0EAE2EA93EAEEF7E10E94767467
:10669400E0912B06E07809F019E0109318081BC06C
:1066A4000E94FE460E9453110E94016E0E94036DD7
:1066B4000E94D746EBE4EA930E947146E0912E08CB
:1066C400EA930E949F41E2E3F6E00E94066EE091A5
:1066D4002E08E0932D08A0912E08A03021F4A0915B
:1066E4002D08A03009F406C0E0E0E0932D08E7E8A7
:1066F400E0931808A0911908A33011F40E94B33E46
:10670400A0911908A13009F42FD9A0911908A23039
:1067140009F401DBA0911908A83009F417DCA09151
:106724001908A53009F493DBA0911908A93009F4DC
:106734001BD90991199108950E94A474E652F84F47
:10674400A6E0A0830E94A474E752F84FAB81A08313
:106754000E94A474E152F84FAA81A0830E94A474F9
:10676400E552F84FA881B981A083B1830E94857254
:106774000E941051249608950E94AA74A881B98198
:10678400AC91A53020F0A881B981E0E0EC9389C0F8
:10679400A0911308BB27E091120805C0A09111082D
:1067A400BB27E0911008F0E031960E941E713596E7
:1067B400DF01E5E0F0E00E948B7B08951A931091CD
:1067C4001308E0911208E117A1F0ABE01A9FF00161
:1067D400E652F84FE081E13011F0E23011F4E1E0EB
:1067E4004DC0EDB7FEB7FA93EA931F93C5DF1F912F
:1067F400E8CFE0E043C01A930E94B120ECEDF5E04D
:106804000E94E3700E94726D0E94706910E015305E
:1068140068F40E945471AFEFA083ABE01A9FF001BB
:10682400EE51FA4F0E9416731F5FF1CF10E015303E
:1068340048F4A7E11A9FF001EC5CF94FAFEFA08395
:106844001F5FF5CFE0912B06E37019F00E94AC7343
:1068540009F402C0689401C0E89421F8EFEFE093D2
:106864002C08E091E20BE03029F41DD06ED1E894BD
:1068740020F804C00E94FE460E94E50E1991089576
:106884001A9310E0153058F40E945471E081AE2F31
:10689400E981EA1711F4E12F03C01F5FF3CFEFEF93
:1068A40018812296089522970E94B47D00E0053055
:1068B40058F40E94B074A0E00E94B674E152FA4FFA
:1068C400A0E0A0830F5FF3CF00E00530C0F50E9485
:1068D400FA72E081EF3F89F10E94FA72E0810E942E
:1068E4006371B9F00E940073DF010E94D27B0E94A1
:1068F4003171EA17FB0751F00E9400730E94317155
:10690400A083B1830E94BB74A1E0A0830E94B074F1
:1069140012C0ABE00A9FF001EA51FA4FE081E03087
:1069240061F40E94FA72AFEFA0830E9400730E9488
:1069340016730E94BB74A1E0A0830F5FC6CF0E94B0
:10694400531E1E2F1F3F11F0E1E001C0E0E0E09371
:106954005D0C1F3F11F40C94013550E000E005304C
:1069640048F40E94FA72E0811E1711F451E002C04B
:106974000F5FF5CF5030E1F500E00530C8F50E9417
:10698400FA72E081EF3F91F50E94FA7210830E943F
:1069940000730E943171A083B183ABE00A9FF001C0
:1069A400E052FA4FA0912A0C0E94B674EF51FA4FAC
:1069B400FF93EF930E945E710E947570AF91BF9137
:1069C400EC930E94BB74A1E0A0830E94B074A1E088
:1069D4000E94B674EC51FA4FFF93EF930E94E6685D
:1069E400AF91BF91ED93FC9351E002C00F5FC5CF0F
:1069F400503029F01A930E945A1E1E2FAACF30E05D
:106A0400353010F00C944735A7E13A9FF001E15D71
:106A1400F94FEE83FF8350E000E0053048F5503035
:106A240029F5ABE00A9FF001EF51FA4F20812A9338
:106A34000E9477180E94B074E081E13059F42A93DF
:106A44000E94A51FE13031F4A32FAF5FE0919D0BAD
:106A5400EA1709F00BC0E22FAE81BF811396EC93C5
:106A6400E02FAE81BF811596EC9351E00F5FD5CF37
:106A7400503049F4AE81BF811396EFEFEC93AE81B1
:106A8400BF811596EC933F5FBBCF0E94BB7D0C94F6
:106A9400EF370E94B67DAC81BD81EBE4EC93EC81D1
:106AA400FD813196FA93EA930E94C174E052FA4F41
:106AB400E0810E94EA6C00E00E94CA74EC91E0302C
:106AC40011F00F5FF9CF0E94CA74E0E2EC930F5FFC
:106AD4000E94D0740E94A06D0E94C174EE51FA4FBE
:106AE400DF010E945F6E0E94D574EE81ABE0EA9FE5
:106AF400F001EF51FA4F10811A930E94771800E0C9
:106B04000E94CA74EC91E03011F00F5FF9CF0E943B
:106B1400CA74E8E7EC930F5F0E94CA74E0E2EC9356
:106B24000F5F30E03A3060F40E94D074EA0FFB1F2C
:106B34000F01AAE8BBE00E94DC740F5F3F5FF2CF55
:106B44000E94CA74EC930C94343864970E94B67D06
:106B540000E010E0153040F40E945471E081EF3FF2
:106B640009F40F5F1F5FF6CF053021F0A0912C08C8
:106B7400A03009F406C0E0E0E0932C08EA930E94F8
:106B8400001010E0153088F5ABE01A9FF001E152D7
:106B9400FA4FE081E03039F11A9FF001E352FA4FE5
:106BA400E081E030B1F01A93FE0135960E9406733D
:106BB400ABE01A9FF001EF51FA4F30813A930E94F3
:106BC40077181A93FE013596FA93EA930E945B10A4
:106BD4000AC01A930E944B10ABE01A9FF001E152D5
:106BE400FA4FA0E0A0831F5FCDCF053021F4A09120
:106BF4002C08A13009F406C0E1E0E0932C08EA93E4
:106C04000E9400100E94BD7D689608950E94B47D84
:106C1400A091E20BA23011F40C94CE3930E034315F
:106C240068F40E94E3740E94E774DA011296E0E0CB
:106C3400EC93DA01EFEFEC933F5FF1CF0E94531E28
:106C44000E2F0F3F11F0E1E001C0E0E0E0935D0C96
:106C54000F3FA1F10E945E71FA93EA930E942718F4
:106C64001E2F1F3F31F1A0911E08E12FEA1B3E2F7A
:106C74003431F8F40E94E3740E94E774FA01329606
:106C84000F01E081AE2F0E94ED74B0E0EA0FFB1F0C
:106C9400D001EC93FA01A281A43620F0DA01129615
:106CA400E3E6EC93DA01AC91AF3F19F4E02FDA019B
:106CB400EC930A930E945A1E0E2FCACF0E94981476
:106CC40030E0343110F00C94ED360E94E3740E94ED
:106CD400E774FA01A381AF3F11F40C94EB360E94E0
:106CE400F2740E946B70E83139F40E94F274EA93F2
:106CF4000E947017E03009F408C00E94F274EA930D
:106D04000E947017DA011296EC93A0919A0BA07866
:106D140039F4FA010280DA011196EC91E01509F4D4
:106D240058C0DA0113962C91ADE02A9FF001EF5E72
:106D3400FC4F0F01DA011296EC91D001EC930E9402
:106D4400F274EA930E94C720EF3F29F0ADE02A9F36
:106D5400F0010E94A56DDA011296EC91E03089F001
:106D64000E94F774DF010E94C76DEC93ADE02A9F87
:106D7400F001E25FFC4FDF01E091980BEF70EC93C0
:106D840013C00E94C76DE03021F40E94F774A0E0A4
:106D940003C00E94F774A8E0A083ADE02A9FF0012D
:106DA400E25FFC4FA7E0A0830E94F274EA930E9482
:106DB400C720EF3F19F0ECE0E0930F04DA011296DC
:106DC400EC91DA011196EC932A93E1E0EA930E94A4
:106DD40060473F5F76CF0C94CE39E7E0E093180824
:106DE4000E94B217A8950E94171CA8950E946F1EB6
:106DF400A895EFEFE093B20BE093890BE093340C8A
:106E0400E0932F0CE0932E060E94FD74EC7F29F092
:106E1400A8E0B0E0E0E00E94147C089524970E946A
:106E2400B67D0E944D42E6E2F7E00E94E3700E94C4
:106E3400D9420E947542E0912108E03061F0E2E01D
:106E4400F7E00E94E3700E94D942E09121080E9479
:106E540002750E9406750E9475420E940E1A00E097
:106E64000A30A0F40A930E94A6180E940470EFE06E
:106E7400EA930E94B342E02FA3EAB6E00E940A75A7
:106E84000E94B1700E940E750F5FEACF0E94874284
:106E9400E6E6F2E0FA93EA93EFE0EA930E94D9423D
:106EA4000E943E6F0E940E750E9489420E947542A4
:106EB40010E0103110F00C94EB370E946C6EE11767
:106EC400E1F5E2E3F7E00E94E3700E94D9420E94F8
:106ED400ED6D0E940675E0E0E0931E08A0911E0887
:106EE400A03448F5E0912108EA93E0911E08EA9362
:106EF4000E948A1A0E94716F3097B9F0E0911E08BF
:106F0400EA930E9477180E94716FFA93EA930E94A1
:106F140014750E94D9420E94DE6FEAE0EA930E944F
:106F2400B3420E94766F0E940E75E0911E08EF5FD7
:106F3400E0931E08D3CF0E9419750E94DD710E9450
:106F4400B67011F00C94E937E2E3F7E00E94E370C5
:106F54000E94D9420E94ED6D0E9406750E941D7523
:106F6400E0E30E94C27029F40E94C7700E944E623E
:106F74009F0100240216030644F50E946D740E94CA
:106F840078620E94E16E0E946D740E9425753A93A6
:106F94002A930E9414750E94D9420E942975EAE03E
:106FA400EA930E94B342EC81FD816E817F810E944D
:106FB4000E750E941D75E1E30E94C27029F40E94BF
:106FC400C7700E944E629F01D4CF0E9419751F5F43
:106FD40070CF0E944E420E94BD7D289608950E9463
:106FE400B67DAD81BE812C910E942E750E94ED6DFF
:106FF4000E94126D0E94686EECE3EA930E9471464F
:10700400EC81EA930E94C9462A93ED81EA930E9497
:107014003F41EEE3EA930E9471460E94A2730E94EC
:1070240048730E94A8730E943375333409F431E223
:10703400313320F0EC81E05DE31708F407C0E32F5F
:107044000E941074E853FF4FE4912E273D3311F052
:10705400313209F401C0CACF3D3319F4AD81BE8188
:107064002C93E32F0E94BD7D279608950E94B47D42
:1070740020E0AF81B8855C910E942E750E94ED6D71
:107084000E94126D0E94686EE2E0EA930E94C94673
:107094005A930E949F410E94A2730E9448730E94C7
:1070A400A8730E943375303310F03A3308F00EC0E1
:1070B400203009F450E021E0A52FEAE00E94887B0B
:1070C400AAE0EA9FF001E30FE0535E2F3B3211F494
:1070D400533608F001C05F5F3D3211F4513008F4BB
:1070E40001C05150333429F4203009F431E250E026
:1070F40020E03D3319F4EE81E51708F005C0AF81B7
:10710400B8855C9130E020E03D3311F0313209F470
:1071140001C0B4CF3D3319F4AF81B8855C93D0C0BE
:107124000E94B47D20E0AF81B8854D915C910E94AE
:107134002E750E94ED6D0E94126D0E94686EAE81E4
:10714400A23051F4E6E0EA930E94C946FA010E9493
:1071540081740E947E4108C0E5E0EA930E94C9461A
:107164005A934A930E9489410E94A2730E944873D1
:107174000E94A8730E943375303310F03A3308F03C
:107184001EC0203011F440E050E021E04031E7E23D
:107194005E0734F0DA01E0E1F7E20E948B7BAF0195
:1071A400493BEBE05E0724F0DA010E940B74AF0167
:1071B400DA010E9438750E943D75D097AD013B32CB
:1071C40021F44033E5E75E070CF002C04F5F5F4FE8
:1071D4003D3221F40024041605060CF002C041508F
:1071E4005040333431F4203009F431E240E050E0CF
:1071F40020E03D3311F0313209F401C09ACF3D3320
:1072040021F4AF81B8854D935C935AC00E94B47D3C
:107214000E942E7520E050E04FEF0E94ED6D0E9419
:10722400126D0E944B740E944275E885EA930E9495
:107234009F46E52FE10FF0E00E9448730E94A87377
:107244000E943375303310F03A3308F021C03053C4
:10725400431729F04F3F09F05F5F20E005C0A22FDC
:10726400AF5FEA2FE3702E2FE52FAF81B8850E9420
:1072740047750F01E32FAAEBB7E00E940A75AE0F22
:10728400BF1FE22F0E944775E491D001EC93432F76
:107294003B3219F4EE815E1708F002C05F5F4FEFD6
:1072A4003D3211F4513008F402C051504FEFEE81D9
:1072B4005E1720F4313211F03D3309F401C0ADCF33
:1072C400E32F0E94BB7D299608951A930A93A091F7
:1072D4009A0BECEDEA231E2F00E00D3040F40E94DF
:1072E4004B750E944F75E11711F00F5FF6CF0E94A6
:1072F4004B75EA0FFB1F0E94E17B0E94066EE02F94
:1073040049C4AAE9BBE00E94576EAE0FBF1FEC91BF
:10731400E17011F4E3E701C0E9E4EA930E947146E5
:10732400219608950E94B47D0E942E750E94ED6DF1
:107334000E94126D0E944B74C8DF5E2F0E94A273DC
:107344000E9448730E94A8730E9433753D3211F065
:10735400363311F4503009F401C051503B3211F06E
:10736400333311F45C3008F001C05F5FA0919A0BD5
:10737400E1E0EA232E2FE52FACE2B2E00E940A7589
:107384000E944F75E20FE0939A0B3D3311F03132B6
:1073940009F401C0CBCFE32F0E94BB7D269608954C
:1073A4000E94B67D0E942E750E94ED6D0E94126DA2
:1073B4000E944B74AAE9BBE0EC810E946770EC91D7
:1073C400E17019F4EAE3F7E002C0EEE3F7E0FA93C0
:1073D400EA930E9488460E94A2730E9448730E9406
:1073E400A8730E943375303310F03A3308F010C09C
:1073F400AAE9BBE0EC810E9447750F01AAE9BBE052
:10740400EC810E946770AC91E1E0EA27D001EC9333
:107414003D3311F0313209F401C0C6CFE32F0E948D
:10742400BD7D259608950E94FA6CE1E0EA930E94DE
:10743400FD0D0E94A46C0E94A46C0E94D7460E9479
:10744400DE6FEAE0EA93E2DEE13209F46CC40E9402
:10745400A46C0E94A46C0E94406EE0EAF0E00E94DA
:10746400066EE5E9FBE00E94E3705ADEE13209F4BE
:107474005AC40E94A46C0E94A46C0E94406EE2E272
:10748400F2E00E94066EE091970BEF5F0E2FEDB7CE
:10749400FEB7FA93EA930F93EAE0EA93E7DD0F91DC
:1074A400E13209F440C400240216030624F4E02F58
:1074B400E150E093970B0E94A46C0E94A46C0E947C
:1074C400406EE2E4F7E00E94066EECEAFBE00E9404
:1074D400547509F428C40E94A46C0E94A46C0E94F0
:1074E400406EE6E4F7E00E94066EEEEAFBE00E94DE
:1074F400547509F418C40E94A46C0E94A46C0E94E0
:10750400406EEAE4F7E00E94066EE9E9FBE0FA93D4
:10751400EA93E3E60E945D7509F405C40E94A46C35
:107524000E94A46C0E94406EE0E5F7E00E94066EA3
:10753400F9DEE13209F4F7C310E0133010F00C94D3
:10754400583B0E94A46C0E94A46C0E94406EE12FE0
:107554000E94CE73E4E5F7E00E94066E0E94627515
:107564000E94D746ADE9BBE00E94DD710E94A06D88
:10757400E0E10E945D7509F4D6C3E9E0F0E00E9401
:10758400D06C0E94D746A0EABBE00E94DD710E9445
:10759400A06DE0E10E945D7509F4C5C30E94A46C6E
:1075A4000E94A46C0E94406EE12F0E94CE730E9440
:1075B40066751A93F5DEE13209F4B5C30E9462756B
:1075C4000E946A7551F40E9495720E947475E2E0FB
:1075D4000E94787509F4A7C309C00E9495720E949D
:1075E4007475E0E00E94787509F49DC30E94A46C50
:1075F4000E94A46C0E94406EE12F0E94CE73E0E6CC
:10760400F7E00E94066E0E9462750E94D746A9EABE
:10761400BBE0EE27A10FBE1F2C913327EDB7FEB7B9
:107624003197FA93EA933F932F93E0E0EA9378DD5E
:107634002F913F91E13209F476C3A9EABBE00E949D
:10764400DD71EA0FFB1F2083123070F50E94A46CD9
:107654000E94A46C0E94406EE12F0E94CE73E8E663
:10766400F7E00E94066E0E9462750E94D746A0EB66
:10767400BBE0EE27A10FBE1F2C913327EDB7FEB759
:107684003197FA93EA933F932F93E0E0EA9348DD2E
:107694002F913F91E13209F446C3A0EBBBE00E9475
:1076A400DD71EA0FFB1F20831F5F47CF3CC30E949D
:1076B400B67D10E01A930E9424740E947D750E9486
:1076C400A46C0E94D7460E94786E0E9466750E9440
:1076D400F96D0E9470700E94536E0E94A46C0E9407
:1076E400016E0E94D7460E947E700E94646EE7E09D
:1076F400F0E0FA93EA930E94016E0E94D746E0916B
:10770400AE0BF091AF0B0E94F07A0E94646E0E945F
:10771400A46CE2E0F0E00E94686EE0E7F7E00E940B
:10772400066EE091970BEF5FEA930E949F41E7E0BA
:10773400F0E00E94F26D0E94D746C7DD0E94446EBD
:10774400E091990BE03029F0E091990BEA930E94C3
:107754009F4100E0033010F00C94EE3B0E94A46CB7
:10776400E02FED5FF0E00E94686E0E94C272EA931F
:107774000E949F41EBE2EA930E9471460E94C97203
:10778400EA930E949F410E94446E0E94D07259F471
:107794000E94D8720E945A6E0E945F6E0E94817588
:1077A400E4E7F7E00AC00E94D8720E945A6E0E9471
:1077B400D27B0E94536EE6E7F7E0FA93EA930E94C5
:1077C40088460E94446E0E94E272EA930E94A54198
:1077D4000E9485750F5FBECF0E9435433E2F3B321A
:1077E40011F4103408F001C01F5F3D3211F4113060
:1077F40008F401C011503D3439F41A930E947718EB
:1078040012DE1A930E949718313209F053CF8BC2BB
:107814000E94B67D10E00E94FE46012F0E94A46CD7
:107824000E94A46C0E94D746E8E7F7E00E94066E27
:1078340031E03C3018F51038F8F40E94A46C0E9432
:107844002A6D0E94686E1A930E94CC180E94786E6A
:107854000E94446EA091350CE3E00E948875A091CB
:10786400360CE7E00E948875E0912B06EA93E8E085
:10787400EA930E943F4113953F5FDBCF0E94110DB5
:107884000E9435433E2F3D3411F00C94883C0E94F5
:10789400E86D0E94FD0D102F1038C0F51A930E9458
:1078A400CC180E94A46C0E94A46C0E94406EECE868
:1078B400F7E00E94066E0E94786E0E9466750E9430
:1078C4007F6E0E94D746E0E9F7E00E94066EE5E38A
:1078D400FCE0FA93EA93E3E00E945D7509F423C2A5
:1078E4000E947F6E0E94406EE6E9F7E00E94066EF9
:1078F400E6E3FCE0FA93EA93E7E00E945D7509F49D
:1079040012C21A930E94FE181F5FC6CF313211F0C3
:10791400103808F001C07FCF06C20E94FA6C0E94A2
:107924007D750E94A46C0E94D746ECE9F7E00E94A2
:10793400066E10E01530F0F41A930E940A190E94A2
:10794400A46C0E94546F0E94786E0E946675E09148
:10795400300C0E948D75E091330C0E948D75E0917E
:10796400310C0E948D75E091320CEA930E94A5417E
:107974001F5FE0CF0E9435430E2F0D3411F00C949D
:10798400023D0E94E86D0E94FD0D10E01530C0F527
:107994001A930E940A190E94A46C0E94A46C0E946B
:1079A400406EE0EBF7E00E94066E0E94786E0E9443
:1079B400667530E03430F8F40E947F6E0E94406EA9
:1079C4000E942A6D0E94E37AE05EF74F0E94E17BF9
:1079D4000E94066E0E942A6D0E94E37AE05EF74FD1
:1079E4000E949175FD013596E4910E945D7509F43C
:1079F4009AC13F5FDFCF1A930E942A191F5FC6CF37
:107A040092C11A930A930E94FE46E1E0EA930E940F
:107A1400FD0D00E0093210F00C94CC3D0E94DD0C09
:107A24000E94A46C0E94A46C0E94D7460E94126D0E
:107A34000E9494750E94E17B31960E94066E0E941A
:107A4400446E0E94126D0E9494753496E491E0385D
:107A5400A9F40E946C6E1E2FEDB7FEB7FA93EA9359
:107A64001F93E0E1EA9302DB1F91E13209F492C033
:107A7400E12FA9E0B0E00E94147C88C0E238A9F4A8
:107A84000E94E8701E2FEDB7FEB7FA93EA931F9396
:107A9400E0E1EA93EBDA1F91E13209F47BC0E12FD4
:107AA400AAE0B0E00E94147C71C0E138E1F40E94C5
:107AB400FD741E2FEDB7FEB7FA93EA931F93E3E02C
:107AC400EA93D4DA1F91E13209F464C00E94DD0C18
:107AD4000E94FD74E11731F0E12FA8E0B0E00E94AC
:107AE400147CFFCF53C0E03069F40E94126D0E94F1
:107AF400947532960E940A6EE1E00E945D7509F465
:107B040049C044C0E13069F40E94126D0E9494752A
:107B14000E949175FD013596E4910E945D75D1F145
:107B240035C0E23061F40E94126D0E949475329661
:107B34000E940A6EEFE00E94787561F127C0E3307D
:107B440071F40E94126D0E9494750E949175FD015A
:107B54003596E491EA9343DAE132E1F017C0E43078
:107B6400A9F40E94126D0E94947532960E94E17BE2
:107B7400E0935E0CF0935F0C0E9448730E9494752E
:107B84003596E491EA9342DBE13221F00E94B51785
:107B94000F5F40CF099119910895E8810E94CE7337
:107BA400E6EFF7E10E94066E0C944B421A930E9492
:107BB400E86D0E94FD0D10E0133010F00C94333E7C
:107BC4000E94A46C0E94A46C0E94406E1A93E5DF8C
:107BD400ECE0F0E00E94D06C0E94D7461A9391DB4F
:107BE4000E9462750E946A7551F40E9495720E9407
:107BF4007475E2E00E94787509F4FCC209C00E9421
:107C040095720E947475E0E00E94787509F4F2C2DE
:107C1400123028F50E94A46C0E94A46C0E94406E4D
:107C24001A93BBDFE4EBF7E00E94066EECE0F0E0B1
:107C34000E94D06C0E94D7460E948575EAE0F0E06D
:107C44000E94D06C0E94D746A0EBBBE00E94DD717D
:107C54000E94A06DE3E60E945D7509F4CBC21F5F2C
:107C6400ABCFC8C20E94B67D10E01A930E94247460
:107C74000E947D750E94A46C0E94D7460E94786E73
:107C84000E9466750E94F96D21E000E0033080F5E2
:107C9400E3E0F0E00E94416D0E94686E0A937DDF8C
:107CA4000E94D07249F40E94D8720E945A6E0E94B7
:107CB4005F6E0E94817508C00E94D8720E945A6E3D
:107CC4000E94D27B0E94536E0A931BDB2F5F02300B
:107CD40068F4E7E0F0E00E94416D0E94686E0E9443
:107CE400DB720E947D6E0E9485752F5F0F5FCECF81
:107CF4000E9435433E2F3B3211F4103408F001C08A
:107D04001F5F3D3211F4113008F401C011503D34AD
:107D140039F41A930E94771849DF1A930E9497182E
:107D2400313209F0A2CF0E94BD7D249608950E94AD
:107D3400E86D0E94FD0D0E94A46C0E94A46C0E9438
:107D4400D746E2E0F7E00E94066EE1E0E093210806
:107D5400E1E2F8E0FA93EA93E0913B0CEA9386D9E6
:107D6400089522970E94B47D0E9435430E2FE0911E
:107D74001B08E03011F00C945E400132D1F4E2EEC5
:107D8400F7E0A0913C0CB0913D0CEA17FB0761F4BD
:107D9400E7E0E0931808EAE2EA93E9EFF7E10E94EA
:107DA400E3700E943C64D6C1E0E0E093C0050E9409
:107DB40099750D3331F4E091C005F0E00E94306D07
:107DC40004910D3441F4EAE2EA93ECEFF7E10E9406
:107DD400E3700E943C64063449F4EAE0F8E0E0937E
:107DE4003C0CF0933D0CE0E0E093C005003311F04F
:107DF4000B3229F4E091C005EF5FE093C0050D322A
:107E040029F4E091C005E150E093C005013329F461
:107E14008EDFED3311F40E94A075033329F487DF5C
:107E2400ED3311F40E941037063329F4E0E0E093B7
:107E340021080E941037043329F4E0E0E09321087C
:107E44000E94A075A0912308A13010F40C94F83F6F
:107E5400023301F56CDFED33E9F40E94AD75D1F422
:107E6400E0912108EA930E94C41A30E0303190F482
:107E74000E942A6D0E94B67059F4E32FE05DEA93E4
:107E8400EFEFF7E10E94BB70E0E3EA930E945E64C7
:107E94003F5FECCF053341F5E0E0E09321080E9419
:107EA400AD7511F511E0E0913B0CE117E8F01A9380
:107EB4000E94C41A30E03031A8F40E942A6D0E9456
:107EC400B67071F4E32FE05DEA93EFEFF7E1FA9314
:107ED400EA93E12FE05DEA93E0E3EA930E945E64B3
:107EE4003F5FE9CF1F5FDFCF013451F4EAE2EA9349
:107EF400E2E0F8E10E947674E1E0E09318082AC118
:107F04000A3409F4AFDE073311F00C94F83F0E94F1
:107F1400E86D0E943F0DE1E0E0931C08E0E0F0E032
:107F2400E0931408F0931508EFE2F6E00E94E37082
:107F3400E3E7F0E00E9497700E94E668EE83FF8317
:107F44000E94B675E8E2F0E00E944E71B9F00E941A
:107F540092110E94E668EE83FF83A091190CA03071
:107F640021F00E94CA33E03009F408C00E94A474CE
:107F7400E652F84FAEE0A0830E9485720E94BB7562
:107F84000E94504340E050E00E947F21E03868F0B6
:107F94000E947F21EF573E2F313010F0313108F02D
:107FA40004C0E32F0E94AC71AF015A934A930E941C
:107FB4003E1F40931408509315080091DB05E0E040
:107FC400E093DB05013211F00B3209F401C0B8CFA4
:107FD4000B3221F4E1E0EA930E943F0D013209F0F3
:107FE400A3CFE0E0E0931C08E093DB05A091230815
:107FF400A23011F00C945740093309F402DD053422
:1080040009F48BDC083309F452DB023409F400DC94
:108014000334B1F510913A0C0E94FE4600E0E09161
:10802400390CE11711F00C3008F01DC00E94A46C4B
:108034000E94126D0E94686E1A930E94611E1A9328
:108044007CD10E94446EE0912A0C0E948D75E091CF
:108054002D0C0E948D750E945E710E94536E0E94C9
:1080640044710395DCCF0E94110D0E9435430E2FFD
:10807400013221F0E091390CE11709F401C0CCCFB1
:10808400043499F40E94AD7581F4A091D30BA0300F
:1080940021F4A091D10BA03031F00E94C0750E9450
:1080A400A46C0E9441530E94AA1CE0911B08E0307A
:1080B40011F40E949A0D49C0E130D1F4A091200836
:1080C400AB3010F4013209F405C00E943C150E9443
:1080D400110D0DC0E0E0E0931E080E94C4750E94DB
:1080E4007674E0E00E94C975E2E0E0931B082DC0BD
:1080F400E23059F5013269F4E0E0E0931B080E9494
:10810400FE46EAE2EA93ECEFF7E10E9476740E94FD
:108114009A0D0B3211F00D3359F40E94C475FA9381
:10812400EA93E1E3EA930E943C64E1E00E94C975AA
:108134000D3259F40E94C475FA93EA93E2E3EA9388
:108144000E943C64E2E00E94C975A0911808A33023
:1081540009F40ACE0E94BB7D289608951A93E3E0A1
:10816400E09319080E94FE460E94A46C0E94A46C2D
:108174000E94D746E0E6F2E00E94066E0E94A46CDC
:108184000E94016E0E94D746E3E1F6E00E94E3708C
:10819400E0E1F0E00E94977010E0E091C90B1E1737
:1081A40000F50E946C6EE117D1F0E12FE05DEA93D7
:1081B400E8E0F8E1FA93EA93E0E3EA93E0E00E946E
:1081C400C27049F40E94DD71ED5EF94FA1E0A08315
:1081D400E12FE05D01C0EEE2EA930E9471461F5F69
:1081E400DCCF0E949975E0E0E093C005E0931B08A2
:1081F4000E949A0D19910895E881E03021F4E6E493
:10820400F8E00E94CE75A881A13021F4E0E4F8E002
:108214000E94CE75A881A23021F4ECE4F8E00E941B
:10822400CE75A881A33021F4EAE5F8E00E94CE756A
:10823400A881A43021F4E0E6F8E00E94CE7529C1BB
:108244001A930A93E0E0E0937D05E0937E0510E045
:10825400143190F400E0033068F4A3E01A9FF001B5
:10826400EC57FA4FDF01EE27A00FBE1FE0E2EC93BC
:108274000F5FF1CF1F5FECCFECC31A9311E0E981DC
:10828400E11780F00E94DD71E853FF4FE491AA8169
:10829400EA2319F0E12FE05D01C0E0E2EA931FD583
:1082A4001F5FEDCF30C51A9311E0E981E11778F033
:1082B4000E94DD71E853FF4FE491AA81EA2311F093
:1082C400E1E301C0E0E3EA930AD51F5FEECF1BC5EB
:1082D4002A97A0911B0CA13038F0EA85FB856C85A8
:1082E4007D850E94817507C00E94D3750E94D77551
:1082F4000E94D375FCD426C12A970E94D3750E948C
:10830400E0750E94E9750E94D375F1D41BC12A97C8
:108314000E94D3750E94FC750E940376E8D41FC1A5
:108324002A970E94D375E7E2F8E10E9408760E943A
:1083340081740E940376DBD412C12A970E94D375FC
:10834400EAE2F8E105C02A970E94D375EEE2F8E16B
:10835400FA93EA93EE850E94EA6C0E94D375C7D41F
:108364002B9608950E94B67D10E0E1E3E09337096F
:10837400E89431F8EA930E94E663E2E3F8E10E94AC
:10838400687300E0E09182050E17E0F40E94126D1C
:10839400EC57FA4FE081E03258F4E3E2EA930E94AA
:1083A4001B630E94126DEC57FA4FE081E05D05C03B
:1083B4000E94126DEC57FA4FE081EA930E941B630E
:1083C4000F5FE0CF0E940D769F010E94A1143A93A3
:1083D4002A93E8ECF0E0FA93EA930E94F2680E2FF5
:1083E400A0E031FCA1E0A03011F4003009F001C09C
:1083F400ECCF31FE09C0E0E0E0938205E89431F867
:10840400E1E00E94BD7DF6C41F5F123008F4ADCFD9
:10841400E0E0E09382050E94BD7DECC4E09181051B
:10842400E03021F4E881EA930E94B35EA0918105D3
:10843400A13069F4A0E09299A1E0A13021F4A895BB
:108444000E94826FF7CFE881EA930E946561A09150
:108454008105A230F1F4E0918205F0E0EC57FA4F87
:10846400A881A083E0918205EF5FE0938205E0910B
:108474008305EF5FE0938305A03218F4EF5FE09388
:108484008305A0918305A83320F06CDFE0E0E0933E
:1084940083052196089508950E9419750E941975FF
:1084A40022D0EBE1EA93BADFE9E6EA93B7DFA091E1
:1084B4008105A13061F4E8ECF0E00E94EA6EE091FD
:1084C4009A00E069E0939A00E9E1E0939900A091B1
:1084D4008105A23021F446DFE0E0E0938305E0E08B
:1084E400E09381050895EDE0EA9398DFEAE0EA93EA
:1084F40095DF08951A9310E0E9811E1728F4EA81A4
:10850400EA938CDF1F5FF8CFFEC3EDE201C0EDE319
:10851400EA93E8E2EA93EEDFE6DF08952A97A09172
:108524001B0CA13038F00E94D3750E94E0750E94A4
:10853400E97504C00E94D3750E94D775FE010E949C
:10854400E3700FD02E9608952A970E94D3750E9447
:10855400FC750E941176FE010E94E37002D02C96F5
:1085640008951A930A9310E0EA81E03011F408E2C6
:1085740001C00A81AB81BC81EE27A10FBE1FAC9163
:10858400A03011F0101708F007C0AB81BC810E9425
:1085940016760E941B76EECFEA81E03039F0EA814C
:1085A4001E1720F4E0E20E941B76F9CF27C01A932D
:1085B4000A9310E0EA81E03011F408E201C00A8174
:1085C400E12FAB81BC810E944775E491E03011F04A
:1085D400101708F009C0E12FAB81BC810E944775D8
:1085E400E4910E941B76ECCFEA81E03039F0EA8115
:1085F4001E1720F4E0E20E941B76F9CF198108814E
:1086040025960895E091C405A091C305EA17B1F039
:108614000E9420760E945A6EEC91E093C6050E9457
:1086240020760E94F771E181E093C505A091C4050D
:108634000E942676E093C405E1E00895E0E0089501
:108644000E942B76A981A0830E942B763196A88163
:10865400A083A091C3050E942676E093C305C2C0FF
:10866400E091DB0508951A93E091DB05E03059F4BD
:108674000E94A1140E948B7221F4A091DB05A0300A
:1086840009F001C0F5CF1091DB05E0E0E093DB05D4
:108694000E948B7209F011E2E12FDDC30E94B67DC6
:1086A4000E94E6688F010E94A114EC81FD81E00F15
:1086B400F11FFF93EF930E94E668AF91BF91AE1B49
:1086C400BF0B9D010024021603061CF40E948B724A
:1086D40009F001C0E8CFE0E00E94BD7D2696089530
:1086E4001A93E9810E94F4720E943176E05FFC4F94
:1086F400108117FF05C0E12F0E943876A0E0A08307
:1087040016FF05C0E12F0E943F76A0E0A083E98117
:10871400ADE0EA9FF001E05FFC4F0E943176E15F3B
:10872400FC4FA0E0A08318815DC00E94B67D30E0BC
:10873400EE81ADE0EA9FF001E05FFC4F108116FF8F
:1087440017C0E12FEF730E2F0E94467611F03A30D6
:1087540008F009C00E944E76DF010E942A6D0E9433
:1087640054763F5FF1CF0E944E760E943D75EC93A4
:1087740017FF17C0E12FEF730E2F0E94467611F0FA
:10878400343108F009C00E945A76DF010E942A6D34
:108794000E9454763F5FF1CF0E945A760E943D7545
:1087A400EC930E94BD7D42C2E881F9810E940A6E69
:1087B400EA81FB8132960E940A6EEC81FD81349637
:1087C4000E940A6EEE81FF8136960E940A6EE88549
:1087D400F9853896E491EA93E985FA8539960E94F9
:1087E4000F6D02D022960895A0970E94B47DEDA546
:1087F400FEA5A9A9BAA9EA0FFB1FAF01E5E0F3E0C2
:10880400EE83FF8310E01431C0F5AE81BF81AC91DB
:10881400A03049F1EE81FF81A381B481EFA5F8A9CD
:10882400EA17FB0701F5EE81FF81A181B281E9A975
:10883400FAA9AE17BF07BCF0EE81FF81A181B28116
:108844004A175B0784F00E946076AE0FBF1FE9A948
:10885400FAA9AE17BF073CF00E946076AE0FBF1FA7
:108864004A175B070CF402C01A933ADFEE81FF81CA
:108874003D96EE83FF831F5FC6CFE5E0F3E0EE8312
:10888400FF8310E0143110F00C94EB44AE81BF81EF
:10889400EC91E03011F00C94E444EAA5EC93E9A9DE
:1088A400FAA9AE81BF811196ED93FC93EFA5F8A9C7
:1088B400AE81BF811396ED93FC93EDA5FEA5AE8129
:1088C400BF811596ED93FC93EBA5AE81BF811796FE
:1088D400EC93E0910904A0910F04EA27AE81BF81D3
:1088E4001896EC93E0911004AE81BF811996EC9335
:1088F400E0911104AE81BF811A96EC93AE81BF81E1
:108904001B960E94AD6D1C96E0E0EC93E887E8A509
:10891400F9A5309741F00E946B760E947076E4E1ED
:10892400EA930E94CF69EEA1FFA1309751F00E9413
:108934006B76E8A5F9A5FA93EA93E4E1EA930E9439
:10894400BB69E0E0EC8F0E946B760E94A6693E2F23
:108954003B30C8F000E00E945A76E081E03011F02C
:10896400053008F002C00F5FF6CF0E945A76E0810E
:10897400E03049F40E945A760E947576E058AE8140
:10898400BF811B96EC93E0E0EA8B3130C8F000E045
:108994000E944E76E081E03011F0043108F002C00C
:1089A4000F5FF6CF0E944E76E081E03049F40E94DA
:1089B4004E760E947576E05CAE81BF811B96EC9387
:1089C400E12F08C0EE81FF813D96EE83FF831F5F98
:1089D40059CFEFEF0E94BB7DE39608951A930A9353
:1089E4000E9480763097A9F1E0916205E03061F54C
:1089F4000E948076049000926205E0916205E03066
:108A040031F4E0E0F0E00E94CE75E0E01AC00E948C
:108A140085760E9480760E94E17BF595E7958F012B
:108A2400D801E0E0F1E00E94597BE0938700D8018F
:108A3400E0E0F1E00E948B7BE09386000E94857663
:108A4400E0E4E0938B0005C0E0916205E150E0931F
:108A540062050991199108950E94B67D00E025E010
:108A640033E010E01431B8F5D901EC91E03079F13C
:108A740011960E94D27B0E948D7624F5D90113961B
:108A84000E94D27BAC81BD81EA17FB07DCF4F901BB
:108A940001801280D90115960E94D27BE00DF11D50
:108AA400AE81BF81AE17BF076CF4F9010380148057
:108AB400D9011796EC910E949172AC81BD81AE17D9
:108AC400BF070CF004C0E12FEF5F0E2F04C0235F3B
:108AD4003F4F1F5FC7CF003049F0E0916305E017B7
:108AE40021F0A0916305A03009F401C022C0A09137
:108AF4006405A53079F40A93E1E0EA93A1DD0093DB
:108B0400630500936505D901EC91E0936605E3E004
:108B1400E0936105A0916405AE3119F4E4E0E093BB
:108B24006105A0916105A33018F0E5E0E0936805C4
:108B340007C0E0E0E0936405E09361050E9492764B
:108B44000E94BD7D0C94D54AE0916305E03091F01C
:108B5400A0916405A93220F4EA93E2E0EA9370DD7F
:108B6400A0916405AD3330F0E0916305EA93E4E04D
:108B7400EA9366DDE0E0E0936105E09364050E941A
:108B84009276E0E0E0936305E0936705089534D1BD
:108B940057DB0895EA81E0937F05E881E09380053F
:108BA400E0910A04E061E0930A0424C10E94B47DC8
:108BB400A0917F05A43120F4A0918005A33008F092
:108BC40033C0E0917F05F0E0ACE0B0E00E942E7B82
:108BD4008F01E0918005F0E0A4E1B0E00E942E7BDB
:108BE4009F010E949876ECE0F0E00E949D76F0E010
:108BF4000E94E17A0E94AE6CEE81E030A9F0E0912F
:108C04007F05A3E0EA9FF001EC57FA4FDF01E09102
:108C140080050E9467704C9155270E9498764A936C
:108C2400EFE0EA930E941B4D0E94BB7D27960895B6
:108C3400E0910A04E07141F0E2E0EA93B7DFE091E9
:108C44000A04EF7EE0930A0408950E94A276AF3EE0
:108C5400E0E0BE0744F4A0910203B0910303AF33F4
:108C6400E1E0BE070CF039C00E94A7760E9479703B
:108C74000E941B4DA0915D05B0915E05549734F49C
:108C8400A0915F05B091600513970CF012C0E091BC
:108C94005D05F0915E05A3E0B0E00E94067BEC5711
:108CA400FA4FA0915F05B0916005EA0FFB1FA981FF
:108CB400A083E0910D04ACE0EA9FF0010E94A2764B
:108CC4000E9447750E94B476E0915D05F0915E05BF
:108CD4003196E0935D05F0935E050C945A4AE88161
:108CE400EA93E0911004EA93B0DF0C94294A1A93B2
:108CF40010E00E94B976E03031F00E94B976EA9330
:108D0400EEDF1F5FF6CF1881239608951A930A9316
:108D140000E010E00E94BC76E03021F00832E0E090
:108D24001E070CF007C00E94BC76EA93D8DF0F5FE1
:108D34001F4FF0CF198108815DC01A930A9300E098
:108D440010E0F801AB81BC810E94C37621F0EA8176
:108D54000E94C8760CF009C0F801AB81BC810E9466
:108D6400CD76BDDF0F5F1F4FECCF198108810EC395
:108D74000E94B67D0E94A2760E94D27631978F011E
:108D84000E94D7760E9498760E94DF7633C00E94B4
:108D9400B67DAC810E94E6760E2F11270E94D7760D
:108DA4000E9498760E94DF76F1C2EA81FB81E0930B
:108DB4005D05F0935E05E881F981E0935F05F0932A
:108DC4006005AA81BB81ECE0F0E00E942E7B0E944A
:108DD400B476A881B981E4E1F0E00E942E7B06C05C
:108DE400EA81FB810E94B476E881F981E093020371
:108DF400F0930303249608950E94EE76143120F430
:108E04001A936EDC1F5FFACF0E94A46C0E94A46CBC
:108E14000E94A96CEFE3F1E00E94AE6C10E0153003
:108E240048F4A5E11A9FF001E051FB4FA0E0A083B4
:108E34001F5FF5CF10E0143148F4ABE01A9FF00146
:108E4400EC5EFB4FA0E0A0831F5FF5CFE0910A0426
:108E5400EF7EE0930A04199108950E94EE7614318E
:108E640000F5ADE01A9FF001BF01E85FFC4FDF01A0
:108E74000E94D27B0F01DF01EB81FC81AE17BF079B
:108E84005CF0E981FA81E015F10534F0FB01E05F63
:108E9400FC4FE081E03009F402C01A9321DC1F5F2B
:108EA400DECF0E94A46C0E94F6760E94A96CA9856C
:108EB400BA850E94FB760E94AE6C67C2A2970E949C
:108EC400B47DE9A50E94F4728F01D8011B96EC9140
:108ED400E03009F415C2D8011B96EC91E9A3E078BF
:108EE40059F0FE013696FA93EA93EBA10E94387684
:108EF400FA93EA930E949069E9A1E07459F0FE01A3
:108F04003696FA93EA93EBA10E943F76FA93EA939A
:108F14000E949069FE013696FA93EA930E94A6692C
:108F2400E8A3E0910D04EB8FE0910E04EA8F0E9418
:108F3400386FD80111962D913C91D80113964D911B
:108F44005C91D80115960E94D27BEEA3FFA3D801B1
:108F54001796EC91F0E0ECA3FDA3D8011896EC91E0
:108F6400EC8FE0910E04A0E10E940077EAA3FBA33A
:108F74000E9404770E9470760E947076ECA1EA93B6
:108F84000E946D4BD8011996EC91EC8FE03011F4EE
:108F9400E8E0EC8F0E9404770E9409775A934A9381
:108FA4000E9410770E9414770E941B770E941E77FC
:108FB4000E9404773A932A930E941E77EEA1FFA1A0
:108FC4000E9425775A934A930E9409770E941E773C
:108FD400A8A5A130B1F43A932A93FA0131960E94DC
:108FE4001B77FA013196FA93EA930E941077F901FC
:108FF40031960E942A77F9013196FA93EA930E94F6
:109004001E77A8A5A230F1F40E94147731970E942C
:109014001B77EAA5FBA5E40FF51F3197FA93EA93B2
:109024000E941077EEA1FFA1E20FF31F31970E9477
:109034002A77EAA5FBA5E20FF31F3197FA93EA9387
:109044000E941E77E8A5E03011F40C945249D8012F
:109054001996EC91EC8FE0910D04ACE00E942F770F
:109064000E94597BED8FA8A1EA1710F40C94814853
:10907400E1E0E0930E04E03021F0ECA1FDA1B5970E
:109084000CF402C00E943577AAA1BBA1ECA1FDA1FA
:10909400EA1BFB0BDF010E94E071EAA3FBA3ABA177
:1090A400AA231AF4E0E0EAA3EBA3A8A10E94E676BF
:1090B400AEA1BFA1F0E00E943D77EE8FA8A5A1303C
:1090C40021F40E9440770E944377A8A5A23031F48E
:1090D4000E9440770E9425770E944F77E0E0E9A341
:1090E4000E945577AE0FBF1FEC91E03039F00E941B
:1090F40055770E94CD760E945A77F2CFD1C0E1E035
:10910400E0930E04E03031F0ECA1FDA1E734A0E0DF
:10911400FA070CF402C00E943577E8A1EF8FEAA1A8
:10912400FBA1EE0FFF1FACA1BDA1AE1BBF0BE3E083
:10913400F0E00E94597BEAA3FBA3ABA1AA2322F48B
:10914400E1E0F0E0EAA3FBA3EF8DE150EF8FEF8DB8
:10915400F0E0DE011696AE0FBF1FAC91A03219F0FD
:10916400AF8DA13008F404C0EF8DE150EF8FEFCF45
:10917400AF8D0E94E676AE2FEEA1FFA1B0E0AE1750
:10918400BF0714F7EF8DE03011F4ED8DEF8FAF8D45
:10919400ECE00E942F770E943D77EE8FA8A5A130C6
:1091A40021F40E9440770E944377A8A5A23031F4AD
:1091B4000E9440770E9425770E944F77E0E0E9A360
:1091C4000E9455770E94C37621F0EF8DA9A1AE17B6
:1091D40008F007C00E9455770E94CD760E945A7706
:1091E400EFCFAF8DE8A1EA1BAE2FED8DEA1768F043
:1091F400AF8DE8A1EA1BACE0EA9FF001A0910D0459
:109204000E942F770E943D7701C0E0E0EE8FA8A571
:10921400A130A1F40E944077E20FF31F31960E941F
:109224009D76AFE00E940077E40FF51FDF01ECA10B
:10923400FDA10E94F77131960E94E66EA8A5A230A6
:1092440089F40E944077E20FF31F0E949D76AFE0FD
:109254000E940077E40FF51FDF01ECA1FDA10E943D
:109264007475BEDD0E945577AE0FBF1FAC91A0325E
:1092740019F4E9A1EF5FE9A30E9455770E94C37630
:1092840039F0AF8DE9A1EA1BAE2FED8DEA1708F492
:1092940007C00E9455770E94CD760E945A77ECCF82
:1092A400D8011C96EC91E03029F10E94386F0E949D
:1092B400047796DDF801A485A43698F4EFE0E093F2
:1092C4001004F801A485AA3028F0A485AA930E946A
:1092D4009F4106C0D8011C96EC91E05DEA93FFDC47
:1092E40009C0ECE0E0931004E2E5EA93F8DCEDE475
:1092F400EA93F5DCEB8DE0930D04EA8DE0930E0424
:109304000E94BB7DAA9608951A9310E0E89427F86A
:10931400143170F40E94156FE03011F00E941C6F3C
:109324001F5FA895E12FE37011F40E949814F0CF09
:10933400EFE0E09310040E9498140C94B64D1A9335
:1093440010E01431F8F40E94216FB1F0A85FBC4F13
:109354000E94D27BDF01EB81FC81EA17FB0764F4F6
:10936400F001E85FFC4FDF010E94D27BDF01E9815D
:10937400FA81AE17BF070CF002C00E941C6F1F5F7A
:10938400A895DFCFEFE0E0931004188125960895A7
:109394001A9310E0143190F40E94216F31F0FD0112
:1093A400E15FFC4FE081E17009F406C01A93E0919B
:1093B4000A04E170EA9382DD1F5FECCF0C94B64D92
:1093C400EA81F0E0EBBBF5BBF7E1F09365001F9891
:1093D400E6E1E0936500F09365001F9AE881F98166
:1093E400EBBBF5BB1F98FFE1F0936500EEE1E09362
:1093F4006500F09365001F9A0C94294EE2E2EBBBE2
:10940400E0E0E5BBE7E1E09365001F98E6E1E09367
:109414006500E7E1E093650008951F9A0895A0911F
:109424000403A23021F4E881AAE9B4E10BC0A091BD
:109434000403A43021F4E881AAE9B4E103C0E8817B
:10944400AAE7B4E1F0E00E94F7710E94E17B219663
:109454000895E0910403E23011F4EEE40AC0E4302C
:1094640039F4E0E2EA93A981BA810E94D27604C079
:10947400E0E2EA93E981FA81FA93EA930E94E249ED
:1094840017C0E0910403E23011F4EFE40AC0E430C1
:1094940039F4E1E2EA93A981BA810E94627704C0B7
:1094A400E1E2EA93E981FA81FA93EA930E94E249BC
:1094B40022960895E0910403E230B9F4E4E4EA93D7
:1094C4000E946777AE0FBF1FFD01FE2FE0E0AF8162
:1094D400B8850E94A06D0E94E249E5E4EA930E94E7
:1094E400F6760E94E249E6E453C0E33089F4E7E308
:1094F400EA93FF81E0E00F010E946777EA0FFB1F08
:109504000E946C770E94F6760E94E249E6E340C02E
:10951400E43049F5E7E3EA93AF81B8850E94D27657
:10952400DF01EB81FC81AE1BBF0BFD01FE2FE0E0F0
:109534000F01AF81B8850E94D2760E946C77AD810D
:10954400BE810E946277DF01E981FA81AE1BBF0B05
:10955400BA93AA930E94E249E6E3EA93AD81BE81FD
:109564000E9462771CC0E0E5EA930E9442750E9463
:10957400E249E1E5EA930E9467770E94A06D0E94A8
:10958400E249E2E5EA930E94F6760E94E249E3E5C5
:10959400EA93E981FA81AD81BE81EA0FFB1FFA9358
:1095A400EA930E94E24928960895E0910403E33087
:1095B40029F4E3E0EA93E0E1F1E00BC0E43029F4BC
:1095C400E3E0EA93E0E2F1E004C0E3E0EA93E0E3FD
:1095D400F0E1FA93EA930E94E2490895E0910403CA
:1095E400E33029F4E3E0EA93E1E2F1E00BC0E43094
:1095F40029F4E3E0EA93E1E1F1E004C0E3E0EA9373
:10960400E8E3F0E1FA93EA930E94E24908951A9399
:109614000A93EFE10E947577EBE10E947577EFE121
:109624000E947577E8EFFFEFE093600CF093610C14
:10963400E491EF3F39F0E091600CF091610C0490FB
:1096440000920403E8E1F5E18F01A0910403A23044
:1096540019F4EAEFF4E18F01A0910403A43019F4A2
:10966400EAEBF4E18F01F801E491ED3F39F4F801FC
:1096740031960E940A6E0E94B37A19C0EE3F71F4CB
:10968400F80131960E94E17BDF01E0910403F0E0F0
:10969400EA17FB0711F00D5F1F4F09C0F801E491B1
:1096A400EA93F80131960E940A6E0E94E2490D5F26
:1096B4001F4FF801E491EF3FB1F60E94BD6DE1E068
:1096C400E0930E04E0930D04E4E1E09313046DDFF2
:1096D4000991199108950E947977AE85AA2362F0C1
:1096E400AD85BE85A03FE0E0BE0734F4AB85BC8504
:1096F400AF33E1E0BE070CF050C00E948177AE0F9B
:10970400BF1FA03FE0E0BE0734F0AD85BE850E94D8
:10971400D276E987FA87EF81F885AB85BC85AE0FF1
:10972400BF1FA034E1E0BE0734F0AB85BC850E94C6
:109734006277EF83F8870E94156E0E94156E0E946F
:10974400156E0E94156EB6DE0E94156E0E94867715
:10975400498554DE0BBB15BB2EE13FE100E010E070
:10976400EF81F885E017F10764F050E0451730F019
:1097740020936500309365005F5FF8CF0F5F1F4F44
:10978400EFCF4BDE0E94A46C0E94A46C0E94A96CD3
:10979400EFE3F1E0FA93EA938DDEC9C00E94797792
:1097A4000E948177EA17FB0741F0EF81F885AB85CA
:1097B400BC85EA17FB0709F03EC00E948E771CF0B7
:1097C4000E94957784F42D853E85ED85FE85E98795
:1097D400FA872D873E872B853C85EB85FC85EF83B7
:1097E400F8872B873C870E94156E0E9486770E941B
:1097F4008177EA17FB0749F4F1DEEB85FC85ED87F9
:10980400FE87EF81F885E987FA87F8DD0BBB15BB86
:109814002EE13FE10D851E85E985FA85E017F10704
:109824003CF020936500309365000F5F1F4FF4CF29
:10983400F4DDBBDE7CC000930B0410930C040E9487
:109844009C770E94A377FF93EF930E94A7770E94CF
:10985400A377AF91BF91EA17FB0780F10E94957738
:10986400B4F420E030E00E94AA77E217F30774F022
:109874000E949C770E94B1770E94AA770E94B677D3
:109884000E94BF7758D02F5F3F4FEDCF16C020E026
:1098940030E00E94A777E217F3077CF00E949C77E0
:1098A4000E94B1770E94A7770E94B677F9010E94BF
:1098B400C67741D02F5F3F4FECCF39C00E948E77DF
:1098C400DCF420E030E00E94CA77E217F3079CF052
:1098D4000E94A7770E94B1770E94CA77D0010E94A4
:1098E400597BAF010E94BF77FA010E94C67723D04B
:1098F4002F5F3F4FE8CF1BC020E030E00E949C77F1
:10990400E217F307A4F00E94A7770E94B1770E94A0
:109914009C77D0010E94597BAF01F9010E94C67760
:10992400FA010E94C67707D02F5F3F4FE7CF0E940E
:10993400BB7D2F960895EA81FB81FA93EA9389DD32
:109944000E94D1779EDDE2E2EA93E0910B04F0916C
:109954000C04FA93EA930E94E249249608950E9423
:10996400B47DEC85FD85309711F40C94534D009132
:109974000D0410E0E0910E041E1710F00C941A4D23
:10998400E885F985FA93EA937CDD2C853D854A8543
:109994005B85022E032A11F40C94124D37FF36C056
:1099A4005A934A9356DDE2E2EBBBE0E0E5BBE7E124
:1099B400E09365001F98F6E1F0936500E09365007D
:1099C400EE81EBBBEF81E5BBEFE1FEE1E0936500E7
:1099D400F0936500E093650001FF04C0F093650017
:1099E400E093650036FF11C0F0936500E0936500D5
:1099F40001FF06C0F0936500E09365004F5F5F4F81
:109A0400220F331F4F5F5F4FEDCF1F9A220F331F7B
:109A140001FF02C04F5F5F4F4F5F5F4F0C94CB4C11
:109A2400E885F9853196E887F9871F5F0C94BC4C6B
:109A340038C022970E94B47DE885EA930E94114AB7
:109A4400EE83FF83E985A8E1EA9FF001E658F74F2A
:109A54008F0130E0383028F5F801E4915E2F0F5F74
:109A64001F4FF801E4914E2F407F0E94D6770E9449
:109A7400DB77EA87FB87F801E4914E2F440F440F0C
:109A8400440F440F0F5F1F4FF801E4915E2F0F5FE7
:109A94001F4F0E94D6770E94DB77EA87FB873F5FE0
:109AA400D9CF0E94BB7D2E96089524970E94B47D41
:109AB400EA85EA930E94114AEE83FF8300E010E0F6
:109AC400EB850E94C876C4F5EF85F889E887F987A5
:109AD40020E030E0EC850E9446701CF5E989FA89A3
:109AE400449155273196E98BFA8B5A934A930E94F5
:109AF4007D6DE989FA89FA93EA93EC85FD85FA93F9
:109B0400EA930E94B14CE0910D04EE0FEE0FEE0FBC
:109B1400A885B9850E944775E887F9872F5F3F4F6D
:109B2400D9CFE0910E04AD85BE850E944775ED87BF
:109B3400FE870F5F1F4FC4CF0E94BB7D63960895BD
:109B44001A93EFEF0E94B872E093380910E00E9474
:109B5400DD71E15CF54FE081EF3F31F00E94DD7192
:109B64000E94E8771F5FF3CF199108951A930A931F
:109B74000091CF0BAA81A53411F4E0E066C0AA815C
:109B8400A23539F4A0913408A13019F40E94EB777E
:109B940009F405C00E94041CE0E0E0933408AA81A3
:109BA400AB3411F0A33599F4E02FE470E43011F4F0
:109BB40014E001C013E0E02FE270E23009F41C5F0E
:109BC400E02FE170E13009F41F5FE12F3EC0AA816C
:109BD400A13511F0A13799F4E02FE470E43011F4C9
:109BE40017E001C016E0E02FE270E23009F41C5FD8
:109BF400E02FE170E13009F41F5FE12F26C0AA8154
:109C0400A33421F0A13411F0A23441F413E0E02F85
:109C1400E170E13009F41F5FE12F17C0AA81A73773
:109C240041F417E0E02FE170E13009F41F5FE12F08
:109C34000CC0AA81A03441F415E0E02FE170E130BA
:109C440009F41F5FE12F01C0EFEF1981088123960A
:109C540008950E94F177008011800E946C6E0E942A
:109C64004672EA17FB0791F10E94F177DF010E9427
:109C7400D27B0E94F9770E94F177DF010E94D27BA8
:109C8400EC59F44FE0810E9401780E9408780E9408
:109C94000B78E855F84F0E94FC710E9411780E94DD
:109CA4001578E9E3F8E10E946873E881E03039F05F
:109CB4000E940B780E9419780E944E6302C00E9491
:109CC4001D780E9415780E94016416C0E881E03076
:109CD40099F00E940B78EC55F84FDF010E94D27B7B
:109CE4000E947570E883A881A03430F4EA93E0916F
:109CF400C605EA930E9488268FC20E94217839F013
:109D04000E940B78ED55F84FE081E23009F01CC059
:109D1400A0913E09A23429F4E6E0E0933F09E03043
:109D240009F405C0E1E0EA9394DF0E942778E0910A
:109D3400640CF091650CFA93EA93E8ECF0E00E946D
:109D4400BD7311F40E9427780E94217839F00E9493
:109D54000B78ED55F84FE081E13009F022C0E0E0E6
:109D6400E09334080E94B172E0E0E0935C0BE2E01F
:109D7400EA930E941B630E940B780E9419780E9448
:109D84004E63E3E0EA930E941B63E0915C0B0E9444
:109D94002D780E9434780E94E668E093640CF09376
:109DA400650C089524970E94B47D2091CF0BA09157
:109DB4003F09A53411F00C94924FE0E0E09334088D
:109DC4000E94B172E0E0E0935C0BE091D30BE030D1
:109DD40029F50E94217839F00E940B78ED55F84F4F
:109DE400E081E13009F01AC0E7E7EA930E941B63BF
:109DF4000E940B78E855F84F0E94FC71FA93EA939D
:109E04000E943A780E9419780E943A78E755F84FF0
:109E1400E081E05D0E942D780E943478E09134085E
:109E2400E03011F00C94924F0E94EB7711F40C94F3
:109E34006C4F0E94F91BE1E0E0933408E22FE870D4
:109E4400E83081F40E943F78E8EEF3E00E94597B09
:109E5400DF010E94AA7D14F4E1E301C0E0E3EA9388
:109E64000E941B63E22FE074E03411F413E001C09C
:109E740012E0E091250C0E9402751A930E948763F8
:109E8400E22FE470E43049F40E943F78E0E1F7E225
:109E94000E948B7BAF0114E006C00E943F780E94B1
:109EA4000B74AF0113E0E22FE071E03111F4415083
:109EB40050405A934A931A930E948763E22FE072A8
:109EC400E03211F414E001C013E0E091280CF091A9
:109ED400290C17C018E0E22FE470E43009F41F5F86
:109EE400E22FE870E83009F41F5FE22FE072E032FD
:109EF40009F41F5FE22FE074E03409F41F5FE0E02F
:109F0400F0E0FA93EA931A930E948763E22FE170D8
:109F1400E13029F4E0915C0BEA930E941B6310DEAC
:109F2400A0913F09A73729F4E2E0E0933408E03038
:109F340009F42BC00E94B1720E9444780E946C7391
:109F44001E2F0E948773AF01E1E0EA930E94C26270
:109F54000E2F0E94217839F00E940B78ED55F84FAE
:109F6400E081E23009F00EC00E940B78EC55F84F06
:109F7400DF010E94D27B4E175F0711F40A9369DE5A
:109F84000E942778E0E0E0933408A0913F09A334CD
:109F940021F40E94CA33E03009F40BC00E94B1726C
:109FA4000E9444780E94C0750E94A46C68D30E94E9
:109FB400AA1CA0913F09A13411F0A23421F40E94FB
:109FC400B1720E944478A0913F09A03421F40E9408
:109FD400CA33E03009F420C00E946C73E887F98723
:109FE400E2E0EA930E94C2621E2F0E944A780E9415
:109FF400CB170E94A4740E945078E152F84F10834A
:10A004000E94A474E652F84FA7E0A0830E948572D0
:10A014000E94B1720E944478A0913F09AB3439F098
:10A02400A33529F0A13519F0A13709F07AC00E94AF
:10A03400CA33E03011F40C948D500E94B1720E9426
:10A044005778E0E4F9E00E948273E22FE270E23094
:10A0540029F4E4E0EA930E94C26202C0E1E0F0E085
:10A06400E887F987A0913F09A13511F0A13721F4C0
:10A074000E9487731E2F02C01091E50BE22FE4703B
:10A08400E43011F4E4E001C0E3E0EA930E94C26228
:10A09400AF01A0913F09A33511F0A13731F4E88550
:10A0A400F9850E94CD7AE887F9875A934A930E94EA
:10A0B40016180E2F003420F0A091D30BA13011F507
:10A0C4001A935A934A93EB85FC85FA93EA930E9478
:10A0D400C91C0E94A377EE83FF83AE81BF810E94D7
:10A0E400AA7D84F40E94B172E6E6EA930E941B639F
:10A0F400EE81FF813197EE83FF83AE81BF810E94A1
:10A10400AA7D94F31A935A934A93EB85FC850E9493
:10A114003F7316DD06C00E94C0750E94A46C0E94A5
:10A12400C91C0E94BB7D2A9608950E945B78E8941E
:10A1340022F80E947C74E2E7EA930E941B63E09198
:10A144003A08EA930E941B63EFE0EA930E941B63C0
:10A15400A0913708AA3219F41A9366D31AC0A091B1
:10A164003A080E94DD71EC59F44FE081EA1721F4BA
:10A17400E0913A08E03349F40E942D6DAC59B44F94
:10A18400E0913A08EC931A934FD322FC02C00E9448
:10A194000164C1C20E945B78E0913A08E053AE2F9B
:10A1A4000E94DD71EB58F44FE081EA1741F51A93F0
:10A1B4003BD3A0913508A23019F40E94637809F4C6
:10A1C40002C00E946978A0913508A33019F40E9456
:10A1D400637809F402C00E946978E0E0E0933508EE
:10A1E400E093660C0E94DD71EB58F44FBF01E081EF
:10A1F400EF5FAE2FEAE00E94887BDB01EC938BC219
:10A20400E881E03019F40E941D7806C0E881E85026
:10A214000E9402750E944E63219608950E94B47DA7
:10A22400A091E40BA63009F468DD25FC24C20E9449
:10A23400637811F40C948B520E946F78E752F84FB4
:10A244009F01D9011196EC91E43071F50E94757863
:10A254000E9478780E947F78F901A681A03021F4C9
:10A26400A281B381109709F007C0ECE3F8E10E94E2
:10A2740068730E94157815C00E9408780E9483783C
:10A284000E948778EFE3F8E10E9468730E948A785D
:10A294000E949078F901A085B185BA93AA930E948F
:10A2A4004E630E949678E7C1E730C9F40E9475783E
:10A2B4000E9478780E947F78E2E4F8E10E94687353
:10A2C4000E948A780E948778E5E4F8E10E94687326
:10A2D4000E9483780E944E630E949678CCC1E93034
:10A2E40089F40E9475780E9478780E947F78E8E467
:10A2F400F8E10E9468730E949D780E9487780E940A
:10A304009678B9C1E63029F5EAE2EA930E94E66359
:10A31400EBE4F8E10E946873D901EC910E94A07803
:10A32400E091CD0B0E94A078EBE4EA930E941B63BA
:10A334000E9483780E944E63E4E5EA930E941B63C3
:10A344000E948A780E944E630E9401640E94697888
:10A3540092C1E530C9F40E944E740E94F977D90184
:10A36400EC910E9401780E9408780E9483780E94F0
:10A374008778E9E3F8E10E9468730E948A780E9472
:10A384004E630E94967877C1E83039F50E9475785B
:10A394000E9478780E947F78EEE4F8E10E94687366
:10A3A400F901A681AA930E945A74309719F00E9469
:10A3B400707004C0D9011696EC91F0E0FA93EA9318
:10A3C4000E944E630E9415780E940164D90111967F
:10A3D400E0E0EC930E9469784EC1E130B9F5A091B8
:10A3E4001908A53029F4E091CD0BE65F1E2F01C0BA
:10A3F40011E0E12F0E94A4780E94DD710E94A978E7
:10A404000E9408780E9483780E948778E1E5F8E149
:10A414000E9468730E948A780E949078D9011796E6
:10A42400EC910E9402750E944E63A0911908A53018
:10A4340041F40E94AE78A481B581BA93AA930E9494
:10A44400BD630E940D760E94B47815C1E330A1F477
:10A454000E944E74F0960E94BF780E944E740E942F
:10A46400A978E4E5F8E10E9468730E948A780E9462
:10A47400C3780E94B478FFC0EB3059F50E94C678C7
:10A484000E94C978E7E5F8E10E946873F901A681A2
:10A49400AA93B6DE0E94AE78A781AA93B1DE0E9489
:10A4A400AE78A085B185BA93AA930E9490780E9451
:10A4B4008A780E949078F901A481B581BA93AA930D
:10A4C4000E9490780E949D780E94C3780E94B4787C
:10A4D400D2C0EC3079F40E94C6780E94C978EAE5CB
:10A4E400F8E10E9468730E949D780E94C3780E94DC
:10A4F400B478C1C0EE3069F40E94C6780E94C9786D
:10A50400EDE5F8E10E9468730E940D760E94B4782C
:10A51400B2C00E94EB7761F0A0913508A03041F4FD
:10A52400A091D20BA13021F40E946C6EE13009F4A9
:10A5340026C0A091850BA03059F0E091870BF091D3
:10A54400880BFA93EA93E8EEF3E00E94BD73B9F442
:10A55400E1E30E94BF78E091760BE05D0E94017810
:10A564000E946C6EEA9314D1E09335080E940D7634
:10A57400E093620CF093630CE0E0E093850BA09110
:10A584003508A03059F0E091620CF091630CFA9315
:10A59400EA93E4E6F0E00E94BD7309F025C0A091BF
:10A5A4003508A23019F40E94637809F402C00E94AD
:10A5B4006978A0913508A33019F40E94637809F4EE
:10A5C40010C0A091660CA33030F00E946978E0E0DE
:10A5D400E093660C06C00E946F78E652F84FA8E03C
:10A5E400A083E0E0E0933508A091860BA13011F040
:10A5F4000C943D53E0913A0CA091390CEA17B1F157
:10A60400EAE20E94BF78E091740BE05D0E94017859
:10A61400E0913A0CEA930E94611E0E940878E0914E
:10A624002A0C0E9402750E948778E0E6F8E10E94F5
:10A6340068730E945E710E941178EAE3EA930E94B3
:10A644001B630E94ED740E9411780E9415780E9489
:10A654000164E0913A0CEA930E94A31CE0913A0C45
:10A66400EA930E94721CE0933A0C05C0E0E0E09388
:10A67400860B689420F80E94BB7D269608951A9351
:10A684000A930E94CA33E030D9F00E94A474E752BE
:10A69400F84F8F01EC81FD81D8011296ED93FC9364
:10A6A400EA81FB81D8011896ED93FC93EE81D801E1
:10A6B4001696EC93D8011196E4E0EC930E9485720F
:10A6C4001981088127960895E091410BEA930E942D
:10A6D4001B63E091420BEA930E941B630895F4DF2D
:10A6E4000E94D1770E94CD780E94CD780E9487780D
:10A6F40099C01A930E944E621E2F103021F0E12F50
:10A70400E150E0933F0BE0DFE0913F0BEF5F0E94ED
:10A7140002750E948778199108950E94B67D31E0F0
:10A724000E94D47828F00E947673AC91A43308F088
:10A734002AC030E00E947673EC91E270E6951E2FF9
:10A744000E947673EC91E1700E2FA091590B1A17A9
:10A7540029F4E1E0EA27E093590B31E0A0915A0B88
:10A764000A1729F0E1E0EA27E0935A0B31E0E0917F
:10A774005A0BEE0FE05DA091590BEA0FEA930E9489
:10A784001B630E946D74E32F0E94BD7D249608957F
:10A794001A9310E00E94EB7711F40C9412540E9467
:10A7A400F91BE4E6F8E10E946873E091250C0E942D
:10A7B40002750E948778E7E6F8E10E946873E091E9
:10A7C400280CF091290C0E9411780E9415780E949F
:10A7D4003F78A031E7E2BE074CF4EAE6F8E10E94D4
:10A7E4006873E091260CF091270C13C0EDE6F8E1B4
:10A7F4000E946873E9810E94CD710E943F78EA0F3C
:10A80400FB1F0E941971E091260CF091270CE05176
:10A81400F742FA93EA930E944E630E94157811E07E
:10A82400E12F18812296089524970E94B47D0E94F6
:10A83400D878E0E0EC930E94F561E13010F40C94D8
:10A84400FB56E091410BEB3441F4E091420BE332CF
:10A8540019F40E944E621E2FC9C2E435A9F4E09196
:10A86400420BE33221F40E944E62EE83FF83E091B7
:10A87400420BEF3441F40E944E621E2F1A930E9441
:10A8840042750E94CB17B2C2E23411F00C94915578
:10A89400E091420BE13251F4AA85AF3F29F40E94C2
:10A8A400C0750E94A46CEBDE0E94AA1CE091420BCE
:10A8B400E134E1F40E944E621E2F113071F4A09134
:10A8C4003508A13019F40E94EB7709F402C00E9404
:10A8D400041CE0E0E093850B09C0E1E0E093850B04
:10A8E4000E94E668E093870BF093880BE091420B9B
:10A8F400E534A9F4E0E7F8E10E9468730E94E11BE3
:10A90400F3973CF00E944E620E9419710E94DD7818
:10A9140001C0E0E3EA930E941B630E941578E09172
:10A92400420BE63409F50E94E97819F40E944E625C
:10A93400AF01E885F9850E9475700E2FE091E50B53
:10A94400E03011F01091E50B003420F0A091D30B0E
:10A95400A13021F40E94F5780E94C91CAA85AF3F5A
:10A9640019F40E94F5788BDEE091420BE23511F088
:10A974000C944E550E94E97819F40E944E62AF017E
:10A9840030E0A091D30BA03021F40E946C6EE13032
:10A9940009F027C00E94D033E03011F10E943373D4
:10A9A400EC55F84FA885B985A083B1830E94337311
:10A9B400E655F84FDF01EA850E9481720E943373E5
:10A9C400E855F84F10830E943373E755F84F4083DE
:10A9D4000E943373ED55F84FA1E0A0830E943973B0
:10A9E40059C00E94CA33E23010F40C944C550E94B2
:10A9F4004A780E94DB1D3E2F3F3F29F00E943171AF
:10AA0400A417B5070CF412C00E94ED74E41BF50BF7
:10AA14000E943F710E94107319F4E0E0E0932A0C45
:10AA24003A930E94681E689420F803C0E0E0E88727
:10AA3400E9870E94A474E752F84FDF01EA85F0E049
:10AA4400EC59F44FE081EC930E94A4740E94507876
:10AA5400EF51F84FDF01EA850E9481720E94A474CD
:10AA6400E152F84F10830E94A474E652F84FA5E017
:10AA7400A0830E948572E885F985309759F00E9479
:10AA84004A78FA010E94CD7A0E943F730E94F578B9
:10AA94000E94531C689422F8E091420BE335F1F5CF
:10AAA4000E944E62E887F9870E946F78DF01E652C0
:10AAB400F84FE081E23081F4FD01EF51F84F00805E
:10AAC40011800E946C6E0E944672EA17FB0721F403
:10AAD400A0913508A23009F01FC00E946F78E5529A
:10AAE400F84FDF010E94D27BDF01E885F985EA1780
:10AAF400FB0779F40E946F78DF01ED51F84FE08194
:10AB0400EA93FD01E752F84FE081EA930E94882618
:10AB140003C0E7E0E0932406689422F867C1E434B4
:10AB240011F00C94F955E091420BE33559F4E3E745
:10AB3400F8E10E9468730E94D85E0E94A078E1E068
:10AB4400E0933809E091420BE03511F00C94F8558C
:10AB54000E94F97811F40C94F85520E00E94FF78D3
:10AB640040F00E947673AC91A23219F00E940379EE
:10AB740009F43CC0E22FE03061F40E947673AC919A
:10AB8400A33211F421E004C00E9407790E94B35E4D
:10AB94002AC0E13051F40E947673AC91A43211F4CE
:10ABA40022E001C020E010E01EC0E23011F0E330EA
:10ABB400D1F40E9407790E94BE68EF3F99F0E12F1B
:10ABC400E295E07FEF930E9407790E94BE68AF91FF
:10ABD400EA0F1E2F2F5F243021F41A930E94B35ED4
:10ABE40020E001C020E00E946D74B8CFFFC0E334C0
:10ABF40011F00C946956E091420BE534B9F4E0E7A6
:10AC0400F8E10E9468730E94E11BF3974CF00E94E4
:10AC14004E62E05FF84D0E9419710E94DD7801C018
:10AC2400E0E3EA930E941B630E941578E091420BD3
:10AC3400E634D9F441E050E00E944E620E2F0E94A7
:10AC44000B79E13019F40E944E62AF01E091E50BFB
:10AC5400E03011F01091E50B1A930E94126DE05F41
:10AC6400F84D0E942A770E94C91CE091420BE335FB
:10AC7400A1F40E940F790E946B70E83141F4E091D5
:10AC8400890BEA930E947A17689420F806C0E88535
:10AC9400EA93EFEFEA930E948826E091420BE134B5
:10ACA400A9F4E6E7F8E10E9468730E940F79EA9339
:10ACB4000E9477180E94BB25E03011F0E1E301C047
:10ACC400E0E3EA930E941B630E9415788FC0E63587
:10ACD40011F00C94D056E091420BE33411F00C9433
:10ACE400CF560E944E621E2F113010F40C94CF5692
:10ACF400A0911908A13011F0A93091F50E940B79A7
:10AD0400E03021F0A091A2061A1709F028C01150D2
:10AD14000E944E62AF011A930E9415213E2F0E9499
:10AD2400D2730E94F7710F010E94D2730E945A6E6F
:10AD34000E9416790E940B79E03071F00E944E62F5
:10AD4400AF010E94E6730E94F7710F010E94E6733F
:10AD54000E945A6E0E9416791A930E9420111DC0F7
:10AD64001630D8F41150A12FEAE00E94387BA3E2F8
:10AD7400EA9FF001E855F94FBF01A12FEAE00E94D4
:10AD8400887BF0E0BB01AAE0B0E00E94067BDB0117
:10AD9400AE0FBF1F14960E948B7128C0E93431F5A1
:10ADA400E091420BE03551F40E944E621E2FE0E028
:10ADB400EA931A930E944A18E0932E06E091420BFC
:10ADC400EC34A1F40E941062E09328060E940B79EF
:10ADD400E03021F00E941062E09329060E940B7972
:10ADE400E03021F00E941062E0932A060E94B161D3
:10ADF40022CD0E94BB7D2B960895A091570BA035C0
:10AE040021F4A091580BA03408F005C0E091580B30
:10AE1400EA930E949718A091570BA33521F4A091AF
:10AE2400580BAA3008F005C0E091580BEA930E9431
:10AE3400C218A091570BAB3421F4A091580BA03841
:10AE440008F005C0E091580BEA930E94FE18A09107
:10AE5400570BA63521F4A091580BA03108F005C07A
:10AE6400E091580BEA930E942A19A091570BA4353C
:10AE740011F40E94B517DDD60895E3EAF6E0FA93DB
:10AE8400EA93E091410BEA93E0E8F0E00E949770C6
:10AE940008950E941E79A0E0A083E0913F0BE09307
:10AEA400580BE091410BE093570B08950E94B47D39
:10AEB4000E94F561E13010F40C94735AE091570B41
:10AEC400A091410BEA1709F098DFE091410BE332BE
:10AED40039F5E091420BEC3431F4CFDFE4E0E09358
:10AEE40018080E942479E091420BE435C1F4C5DFCF
:10AEF400E091690CE03029F0EF77A9E0B0E00E941E
:10AF0400147CE0916A0CE03029F0EF77AAE0B0E01D
:10AF14000E94147C0E942479E7E0E0931808DEC2C2
:10AF2400E934E9F4E091420BE434C1F40E94F97885
:10AF3400A9F010E010E0183178F4A3E2B7E00E9421
:10AF4400DD71EA0FFB1FFF93EF930E941062AF9134
:10AF5400BF91EC931F5FEFCF0E94CB0CBFC2EB34C9
:10AF6400E1F5E091420BE13211F487DF35C0E532BF
:10AF740011F443DF31C0E33299F40E942A7921F0BD
:10AF84000E9435790E94CC180E941E79E081EB342E
:10AF940029F4E0E0E093350CE093360C7ADF1CC032
:10AFA400E134D1F40E944E629F012093350C0E943B
:10AFB4003B7991F00E944E629F01A091350CF901FA
:10AFC400E270F070EA2BE093350C0E943B7921F09B
:10AFD4000E944E62E093360C81C2E33581F5E09124
:10AFE400420BE13211F449DF29C0E33299F40E94A3
:10AFF4002A7921F00E9435790E94A6180E941E79B0
:10B00400E081E33529F4E0913F0BEA930E94EC1AC6
:10B0140040DF14C0EE3491F40E94257510E01A301C
:10B0240068F4A3EBBBE0EE27A10FBE1F0E94DD7105
:10B03400ED5BF44FE081EC931F5FF1CF4FC2E63537
:10B0440011F00C946D58E091420BE13211F415DFCC
:10B0540041C0E33299F40E942A7921F00E943579A3
:10B064000E940A190E941E79E081E63529F4E091D4
:10B074003F0BEA930E943D190CDF2CC0E63531F4F6
:10B084000E944E629F012093310C24C0E53471F478
:10B094000E944E629F012093300C0E943B7929F05C
:10B0A4000E944E629F012093330C14C0E43591F446
:10B0B40040E050E00E944E629F01022E032A11F0EC
:10B0C40042E050E00E943B7919F00E944E62AF01C9
:10B0D4004093320C03C2E43511F00C942759E091EB
:10B0E400420BE33231F40E944E623197E0933F0BFE
:10B0F400ABC0E03511F00C94265910E00E94FF78A3
:10B1040050F00E947673AC91AD3329F00E9403791C
:10B1140011F01E3008F005C00E94DD710E944179D3
:10B12400EDCF0E94DD710E944A79EDE30E944F79D0
:10B1340011F00C942659E4E5E093570B10E00E94BB
:10B14400F7703496E491EF3F11F40C9426590E9461
:10B1540029750E94F7700E940A6E0E947E69E03091
:10B1640011F00C9424590E94F7703496E491E0385D
:10B1740051F40E944E62E058FF4FE093690CE0E8FE
:10B18400E0936A0C5FC0E23839F40E944E62E058E2
:10B19400FF4FE0936A0C56C0E13839F40E944E62C6
:10B1A400A8E0B0E00E94147C4DC0E03011F0E13022
:10B1B40051F40E94ED70FF93EF930E944E62AF91A1
:10B1C400BF91EC933FC0E23059F40E94ED70FF93BD
:10B1D400EF930E944E62AF91BF91ED93FC9332C006
:10B1E400E33051F40E94ED70FF93EF930E942D62BF
:10B1F400AF91BF91EC9326C0E43021F50E94F77023
:10B204003596E491EA930E94FC620E94ED70E0930B
:10B21400670CF093680C00E00E94F7703596E49197
:10B224000E1780F40E94126DED5BF44FE081A09143
:10B23400670CB091680CEC93A7E6BCE00E940F6F1A
:10B244000F5FEACF1F5F7BCF49C1E03511F00C944B
:10B25400705AE091420BE33299F40E942A7921F06A
:10B264000E9435790E9477180E941E79E081E035AA
:10B2740029F4E0913F0BEA930E94031B0ADE2EC1DE
:10B28400E13211F4FADD2AC1E134D1F40E944E62B4
:10B294001E2F00E00D3098F40E944B75EA0FFB1F3F
:10B2A4003396E491E11749F40E944B750E944F755F
:10B2B400A0919A0BEA2BE0939A0B0F5FEBCF0EC190
:10B2C400E63559F5E0E0E093400BADE9BBE00E94C0
:10B2D4005479FF93EF930E944E62AF91BF91EC9328
:10B2E400EBE2EA930E94C161E03059F0A0EABBE0CE
:10B2F4000E945479FF93EF930E944E62AF91BF91E5
:10B30400EC930E945779A091400BA33018F40E944B
:10B314003B7909F401C0D9CFE1C0ED34D1F4E0E0C8
:10B32400E093400BA9EABBE00E945479FF93EF93AA
:10B334000E944E62AF91BF91EC930E945779A09105
:10B34400400BA33018F40E943B7909F401C0EACF02
:10B35400C5C0E735D1F4E0E0E093400BA0EBBBE0DF
:10B364000E945479FF93EF930E944E62AF91BF9174
:10B37400EC930E945779A091400BA23018F40E94DC
:10B384003B7909F401C0EACFA9C0E434C9F5E0E08F
:10B39400E093400B0E944E629F01E2E0EA930E9418
:10B3A400CE61AF01E3E70E944F7959F40E945D79C1
:10B3B400BF01D9010E947C72E40FF51FDB01ED93FC
:10B3C400FC93E9E40E944F7979F40E945D7920832B
:10B3D4003183AAE9BBE00E9454790F010E9463798A
:10B3E400EC91E160D001EC930E945779A091400B5D
:10B3F400A33018F40E943B7909F401C0CBCF6EC08E
:10B40400EE3499F40E94257510E01A3068F4AAE825
:10B41400BBE0EE27A10FBE1F0E94DD71ED5BF44F70
:10B42400E081EC931F5FF1CF59C0E33459F4E2E2B9
:10B43400EA930E94C1610E944E62E093950BF093DF
:10B44400960B4CC0E33589F40E944E629F010024A0
:10B454000216030624F42B30E0E03E070CF004C08F
:10B46400F9013197E093970B39C0E53529F40E942F
:10B474004E62E093990B32C0EF3491F40E944E6215
:10B484001E2FECE2EA930E94C161E12FE295E07F76
:10B49400EF930E944E62AF91EA0FE093980B1EC0A7
:10B4A400E035E1F4E0E0E093400BACEABBE00E945D
:10B4B40069790E94F771FF93EF930E94DC62AF9168
:10B4C400BF91ED93FC930E945779A091400BA23059
:10B4D40018F40E943B7909F401C0E7CF0E94B161DE
:10B4E400E7CC0E94BB7D269608950E94B67D0E94FB
:10B4F400F561E13010F40C944A5DE091410BE332C4
:10B50400A9F4E091420BE03519F4E9E7F8E109C048
:10B51400E83419F4EAE9F8E104C0E33531F4E5EB81
:10B52400F8E1FA93EA930E942C63AFC2E934C1F4C0
:10B53400E091420BE43499F40E94C00CC5D80E94F7
:10B544006D7910E0183148F4A3E2B7E00E94167652
:10B55400EA930E945C631F5FF5CF0E946D7995C2E8
:10B56400E43511F00C944E5BE091420BE43229F483
:10B57400E9E2F0E00E9471798EC0E33211F4B9D8A7
:10B584008AC0E03511F00C944D5B9ED8A0913F0B1E
:10B59400A93210F00C944D5B0E9475790E940A6EDA
:10B5A4000E942C63EDE3EA930E941B630E94757969
:10B5B4003496E491E03839F40E946C6E0E9402756E
:10B5C4000E944E6368C0E23839F40E94E8700E9419
:10B5D40002750E944E635FC0E13839F40E94FD7425
:10B5E4000E9402750E944E6356C0E03011F0E130B3
:10B5F40051F40E94757932960E94E17B0E94FC719D
:10B604000E94117848C0E23059F40E94757932964C
:10B614000E94E17BDF010E9468740E944E633BC07C
:10B62400E33051F40E94757932960E94E17BE08107
:10B63400EA930E946B632FC0E43069F50E94757928
:10B6440032960E94E17BE093670CF093680C10E063
:10B654000E9475793596E4911E1790F40E94DD716D
:10B66400ED5BF44F0F01A091670CB091680CEC9165
:10B67400D001EC93A7E6BCE00E940F6F1F5FE8CFF8
:10B684000E9475793596E491F0E00E944A790E940F
:10B6940029750E94B463F9C1E33581F5E0913F0B4C
:10B6A400EA930E94A618E091420BE43229F4EAE0FE
:10B6B400F0E00E94717921C0E33211F41AD81DC060
:10B6C400EE34D9F40E94665310E01A3068F40E94F4
:10B6D400DD71ED5BF44F0F01A3EBBBE00E94167626
:10B6E400D001EC931F5FF1CFE0E0E0934D0B0E949B
:10B6F40029750E94B4630E941578C7C1E63511F01C
:10B704000C94C35BE0913F0BEA930E940A19E09109
:10B71400420BE43229F40E94BB750E94715330C07D
:10B72400E33219F40E947B532BC0E53459F40E9490
:10B734006653E091300C0E9402750E947979E09181
:10B74400330C19C0E63529F40E946653E091310C9C
:10B7540012C0E435A9F40E946653E091320CE03043
:10B7640011F0E1E301C0E0E3EA930E941B630E944D
:10B774007F79E091320CF0E00E9411780E941578F4
:10B7840084C1E03511F00C94145DE0913F0BEA9311
:10B794000E947718E091420BE43229F4E0E4F0E0EF
:10B7A4000E9471793EC1E33219F40E947B5339C17E
:10B7B400E13411F00C94205C0E94665312E0A091D5
:10B7C4009A0BECEDEA233E2F00E00D3078F40E9452
:10B7D4004B750E944F75E31739F40E944B75EA0FBD
:10B7E400FB1F3396149102C00F5FEFCF0E94ED6DE3
:10B7F4000E948778E091980BE03089F0E0EDF8E161
:10B804000E9468730E94C76D0E9402750E94797934
:10B81400E091980BEF700E9402750E948778E09186
:10B82400990BE03051F0E3EDF8E10E946873E09188
:10B83400990B0E9402750E948778F3C0E43479F56D
:10B844000E948379A091400BA33040F5E091400B16
:10B85400E03011F00E947F790E946379EC91E170ED
:10B8640061F4A3EABBE00E9469790E945A6E0E94C7
:10B8740068740E94BD63E3E70BC0A3EABBE00E94C7
:10B8840069790E945A6E0E9468740E944E63E9E4CA
:10B89400EA930E941B630E945779D4CFBEC0ED3453
:10B8A400C9F40E948379A091400BA33090F4E091F5
:10B8B400400BE03011F00E947F79A9EABBE00E94BE
:10B8C4008979EC910E9402750E944E630E94577917
:10B8D400EACFA3C0E735C9F40E948379A091400B55
:10B8E400A23090F4E091400BE03011F00E947F7997
:10B8F400A0EBBBE00E948979EC910E9402750E9442
:10B904004E630E945779EACF88C0E63531F50E942C
:10B914008379A091400BA330F8F4E091400BE03020
:10B9240011F00E947F79ADE9BBE00E948979EC9126
:10B934000E9402750E944E63EBE2EA930E941B632D
:10B94400A0EABBE00E948979EC910E9402750E94F2
:10B954004E630E945779DDCF60C0EE34D1F40E946B
:10B96400665310E01A3068F40E94DD71ED5BF44F09
:10B974000F01AAE8BBE00E941676D001EC931F5F8A
:10B98400F1CFE0E0E0934D0B0E9429750E94B4636F
:10B9940044C0E33499F40E9466530E942975EBED88
:10B9A400F8E1FA93EA930E9470700E9481740E94F5
:10B9B40011760E9429750E94B4632FC0E035A9F462
:10B9C4000E946653E091AC0BF091AD0BFA93EA93AD
:10B9D4000E94D5630E947F79E091AE0BF091AF0B8A
:10B9E400FA93EA930E94D56318C0E33531F40E94B8
:10B9F4006653E091970BEF5F0DC0EF3491F40E9412
:10BA040066530E94C76D0E9402750E947979E09185
:10BA1400980BEF70F0E00E941178EBE3EA930E9438
:10BA24001B6333C0EB3489F5E0913F0BEA930E942A
:10BA3400CC18E091420BE43229F4E0E8F0E00E94F3
:10BA4400717923C0E33219F40E947B531EC0E134A0
:10BA5400E1F40E946653A091350CE1E0EA230E94D0
:10BA640002750E947979A091350CE3E0EA230E94E3
:10BA740002750E947979E091360C0E9402750E9449
:10BA84004E63EEEDF8E10E9468730E94B1612FCD20
:10BA94000E94BD7D249608951A930E94B172EFE32B
:10BAA400F9E00E9482730E948D79E181E43471F49B
:10BAB4000E948D7902800E946C6EE05DE01529F091
:10BAC4000E948D79E281EA3209F401C05BC00E94D0
:10BAD40092790E948D79E1810E9496790E948D79F4
:10BAE400E2810E9496790E9476731C910E948D795E
:10BAF40033960E948273E12FE23139F40E94D878A0
:10BB04001397E6E0EC93D2D93DC0E13139F40E94B9
:10BB1400D8781397E2E1EC93E8DC34C0EF30B1F469
:10BB24000E94D8781397EEE0EC930E948F53E13093
:10BB340039F4A0913408A03019F00E94EB7709F48D
:10BB440002C00E94041C0E9499791CC0EE30D1F4FA
:10BB54000E94D8781397EFE0EC930E948F53E13062
:10BB640089F4A0913408A03019F00E94EB7709F40D
:10BB740002C00E94041CE0E0E0933408EFEFEA9373
:10BB84000E9416540E94D878E0E0EC9373C21A9392
:10BB94000E947C740E94C770EAE7EA930E941B63C8
:10BBA4000E94767311971C91E12FE23131F4E6E0A3
:10BBB400EA930E941B637AD931C0E13131F4E2E1A6
:10BBC400EA930E941B6391DC29C0EF3089F4EEE014
:10BBD4000E94A07939F4A0913408A03019F00E9491
:10BBE400EB7709F402C00E94041C0E94997916C0E4
:10BBF400EE30A1F4EFE00E94A07981F4A091340822
:10BC0400A03019F00E94EB7709F402C00E94041CD2
:10BC1400E0E0E0933408EA930E9416540E94D87836
:10BC2400E0E0EC93A0913708AA3211F00E9401647D
:10BC340021C2EFEFE093570BE093580B0895AC81CA
:10BC4400A03310F0AA3308F006C00E94A779E0538D
:10BC54000E94AF79ADC4AC81A13410F0A73408F0D0
:10BC640006C00E94A779E7530E94AF79A1C4A881B6
:10BC7400B981E0E0EC939CC4AA93EA93FA93EFB7FA
:10BC8400EA931A930A931BB10CB1E091A30CF0E070
:10BC9400EF58F34F0083A091A30CAF5FA093A30CC4
:10BCA400A23319F4E0E0E093A30C0991199105C3C0
:10BCB4001A93E091A40CA091A30CEA17D1F3F0E03D
:10BCC400EF58F34F1081A091A40CAF5FA093A40C84
:10BCD400A23319F4E0E0E093A40CCBC1A091A30C2F
:10BCE400AE5CE091A40CAE1BE2E30E94887B089555
:10BCF4000A921A92FA926A937A938A939A93AA93DB
:10BD0400BA93EA93FA93EFB7EA930E94B47949F0AD
:10BD1400A0913809A03021F00E94BA0CE13009F456
:10BD240001C011C0E0910A0DF0E0EB55F34FE08142
:10BD3400ECB9A0910A0DAF5FA0930A0DA43619F4D3
:10BD4400E0E0E0930A0DE991EFBFF991E991B9912F
:10BD5400A9919991899179916991F9901990099092
:10BD640018951A930E94B47959F45D9B09C0A09167
:10BD74003809A13021F40E94BA0CE03009F013C054
:10BD84001091090D0E94DD71EB55F34FA981A08339
:10BD94001F5F143609F410E0E0910A0DE117E1F396
:10BDA4001093090D02C0E981ECB9B3C20E94B479C1
:10BDB40021F40E94BA0CE13009F001C02BC362C126
:10BDC4000E94B67D8BDFE03011F40C94F25F70DFDB
:10BDD4001E2FA0916E0CA53618F0E0E0E09339090F
:10BDE40030913909E0913909E03011F00C94595F30
:10BDF400A091E40BA63029F4163011F0153109F4A2
:10BE040001C004C010933F09E2E4E0C0A091E40B38
:10BE1400A13041F0A091E40BA23021F0A091E40BF9
:10BE2400A53031F4E12FEF77E0933F09EBE4CEC086
:10BE34001A3521F4E1E0E0933909CAC0123049F41B
:10BE4400E4E1E0933909E0E0E0933A09E0933C0946
:10BE5400BFC0A091E40BA33069F4173729F01A335B
:10BE640010F4103308F402C0E7E001C0E0E0E0930E
:10BE74003B0905C01A930E94B84DE0933B09A09179
:10BE84003B09AF3F99F010933F09E1E0E0933A0991
:10BE940010933C09E0913B09E03011F4E5E404C05F
:10BEA400EAE0E0933909E0E0E0933E0991C0E13033
:10BEB40069F4103039F4E2E0E0933909E0E0E0930A
:10BEC4003E0903C0E0E0E093390982C0E23059F44E
:10BED40010933B0910933C09E0E0E0933A09E3E056
:10BEE400E093390975C0E330F1F40E94BA790E94F5
:10BEF400C079EA0F0E94CA79A9F4E0913C09E030C4
:10BF040071F4E4E0E0933909E0913A090E94137076
:10BF14000E94D3790E94BA79A0E0A08303C0E0E034
:10BF2400E093390955C0E43049F41D3019F4EAE5C9
:10BF3400E0933E09E0E0E09339094AC0EA3079F43D
:10BF44000E94BA790E94C079EA270E94CA7931F422
:10BF5400E0E0E0933909E5E4E0933E0939C0E431D7
:10BF6400B9F40E94BA791083E12FA0913C09EA2721
:10BF7400E0933C09E0913A09EF5FE0933A09E0E08D
:10BF8400E0936D0C133019F4E5E1E093390920C016
:10BF9400E53111F0E63159F41A93EDE6FCE0FA9339
:10BFA400EA93E9E3F9E0FA93EA9349DE11C0E73151
:10BFB40079F4E0E0E0933909173131F4E0916D0C44
:10BFC400A0913C09EA1709F003C0E3E4E0933E09B9
:10BFD400A09139093A1719F0E0E0E0936E0CF2CE23
:10BFE4000E94BD7D50C4AA93BA93EA93FA93EFB723
:10BFF400EA931A930A9310919B0000919C00E12FFD
:10C00400EC71A9F4E091D30DF091D40DE55FF24FFA
:10C014000083A3EDBDE00E940F6FE83CA0E0FA07A7
:10C0240031F4E0E0F0E0E093D30DF093D40D099106
:10C034001991E991EFBFF991E991B991A9911895F5
:10C044001A930E94D8790E94DD79D9F30E94D87995
:10C05400E55FF24F1081A5EDBDE00E940F6FE83C53
:10C06400A0E0FA0731F4E0E0F0E0E093D50DF093BE
:10C07400D60DE12F199108950E94D8790E94DD7997
:10C0840009F0C8C1E0E008950E94B67DF5DFE03014
:10C0940021F0A0916C0CA03009F0E5C0D1DF1E2F77
:10C0A400A091DF0DA53618F0E0E0E093D90D3091B2
:10C0B400D90DE091D90DE03059F4113019F4E4E0D0
:10C0C400E093D90D1A3519F4EAE0E093D90DC3C011
:10C0D400E430C1F4E0E0E093D90D1A3229F00E9473
:10C0E4006C6EE05DE11769F4109337081093DA0D74
:10C0F400E5E0E093D90DE0E0E0936C0CE1E0E0933F
:10C10400DC0DA9C0E530A9F4E0E0E093D90D0E946C
:10C114006C6EE05DE11761F00E94E4790E94ED79B4
:10C12400E091DC0DEF5FE093DC0DE6E0E093D90DE8
:10C1340092C0E63091F4E091DC0D0E94ED790E940A
:10C14400E479EF5FE093DC0DE0E0E093DD0D133084
:10C1540019F4E7E0E093D90D7EC0E73011F0E83040
:10C1640059F41A93EDEDFDE0FA93EA93E9EDFDE05D
:10C17400FA93EA9364DD6FC0E93081F4E0E0E09380
:10C18400D90D173131F4E091DD0DA091DA0DEA17E4
:10C1940009F003C0E4E5E0936C0C5DC0EA3041F4BF
:10C1A400103011F4EBE001C0E0E0E093D90D53C08E
:10C1B400EB3071F4E0E0E093DC0D1093DB0D1093B1
:10C1C400DA0DECE0E093D90DE0E0E0936C0C43C0B1
:10C1D400EC30A1F5E091DC0DF0E0E15CF64F10836A
:10C1E4000E94E479EF5FE093DC0DE091DB0DE15018
:10C1F400E093DB0DA091DB0DA03021F4A091DA0DCA
:10C20400A03009F00EC0EDE0E093D90DE091DC0D13
:10C214000E9413700E94D379E091DC0DF0E00E943B
:10C22400D379A091DB0DA03021F4A091DA0DA030D8
:10C2340009F403C0E0E0E093D90D0DC0ED3059F4EA
:10C24400E0E0E093D90D1D3031F4EAE5E0936C0CA5
:10C25400EFEFE0936B0CE091D90DE31719F0E0E0F8
:10C26400E093DF0D13CF0E94BD7D0DC3AA93EA9323
:10C27400FA93EFB7EA93E091E10EA091E00EEA178A
:10C2840091F0E0913608E03019F0E89426F80AC0FD
:10C294000E94F279F0E0E030A1E0FA0719F4E0E05E
:10C2A400E093E10E03C0E89425F826F8E0916B0CC6
:10C2B400E03019F0E0E0E093D90DE991EFBFF99196
:10C2C400E991A99118951A93E091E10EA091E00EDD
:10C2D400EA1721F4E0919B00E072C1F4E091E00ED2
:10C2E400F0E0E052F24FA981A0831091E00E1F5FAD
:10C2F4000E942D6DA030E1E0BE0709F410E0E0914A
:10C30400E10EE117E1F31093E00E03C0E981E0933D
:10C314009C00188122960895E0E0E093E10EA0913C
:10C32400E00EA13020F00E94F279689426F8089576
:10C33400AA93BA93EA93EFB7EA93E0916B0CE030D7
:10C3440041F4E0E0E093E10E0E946C6EEF5FE09355
:10C354003608E991EFBFE991B991A99118950E9426
:10C36400FF7818F00E94037909F403C00E946D74E9
:10C37400F6CF0E94037911F40E946D7408950E940F
:10C384007673AC91E881EA1729F40E946D743197B1
:10C39400E1E05EC1E0E05CC10E94B67D00E010E037
:10C3A400EEE20E944F79E9F420E030E0EC810E9453
:10C3B4004670BCF4D8010E9438758F010E94D4786D
:10C3C40018F00E94007A08F009C00E947673EC917C
:10C3D4000E9410740E0F1F1F0E946D742F5F3F4F39
:10C3E400E5CFF801E3C00E94FF7828F00E948D7920
:10C3F400E181E03208F410C00E947673EC91E0937E
:10C40400410B0E946D740E947673EC91E093420B91
:10C414000E946D74E1E008950C9420671A930A93C6
:10C4240000E010E01230A8F40E9407790E94BE6870
:10C43400EF3F69F0E02FE295E07FEF930E940779E8
:10C444000E94BE68AF91EA0F0E2F0E946D741F5FA9
:10C45400E9CFE02F1EC01A930A9310E00E9476736E
:10C464000C910B3311F0003208F412C0013310F0B8
:10C47400093308F007C0E02F0E941074E853FF4FFF
:10C48400E4911E2B0E946D740E9476730C91E9CF87
:10C49400E12F0991199108950E94B67D00E010E002
:10C4A4000E947673AC91AD3221F40E946D7431E038
:10C4B40001C030E00E94D47818F00E94007A08F09D
:10C4C40009C0D8010E9438750E94047A8F010E9425
:10C4D4006D74F0CF303021F4F8010E94BD7DD3C1DA
:10C4E400F8010E94CD7A0E94BD7DCDC124971A9394
:10C4F400E0E0E983EA83EB83EC830E947673AC91FA
:10C50400AD3221F40E946D7411E001C010E00E946C
:10C51400D47818F00E94007A08F022C0A981BA8168
:10C524008B819C81EAE0F0E060E070E00E94337B64
:10C534007F936F93FF93EF930E947673EC91E05394
:10C54400AF91BF918F919F91FF27662777270E9414
:10C55400C37AE983FA836B837C830E946D74D7CF9B
:10C56400103031F4E981FA816B817C81188120C01B
:10C57400E981FA816B817C810E94D17A188118C08B
:10C584000E94B67D20E030E000E010E0EC810E94E3
:10C59400C8765CF4D9010E9438750E94047A9F0120
:10C5A4000E946D740F5F1F4FF1CFF9010E94BD7D92
:10C5B400259608950E94B67D6FDF8F0120E030E05C
:10C5C400EEE20E944F7911F467DF9F01112322F4F8
:10C5D400F9010E94CD7A9F01A0911B0CA13030F08B
:10C5E400D8010E947C72E20FF31F8F01F8010E94B0
:10C5F400BD7D49C11A9310E00E94F978A1F00E9410
:10C60400FF7858F00E947673AC91A23231F00E9408
:10C61400037919F0E9811E1708F005C00E94DD7145
:10C624000E944179ECCF0E94DD710E944A790C94FA
:10C634007C67E8810E949679E881A0915B0BEA0F00
:10C64400E0935B0BE881A0915C0BEA27E0935C0B21
:10C65400219608951A9310E0E12FA981BA810E94CE
:10C664004775E491E03049F0E12FA981BA810E9435
:10C674004775E4910E94097AEFCF0BC01A9310E03A
:10C684000E94B976E03029F00E94B9760E94097AB6
:10C69400F7CF18812396089564970E94D3750E945A
:10C6A4000E7AE88DF98D0E9481740E940376E6DF8C
:10C6B4006696089564970E94D375E7EEF8E1FA93BD
:10C6C400EA93E88D0E94EA6C0E94D375D7DF6596E1
:10C6D40008951A93ECE3EA93ACDF11E0193080F487
:10C6E4000E94DD71E853FF4FE491A981EA2319F018
:10C6F400E12FE05D01C0E0E2EA939BDF1F5FEECF34
:10C70400EEE3EA9396DF0C947C6764971A930E9495
:10C71400137A0E940E7AEA8DFB8D0E9481740E9426
:10C7240011760E94137A0E94A6691E2FED891E17A6
:10C7340020F40E941D781F5FF9CF0E94137A9EDFB8
:10C7440018810EC064970E94D3750E940E7AE88DFA
:10C75400F98D6A8D7B8D0E94D5740E94D3758EDF0E
:10C76400689608950E946D790E94D17787DF0E94B0
:10C774006D790C947D67A881B981E4E6F0E00E94AC
:10C78400597B0E941178EEE2EA9353DFA881B981C4
:10C79400E4E6F0E00E948B7BFA93EA93E2E0EA930A
:10C7A400B4DF0C947D67A0911B0CA13020F00E9493
:10C7B400D177E1DF07C00E94D1776EDFECEEF8E1BC
:10C7C4000E9468730C947D6725FE06C0E5E0F0E0E6
:10C7D4000E94EA6EA895F8CFE0EEFDE0E0935D0BD1
:10C7E400F0935E0BE1E00E94B872E0935B0B0E9451
:10C7F400187A0E946C6E0E94A0780C94E7691A93D0
:10C804000A93E0916B0CE03011F00C94EF68E3E0D4
:10C81400EA930FDFE0915B0BE295EF70EA930E94DD
:10C82400D5681E2FE0915B0BEF70EA930E94D568E8
:10C834000E2F1A93FEDE0A93FCDEE7E1EA93F9DE9B
:10C84400E0EEFDE00E94D8780E94F57BEA1BE093BD
:10C85400E00E689425F80C94EF68EE81EA93B4DF57
:10C86400EC81FD810E9468730E941C7A6BDFC7DF34
:10C874000C940E6AEB81EA93A7DF0E94D871EADE7A
:10C884000E94187ABCDF24960895ED81EA939CDF18
:10C89400EB81FC810E946873EA81EA93CADEE98134
:10C8A400E03011F0EA93C5DEE881E03011F00E9437
:10C8B400187AA5DF269608950E94B47D10E0E0EF73
:10C8C400F8E1A885B985EA17FB0719F444E150E0BB
:10C8D40002C048EC50E0EA85E0933709E89431F867
:10C8E400EA93E985FA85FA93EA93EA85EA93EA8575
:10C8F400EA93E0E0EA93C9DF0E94E6689F010E94A0
:10C90400A1140E9404770E94F2680E2F31FC02C029
:10C91400003009F001C0F3CF31FE04C0E89431F8CF
:10C92400E1E004C01F5F1230B0F2E0E00E94BB7D82
:10C934002B9608951A930A93E0913F0AE03011F47C
:10C944000C94EF68E0E0E0933809E2E0EA9309DA56
:10C9540010E003E00E94DD710E94237A61F00E94DE
:10C96400DD710E94E8770E94DD71E15CF54FE081A2
:10C974000E271F5FEFCFE3E0EA93F3D9E02FE295B0
:10C98400EF700E94287AE02FEF700E94287AE7E186
:10C99400EA93E7D90C94EF681A930A93E0913F0A5B
:10C9A400E03011F40C94EF680E94E870E03021F05C
:10C9B400E091410AEA3209F405C00E94E870E05DA2
:10C9C400E093410AE0E0E0933809EAE5EA93C9D943
:10C9D400E0E0EA93C6D910E00E94DD710E94237A58
:10C9E40011F01F5FF9CF1F5F012F0A93BAD910E02E
:10C9F4000E94DD710E94237A61F00E94DD710E9421
:10CA0400E8770E94DD71E15CF54FE0810E0F1F5F56
:10CA1400EFCFE02FE195EA93A4D9EDE0EA93A1D911
:10CA24000C94EF681A930A93F894E0E0E0933608C4
:10CA3400E091E10EE093E00E7894E0913F0AE0305B
:10CA440011F40C94EF68EAE5EA933DDCE0E0EA9344
:10CA54003ADC10E00E94DD710E94237A11F01F5F1E
:10CA6400F9CF1F5F012F0A932EDC10E00E94DD71C5
:10CA74000E94237A79F00E94DD71E15CF54FE08138
:10CA8400EA9321DC0E94DD71E15CF54FE0810E0F39
:10CA94001F5FECCFE02FE195EA9315DCEDE0EA931C
:10CAA40012DC0C94EF68E881EA938EDEEAE5EA93FF
:10CAB400C0DDE0913F09EA93BCDD0E947673EC91FE
:10CAC400E03031F00E940779B4DD0E946D74F5CF37
:10CAD40096DE0C94E7691A930E94B172E0913A08C9
:10CAE400EA93A7DDE4E4EA93A4DDE0913808EA934D
:10CAF400A0DD14E00E94DD71E95CF74FE081E430D1
:10CB040040F00E94DD71E95CF74FE0810E94097AF0
:10CB1400F1CFE0E0EA938DDD3FDF8BC11A930A93F6
:10CB24004FD9E0913E09E03011F40C941766A091BE
:10CB34003E09AA3541F4A0913A09A33020F0E091CE
:10CB44004009E43409F04BC00E94E870E03021F061
:10CB5400E0914109EA32C1F40E946C6EE05DA0915B
:10CB64004109EA1721F0E0914109EA3221F40E94D7
:10CB74004E5D12DF08C0E2E4F9E00E948273E091A6
:10CB840041090E942E7A2BC00E94E870E05DA091BA
:10CB94004109EA1721F50E946C6E1E2FE0914209AB
:10CBA400ED3421F4E0914309E33209F007C0E4E4F1
:10CBB400F9E00E94827370DC1E2FD1DB0E946C6E40
:10CBC400E11729F0E12FE05D0E942E7A08C00E944F
:10CBD4006C6EE05DE09341090E944E5DDDDEA09144
:10CBE4003E09A53449F4A091E40BA33019F40E9442
:10CBF400122B02C00E94D44EA0913E09A33411F41A
:10CC04000E94C32AA0913E09AB3411F40E94BE2AAB
:10CC1400A0913E09A23431F4A091E40BA63011F4A2
:10CC24000E947F4EE0E0E0933E09E0E00C94EF6860
:10CC34002BDAA0916C0CA43529F4A0E025FCA1E02A
:10CC4400A03009F03AC0E0913908E03581F4E09170
:10CC54003A08EA93E6E0EA930E942243A0913A0854
:10CC6400A03820F0E0913A08E093650523C0E0374E
:10CC740021F4E0E0E09365051DC0EA3519F40E9453
:10CC8400C95D18C0EA3711F426DF14C0E23519F47F
:10CC94000E9497500FC0E23719F40E94CC500AC08A
:10CCA4000E94A130E0913808A0913709EA1711F4E5
:10CCB400689431F8E0E0E0936C0CA0916C0CAA3518
:10CCC40031F40E944E5DAEDEE0E0E0936C0CB6C041
:10CCD400A0916F0CA13050F0E0916F0CE150E09303
:10CCE4006F0CE03019F4E1E0E093700CA0E025FC57
:10CCF400A1E0A13049F4A0E026FCA1E0A03021F499
:10CD0400A0913608A03009F001C006DBE091360896
:10CD1400E03019F0E150E09336080895E091DF0D1A
:10CD2400EF5FE093DF0DE0916E0CEF5FE0936E0C2C
:10CD3400E0916B0CE03019F0E150E0936B0C089536
:10CD4400E0911C0CE03029F4E3E0E0939000E8E388
:10CD5400E9B9A0911C0CA13029F4E1E0E093900022
:10CD6400ECE9E9B9A0911C0CA23029F4E0E0E093CD
:10CD74009000EEECE9B9A0911C0CA33029F4E0E09A
:10CD8400E0939000E7E6E9B9A0911C0CA43029F4E3
:10CD9400E0E0E0939000E3E3E9B90895E091610BEA
:10CDA400E0937100E0E0E0937400E2B3E360E2BB7F
:10CDB400E1B3E360E1BB85E38A95F1F7E1B3EC7F8E
:10CDC400E1BBE4E4E093740088EC90E00197F1F7B0
:10CDD4000895E2E001C0E0E0E093610BDFDF089535
:10CDE4001A931FEFF6DF16D0E03089F4E9810E9430
:10CDF400357A41F4EDB7FEB7FA93EA931F930E9494
:10CE04003A7A1F9118D080E991E00197F1F7E3DFB6
:10CE1400E12F70C01A9314EAE4EA0E943E7A41F4C6
:10CE24000E94437A183011F0103111F4E0E001C08F
:10CE3400E2E019910895E4E9E0937400E0E00895D4
:10CE44001A93E981E1600E94487A31F40E94437A9E
:10CE5400103411F4E0E04EC04CC01A93E9810E94F2
:10CE6400487A31F40E94437A183111F4E0E042C068
:10CE740040C01A93E9810E94487A31F40E94437AAF
:10CE8400183211F4E0E036C034C01A93E981E0307E
:10CE940011F0E4EC01C0E4E80E943E7A79F40E94C7
:10CEA400437AE0917300AA81BB81EC93103511F0B1
:10CEB400183521F4E0E018810C944D6CE1E0188100
:10CEC4000C944D6C1A93E981E093740010E0E091A6
:10CED4007400E07811F4163908F005C08BE18A95E6
:10CEE400F1F71F5FF4CFE0917400E07811F0E0E017
:10CEF40001C0E1E01881229608950E94B67D3D812B
:10CF04000C8120E087DFE03011F5EE810E949D6FF7
:10CF1400F1F43A93AEDFE030D1F40E944C7AB9F4E4
:10CF240079DFE030A1F4EE810E94357A81F4EDB727
:10CF3400FEB7FA93EA931F930E943A7A1F91E03066
:10CF440031F479DFE12F0E94BD7D0C940E6A26DF57
:10CF5400D9CF0E94B67D30E00E811D815BDFE030C9
:10CF640099F4EF810E949D6F79F40E944C7A61F4E8
:10CF74001A937FDFE03041F4EC81EA937ADFE0300A
:10CF840019F459DFE0E002C009DFE8CF0E94BD7D5B
:10CF94002896089522970E94B47D50E02B853A8507
:10CFA400A89538DFE03011F00C942E68EE850E94CD
:10CFB4009D6F11F00C942E682A935BDFE03011F022
:10CFC4000C942E683A9355DFE03011F00C942E68DF
:10CFD40021DFE03011F00C942E68EE850E94357A42
:10CFE400D9F5E0E0EE83EF83EC85FD8531970E946F
:10CFF4008D7649F4EDB7FEB7FA93EA931F930E9436
:10D004003A7A1F9109C0EDB7FEB7FA93EA931F93DA
:10D01400E1E0EA933ADF1F910E2FEE81FF81A885AC
:10D02400B985EA0FFB1F1083EE81FF813196EE83F1
:10D03400FF83003039F4EC85FD85AE81BF81AE17E6
:10D04400BF0708F001C0D0CFEC85FD850E948D7626
:10D0540019F4F1DEE0E002C0A1DEA3CF0E94BB7DA3
:10D064002F96089568970E94B47D20E0E0E0EC8F4D
:10D07400ED8F31E0A895E9A1FAA1662777270E94F0
:10D084008B7CEA87FB876C877D87EE8D0E94517AC3
:10D09400EE83FF8368877987AA85BB858C859D8508
:10D0A4000E94617DEA8BFB8B6C8B7D8B0E94E57B00
:10D0B400FE017296FA93EA930E944F6CEE8BFF8BFB
:10D0C400688F798F0E94577A0E94527CAF010E9428
:10D0D400577AAE8DBB27882799270E94EC7B0E9444
:10D0E4006A7ADE015A960E94527CED93FC930AA15F
:10D0F40019A190DEE030D1F5EDA10E949D6FB1F54C
:10D104000E944C7A99F51A93B4DEE03079F5303008
:10D1140051F14F5F5F4FEC8DFD8D3196EC8FFD8F9C
:10D12400AC8DBD8D1197EBA1FCA1EA17FB0711F49F
:10D1340030E018C0EC8DFD8D3197AF8DB8A10E9401
:10D14400CD7697DEEE8DDA01F0E0EA17FB0751F4B5
:10D1540072DEEA8DFB8DA9A1BAA1EA0FFB1FE9A338
:10D16400FAA389CFD4CF67DEE0E002C017DEC1CFD7
:10D174000E94BB7DA6960895A881A03310F0AA331F
:10D1840008F004C0E881E0530C94E769A881A13455
:10D1940010F0A73408F004C0E881E7530C94E76961
:10D1A400EFEF0C94E769A881AA3020F4E881E05DF0
:10D1B4000C94E769A881AA3020F0E881E95C0C941A
:10D1C400E769E8E50C94E7691A930A93F8940091E7
:10D1D400620B1091630B7894F801099119910895E9
:10D1E4001A930A93F1DF8F01EA81FB81AC81BD813F
:10D1F400EA0FFB1FE01BF10BDF010E94AA7D2CF458
:10D20400E0E0198108810C947B6CE1E019810881CC
:10D214000C947B6CEEEEF5E1FA93EA93EAEBF0E022
:10D22400FA93EA930E94BB75E4E0EA93E6E2EA9398
:10D23400EEE0EA930E94574DE6E8F6E1FA93EA93AA
:10D24400EAEAF0E00E946F7AE8E0EA93E0E2EA9327
:10D25400E1E0EA930E94574DE6E8F7E1FA93EA9396
:10D26400E2EDF0E00E94CB6CFA93EA93E2E0EA93F9
:10D27400E2E1EA93E1E0EA930E94574D0E94A46C34
:10D284000E94FB6EEFEAF0E00E946F7AE3E0EA931B
:10D294000E946D4BEAE0F0E0FA93EA93E4E3F0E0F5
:10D2A4000E94E66EE0E0E0931004E4EFF8E10E94EF
:10D2B400066EEFE0E0931004089508959981888143
:10D2C400009641F0BD81AC81FB81EA8105900D920D
:10D2D4000197E1F7FD81EC810C947B6CB981A88105
:10D2E400109631F0FC81EB816A8161931197E9F723
:10D2F400EB81FC8125960895E991F991A991B99161
:10D304001D900590011421F40020D1F7EE27089513
:10D314001018E1F3E1E008F4E2500895E991F9917D
:10D32400A991B991CD0161916D936623E1F7FC0157
:10D334000895E991F991A991B991CD0105900D92C2
:10D344000020E1F7FC010895A991B991EE27FF2788
:10D354006D91662311F03196FBCF0895AA27BB2760
:10D36400E991F9910590002011F01196FBCFFD0190
:10D3740008957991E991F991A991B991CD01772312
:10D3840051F07A9561916D936623C9F7772319F06B
:10D394007A956D93FBCFFC0108956991E991F99118
:10D3A400A991B991CD01662351F06A9505900D922A
:10D3B4000020C9F7662319F06A950D92FBCFFC0192
:10D3C40008955D9BFECFE881ECB9219608951A93E8
:10D3D4000A93AC81BD810E94D27B3097C1F0AA81AF
:10D3E400BB810E94D27B8F01309749F00230E0E08C
:10D3F4001E0760F0F80131978F01ED93FC93AC8127
:10D40400BD810E940F6F3197AE81A08303C0EE816E
:10D41400EA93D7DF19810881279608952C970E94F3
:10D42400B47D10E0E88DF98D3196E88FF98F31974E
:10D43400E4912E2FE03011F40C94CE6BE12FE03008
:10D4440039F4253211F411E002C00E94767AA3C1A6
:10D45400E130C1F4253219F40E94767A9BC112E0BE
:10D46400E0E0E98B00E02D3211F401E094C12B32AD
:10D4740019F4EBE2E98B8FC1203219F4E0E2E98B75
:10D484008AC102C0E23039F450E013E0203311F4D1
:10D49400006881C102C0E330A1F4203310F02A33C4
:10D4A40008F009C0A52FEAE0EA9FF0015E2FE22F01
:10D4B400E0535E0F70C140E02E3211F414E06BC1F2
:10D4C40010C0E430A1F4203310F02A3308F009C06E
:10D4D400A42FEAE0EA9FF0014E2FE22FE0534E0F13
:10D4E4005AC12C3619F4026015E055C104C0E53068
:10D4F40011F00C94CD6BE22FE33649F40E94817A4B
:10D50400EE89FF89A481AA930E94877A43C1E337F5
:10D5140041F40E94817A0E94917A0E94A6691E2F8A
:10D524000AC0E037A1F40E94817A0E94917A0E9495
:10D53400B0691E2F08600F77403011F0411708F0D2
:10D5440001C0142F40E0E0E0E88B30E076C0E43620
:10D5540011F0E93611F4046002C0E537A1F4EAE001
:10D56400E88B01FF08C0E0E0FAEC6AE97BE30E9483
:10D57400C96E1AE023C0E0E1F7E260E070E00E94C7
:10D58400C96E15E01BC0E83511F4086004C0E83723
:10D5940011F00C94CC6BE0E1E88B01FF08C0E0E0F3
:10D5A400F0E060E070E10E94C96E18E007C0E0E0BE
:10D5B400F0E160E070E00E94C96E14E0403011F0C8
:10D5C4000F7701C041E001FF08C00E94817AAE8953
:10D5D400BF8914960E94D67B13C002FF08C00E9424
:10D5E400817AAE89BF8914960E945F6E09C00E9439
:10D5F400817AAE89BF8914960E94D27B66277727E9
:10D60400EC87FD876E877F8702FF16C0AF85AA234C
:10D6140062F4EC85FD856E857F850E94D17AEC8766
:10D62400FD876E877F87EDE2E98BE989E03019F0A9
:10D634001F5F4F5F01C00B7F342F00FD14C015170F
:10D6440010F4351708F00FC007FF08C002FF04C02C
:10D654000B7F2989115001C020E301C020E20E9400
:10D66400767A5150ECCF1417B0F4006102FF0AC06F
:10D674000B7FE989EA930E94877A503009F0515070
:10D6840011504150E0E3EA930E94877A503009F048
:10D6940051504150E8CF312FE889E030D1F4303097
:10D6A400B9F003FF08C0EE81FF813196EE83FF835A
:10D6B4003197E49105C0AE81BF81ED91AE83BF8304
:10D6C400EA930E94877A503009F051503150E7CFE5
:10D6D40057C00E94997A0E945E7B2E2F2A3030F028
:10D6E40003FF02C0295C01C0295A01C0205D04FD6A
:10D6F40025C0213360F4A885B9858A859B85A1302E
:10D70400E0E0BE07E0E08E07E0E09E0709F40BC00E
:10D71400431740F4531710F000FF01C014C020E277
:10D7240007FF0CC020E3006102FF08C00B7FE989FA
:10D73400EA930E94877A503009F051500E94767A19
:10D74400503009F0515031500E94997A0E94997BCF
:10D75400EC87FD876E877F87E889A885B9858A85E8
:10D764009B85FF27662777270E945E7B0E94C96EF0
:10D77400E885F9856A857B850E94A67D09F0A9CF95
:10D7840000FF08C0503031F05150E0E2EA930E94AB
:10D79400877AF8CF10E046CE0E94BB7D6A96089542
:10D7A400FF92F82E22971A930A93DE010E94BF7A01
:10D7B4008D01DE0116960E94BF7A0E94D27BEA8315
:10D7C400FB83DE0114960E94BF7A0E9468741A9348
:10D7D4000A93FE0136960E94D06C20DEAA81BB819A
:10D7E400E0E0EC93198108812496FF9008957B81F1
:10D7F4006A81F981E88177FB770F67FD7160972F64
:10D804009E5781F078F0983190F4AA27BB27882797
:10D8140008948795B795A7959A95D1F7EA23FB23A2
:10D82400682305C0E8947727EE27FF2766276F77DC
:10D83400769508F4606877F9A991B99189919991DD
:10D84400EA17FB076807790797FB08950E941C7A7B
:10D854000E94A27A19F40E94A97A1DC0E6F7A88151
:10D86400B9818A819B81E0E0F0E060E87FE30E9477
:10D874006A7A11C00E941C7A0E94A27A19F40E944A
:10D88400A97A09C0E6F30E94A97AA0E0B0E080E892
:10D894009FE30E94C57C249608950E94AE7A0E945C
:10D8A400A67D39F4A881B9810E949B700E94DC7B1B
:10D8B40020C0AA81BB818C819D810E94AE7D34F4FD
:10D8C4000E94AE7A0E94E57BC1DF05C00E94AE7A59
:10D8D4000E94E57BCFDFA881B9810E94DC7BA8810F
:10D8E400B9810E94D67BAA81BB818C819D810E94D3
:10D8F4006A7A26960895E991F99130971AF4E09599
:10D90400F095319608950E94EB66E0EBEA93E8E126
:10D91400F0E0FA93EA93E1E0F0E0FA93EA93E3E2C9
:10D92400F7E0FA93EA930895E0EBEA93E0E0F0E09D
:10D93400FA93EA930E947F670C94ED66E0E2EA931F
:10D944000C943468E0E0F0E0FA93EA930895EFEE83
:10D95400F0E0FA93EA930895FA93EA93E0E0EA9305
:10D964000C946D4BFA93EA930C94D643E12FAEE3F7
:10D97400B3E0F0E00E94E57AEA0FFB1F0895A12FBF
:10D98400B0E0ECE3F0E00E942E7B3896FA93EA9341
:10D994000895FA93EA93E2E3F0E00895FA93EA93A0
:10D9A400D1CFE0911004E0930F0408950E94E80C95
:10D9B4000C948649E32FF0E0E65AFC4FE491089575
:10D9C400EA930E94FE0CFE013696FA93EA930895B8
:10D9D400FF27662777270E94E57B84E00E94D26BAD
:10D9E40028960895FE017196FA93EA930C94F643EF
:10D9F4000E94B67D0C94FE46E8E0F0E0FA93EA93C8
:10DA04000895E4E0F0E0FA93EA930895FA93EA9330
:10DA1400E8E3F0E0FA93EA9308950E94E17BBECF35
:10DA2400E02FF0E00895A0913C0CB0913D0CBD01B5
:10DA3400A3E0B0E00E94067BE60FF71FE491E0301C
:10DA44000895E091C005EE0FEE0FEF5F3E2F0895AD
:10DA5400E32FF0E00895A12FB0E00895A0913C0CCD
:10DA6400B0913D0CBD01A3E0B0E00E94067BE60F3F
:10DA7400F71F08950E94E37AE254FD4F0895FA9344
:10DA8400EA93E22FF0E008950E94B47DA091190872
:10DA94000895E091C20BF0E00895AFE3B1E00E9475
:10DAA400597B089530911E08E1E0E0930D04E2E013
:10DAB400E0930E043A930E947718E091980BE29554
:10DAC400EF70E0930F04E091980BEF70E093100473
:10DAD4000895FA93EA93E52FF0E0FA93EA93089510
:10DAE400E7E3F0E0FA93EA930895E22FE450F0E0DC
:10DAF400FA93EA930895EA85FB85FA93EA930895E5
:10DB0400E32FE058EA931ECFEAE8FBE0FA93EA93A6
:10DB14000C94F6433A930E947718A0918A0BAD3285
:10DB24000895E091980BE295EF70E0930F04E09173
:10DB3400980BEF700895E52FF0E00895EA0FFB1FAE
:10DB4400FA93EA930895EF5EFC4FBF01E081E05839
:10DB5400DB01EC930895E0E0EC93AE81BF8108957E
:10DB6400E3E0F0E0FA93EA930895E52FE450F0E05F
:10DB7400FA93EA930895E0E0E0930F04EFE0E09372
:10DB840010040895E550F0E00895E091980BE295B3
:10DB9400EF700895EA1BA2E5B7E0F0E00E94E57A91
:10DBA4000895F0E0EE0FFF1FE05BFC4F0895AEE434
:10DBB400B3E0F0E0EE0FFF1FEA0FFB1F0895FA93A6
:10DBC400EA93E12FF0E0FA93EA9308950E94FE4667
:10DBD400E0E0EA930895E12FF0E0FA93EA930895E0
:10DBE400FA93EA93E2E0F0E0FA93EA930895EAE81C
:10DBF400FBE0FA93EA93EAE0EA930C949F46E1E0AF
:10DC0400F0E0FA93EA930895FA93EA930C94884621
:10DC14000E94E17BFA93EA930895ABE0EA9FF00156
:10DC2400E252FA4F0895ED85FE85FA93EA9308953A
:10DC34001A930A932ECF1A930A93E0E0EA930E9470
:10DC44006D4BDDCFE1E0E0933E0C0E94E668E0938B
:10DC5400400CF093410C0895BD01AAE0B0E00E948D
:10DC6400067BE60FF71F0895FA93EA93EAE0EA9336
:10DC74000C949F46E1E0E0930E0464CE0E94D746E4
:10DC84000C94BA46E0E2EA930C947146A3E2B7E03E
:10DC9400E881F0E0EE0FFF1FAE0FBF1F0E94D27BA2
:10DCA4000895FA93EA930C948941E881F0E0089589
:10DCB400EE0FFF1FAE0FBF1F08950E94D27B0E947C
:10DCC400F07A08950E94E57B0C946A41FA93EA93F2
:10DCD4000C94D746A9E0B0E00E94007C0895A7E127
:10DCE4001A9FF001EF5CF94FE0810895E12FEF5F97
:10DCF400EA930C949F41F0E0D4CFE8E0F0E04ECEFC
:10DD0400EA93E6E0EA930E94554176CEE0936200FE
:10DD140088EC90E00197F1F70895E093610088ECB6
:10DD240090E00197F1F70895E0916D05F0916E058B
:10DD34000895E0916905F0916A050895AE0FBF1F3B
:10DD4400E3E0F0E00E94597B0895FA93EA931A9372
:10DD54000A930C941D12FA93EA933A932A930C941F
:10DD64001D12A0917105B09172050895A0917305DB
:10DD7400B09174050895A0E0B0E00E94FC7B089582
:10DD84000E94F57BEA1BFB0B0E94F07A0895E8875A
:10DD9400F9876A877B870895A885B9858A859B85D5
:10DDA400EFEEF0E060E070E008950E94F07A0E94E7
:10DDB400837B0895A4E0B0E00E94FC7B0895EC838B
:10DDC400FD836E837F830895FA93EA930C94F2465D
:10DDD400FA93EA930C94B37AA9E01A9FF001E25003
:10DDE400FC4F089537960E94E17BDF010E94D27BAD
:10DDF4000895E2E3F0E0FA93EA9308950A921A92FE
:10DE0400FA926A937A938A939A93AA93BA93EA9327
:10DE1400FA93EFB7EA931A930895ED91FD91319631
:10DE2400FE93EE930895ADE01A9FF001EB5FFC4F73
:10DE3400E08108951A93E1E0EA930C946047ADE021
:10DE44001A9FF001DF01EB5FFC4FE081E0300895A1
:10DE5400E2E0EA930C946047FA93EA93E4E6F0E094
:10DE6400FA93EA930E94F268E0300895E1E0E093C7
:10DE74000D04E0930E040895E0912808F091290818
:10DE840060912A0870912B080895E0912008E150D0
:10DE9400A3EAB6E0F0E00E94E57AAE0FBF1F0E944D
:10DEA400D67B0895E12FEF5FF0E010CFE0912108D9
:10DEB400EA93E0911E08EA930E948A1AA0911F0C2B
:10DEC400B091200C10970895A091210CB091220CD0
:10DED4008091230C9091240C0E94AE7D0895E091D2
:10DEE4001F0CF091200C0895E091210CF091220C6C
:10DEF4006091230C7091240C0895EAE0F0E068CF5F
:10DF0400E2E3F0E065CF1A93E0EAEA93EA81F0E015
:10DF1400E054F14FFA93EA930E947F671E2F08950D
:10DF2400E0EAEA93EA81F0E0E054F14FFA93EA93ED
:10DF34001A930C94AB67EA930E942F67E03008951C
:10DF4400E0EAEA93EFE5F0E0FA93EA93E0E0FFE039
:10DF5400FA93EA93EEEBFBE00895FA93EA93EECC9E
:10DF6400E0EAEA93E981FA81E050FE4EFA93EA93FB
:10DF74000895EA81F0E0A8E2B0E00E942E7B0895C3
:10DF8400E0EAEA93E2E0F0E0FA93EA931A930A9360
:10DF94000895FA93EA930C94CC67FA93EA930C9459
:10DFA4007F67E0EAEA93E8E2F0E0FA93EA931A93EF
:10DFB4000A93EAE8FBE00895EAE8FBE0FA93EA93BF
:10DFC4000895EDE2EA93EAE0F0E0FA93EA930E941E
:10DFD4007069E0E00895EA81F0E0ABE0B0E00E940F
:10DFE4002E7BE050F24F8F01AA81AA300895E0EA17
:10DFF400EA93EBE0F0E0FA93EA931A930A93E2EBE4
:10E00400FBE00895E3EBFBE0FA93EA930895EA81D9
:10E01400F0E0EE0FFF1FE050F04F8F01AA81A0380F
:10E024000895E150F0E00895EA81F0E00E94E57A75
:10E03400E058F14F8F01AA81A5300895E0E3FCE098
:10E04400FA93EA93E0E0EA93DCCCEDE1FCE0FA93A6
:10E05400EA93E0E0EA93D0CC0E94E57A0E94E17A68
:10E06400DF01EA85F0E0AE0FBF1FE8E0F0E00E94B8
:10E074002E7BE050FA4E8F01E0EAEA93BDCC1A936E
:10E084000A93EDE1FCE085CFD901F0E0AE17BF07BC
:10E094000895AE81BF81888599850E94C37AEE83F5
:10E0A400FF8368877987089540931F0C5093200C51
:10E0B400EE81FF8168857985E093210CF093220C31
:10E0C4006093230C7093240C0895F0E0AE0FBF1FEF
:10E0D4000895EA930E9477180C94841FE091950B9D
:10E0E400F091960B0895FA93EA930C941618ED8127
:10E0F400EA93ED81EA930895E091AC0BF091AD0BB6
:10E104000E94F07A0895E0912608F0912708089576
:10E11400E093280CF093290C0C94E71BE3EAF6E057
:10E12400FA93EA93E0E0EA930895FA93EA930C945D
:10E134007069E0E0F0E060E070E00895E0932808A2
:10E14400F093290860932A0870932B080895E091AE
:10E15400970BA3EAB6E0F0E00E94E57A0895AE0FCB
:10E16400BF1F0E94D67B0895ED5EF94FE081E13038
:10E174000895FA93EA93E0912108E05DEA93089503
:10E18400EA930E945E64E1300895EBE3F8E0E093E3
:10E194005F0BF093600B0895E12FA3EAB6E0F0E083
:10E1A4000E94E57A0895A881AF5FEAE00E94387B77
:10E1B400E05D0895A881AF5FEAE00E94887BE05D9E
:10E1C4000895FA93EA93E0E0EA930895AAE0B0E0B0
:10E1D4000E94007C0895E12FF0E00E94E37AEE5261
:10E1E400FF4F32960E94E17B0895E12FF0E00E94F8
:10E1F400E37AEE52FF4F08953696E491D901EC93F9
:10E204000895E0EAEA93E5E0F0E0FA93EA930895EA
:10E21400EA930E94D81BFA93EA93E5E2FCE008959E
:10E22400FA93EA93EFEFEA93E5E0F0E07ECFE09330
:10E23400260CF093270C08950E94F57BEA1BFB0B38
:10E244000895EAE2FCE0ECCFA0912B0CB0912C0CE9
:10E254000895E0E0E093390CE0933A0C0895A0911E
:10E264002D0CB0912E0C0895E0912D0CF0912E0CF4
:10E27400AC81BD81EA0FFB1F0895E0932D0CF09350
:10E284002E0C08951A930E94721C1E2F0895E09379
:10E294002B0CF0932C0C0895FA93EA930E94F268E5
:10E2A400E0300895ABE01A9FF001E452FA4F08956C
:10E2B4001A930E94611ED3CFE0912B0CF0912C0C89
:10E2C4000895EA930E94611E0E94FE1DE0300895A5
:10E2D400EB81EA930E94991CFA93EA93EAE2FCE048
:10E2E40008951A930A93A09119080895E0E0E09321
:10E2F400510CE093500C08951A930A93E09112087C
:10E30400ABE0EA9FF001E752F84F8F01D801119674
:10E314000895E0E0F0E0ED93FC930895EA81D801DC
:10E32400EC93E2E1F8E0FA93EA930E94BE33198198
:10E3340008810895E12FA6EAB0E0F0E0EE0FFF1F98
:10E34400EA0FFB1F0E94E17B0895E150ADE0EA9FD4
:10E35400F0010895A6EAB0E0F0E0EE0FFF1FEA0F27
:10E36400FB1F0E94E17B0895A0911608B091170845
:10E37400EA2BFB2BE0931608F09317080895E1505D
:10E38400A7E1EA9FF0010895A7E10A9FF001E15D8A
:10E39400F94FAF010895F0E0A4E6B0E00E942E7BAF
:10E3A4000895ED55F94FE081E0300895E981FA814F
:10E3B400FA93EA930895E12FF0E00895E2E0F0E0A3
:10E3C4000E94597B0895AAE9BBE0E0911A080895D8
:10E3D400ADE9BBE0E0911A0878CEA0EABBE0E09199
:10E3E4001A0873CEA3E2B7E0A6CBEE0FFF1FEA0F25
:10E3F400FB1F0895E081F0E00895A7E11A9FF00162
:10E40400E15DF94FEE83FF83AE81BF810895EE8114
:10E41400FF81A481AA930C94DA1F0D901C90AE8105
:10E42400BF811296EC91F0E0E00DF11DDB01ED935C
:10E43400FC930895ED91FD913197FE93EE93089529
:10E444000E947F21EF770E2EAA85BB851296EC9150
:10E45400E0150895A3E20A9FF001E855F94F0895E5
:10E46400E0911208ABE0EA9FF001E752F84FEC8725
:10E47400FD87AC85BD85119608951296EC91AC8507
:10E48400BD851696EC930895D001F0E00895A88513
:10E49400B98518960E94D27B0895AC85BD85EC930E
:10E4A400E2E1F8E0FA93EA930C94BE33E885F98547
:10E4B400A281AA930895AA85BB85EC91EA93E3E02F
:10E4C400EA930C942243AA85BB85E0E0EC93E2E056
:10E4D400E09324060895BF0100801180AE81BF81BE
:10E4E4001296EC910895DB01ED93FC93AE81BF810C
:10E4F400129631CBE4E6F0E00E942E7B0895F0E022
:10E50400ED93FC930895E2E1F8E0FA93EA930C9416
:10E51400BE33E0911908A0911808EA170895F0E0B5
:10E52400E00DF11D0895A3EABBE045CFADE9BBE0E2
:10E53400EE27A10FBE1FEC910895A0EABBE0EE27E1
:10E54400A10FBE1FEC910895BD01AAE0B0E00E94A6
:10E55400067BDB010895E081EA930C94B35EEFE35C
:10E56400FAE0E0935D0BF0935E0B0895EA930E944A
:10E574001B63E0E00895EA930E941B630C949C647F
:10E58400ADE9BBE0EE27A00FBE1FEC910895A0EA11
:10E59400BBE0EE27A00FBE1FEC910895AAE9BBE0F3
:10E5A400EE27A00FBE1FEC91E1700895A3EABBE033
:10E5B40037CAA0EBBBE0EE27A00FBE1FEC91089575
:10E5C400A9EABBE0EE27A00FBE1FEC910895EA81F3
:10E5D400ADE0EA9FF001E15FFC4FA0E0A083EA8197
:10E5E400EA930895ADE0EA9FF001EB5FFC4F0895D4
:10E5F400ABE00A9FF001E452FA4F0895ABE00A9FA2
:10E60400F001EE51FA4F0895FA93EA930C944B35C6
:10E61400FA93EA930E9497433A931ACCE0912D0C13
:10E62400F0912E0C30970895AFEFBFEFA083B18324
:10E6340008950E94E668E093560CF093570C0895F1
:10E64400FA93EA93E0E0F0E80895E0911208ABE071
:10E65400EA9FF001E752F84FFA93EA930E942729C0
:10E6640052CFE0911008ABE0EA9FF0010895E0E199
:10E67400F8E0FA93EA930C94BE33FA93EA930C9479
:10E684004153E88DABE0EA9FF0010895FA93EA93D1
:10E69400C7C9E0E1EA93E0912506EA930E944A188B
:10E6A4001E2F089530DDFA93EA930895FA93EA93BE
:10E6B4000C942C1EE0932506E0E0E093530CE1E378
:10E6C400E093540C0E94662A0C943226FA93EA933F
:10E6D4000C942C63E0E4F9E0E0935F0BF093600B9F
:10E6E400E3E0EA930C94C262A0915F0BB091600BDB
:10E6F40008950E94E668E0934B0CF0934C0C089547
:10E70400E0935F0BF093600B0895E3E0EA930C94BD
:10E71400C262E0932608F09327080895E0E0F0E051
:10E72400E0932408F0932508E2E0E0930E040895B2
:10E73400E091130427CAE0912408F0912508B1CA96
:10E74400E0915D05F0915E0531970895FA93EA939F
:10E754000C94CC45A0E024FCA1E0A0300895E7E0AF
:10E76400EA93E0E0EA93EEC8E0913208F0913308CE
:10E77400FA93EA930895FA93EA930E94F268E130D7
:10E7840008950E94E668E0933208F09333080895F0
:10E79400E0E0E093500C0895EF5CEA930C9471462A
:10E7A400A3EEB6E055C9A3EABBE0E0911A08F0E095
:10E7B4001CCE0E94D27BD001ED93FC9304CEF0E0FA
:10E7C400EA0FFB1F0F01FFCDA3E2B7E041C9E091BF
:10E7D4001908EA93E0E0EA930C94DE2BEA930E9492
:10E7E400FE400E9435431E2F0895EAE2EA93E0EDCD
:10E7F400F7E1E7CC0E94652CE1E0EA930C944D2C00
:10E804001F771A930C947718A0912408B0912508C7
:10E814000895E8EEF3E00E948B7B0895E053F0E066
:10E824000895F2DFEA17FB070895E0931808E0E083
:10E83400E0932F0808950E943C640E94852DE09384
:10E84400230808950E9477180C94FE460E94D92844
:10E854000E94641F0E943243E03008950E943543B1
:10E864001E2F1A930E94B82D103808951A93E09120
:10E87400C605EA930895E091890BEA930E948417F0
:10E88400E03008950E94E668E093580CF093590C28
:10E894000895FA93EA93F2C9D90118960E94D27B9B
:10E8A4000895E4E6F0E060E070E00E94837B089560
:10E8B4000E94771813CC0A93E091C605EA93089551
:10E8C400E0912E08EA930A930C94AD190E94D27B2E
:10E8D400FA93EA930895AFE5BBE09FCAE0913B0841
:10E8E400E053E09321080895FA93EA93E0E3EA936E
:10E8F4000C943C64E0913808EA930C94E6630E941B
:10E90400F07A0E94E57B08950E94A463EBE3EA9306
:10E914000C941B63E89423F8E0E0F0E0FADEE0E016
:10E92400E0931E080A93E1E0EA930C94DE2BE8944A
:10E9340023F8E0E0F0E0EDDEE0E0E0931E08EA9387
:10E944000C944D2CE0911208ABE0EA9FF00108957D
:10E95400A881B981EC91EF5FEC930895ABE00A9F35
:10E96400F001E352FA4F0895A083ABE00A9FF0014F
:10E974000895ABE00A9FF001E152FA4F0895EDEEDD
:10E98400F7E1FA93EA93EA85ABE0EA9FF001089590
:10E99400AC81BD81EE27A00FBE1F0895E02FAC818E
:10E9A400BD81F0E008950E94E57B84E00E94D26B73
:10E9B40028960895EE27A30FBE1FEC91D001EC9387
:10E9C4000895A2E5B7E00C942A6D0E94E57AEA0F57
:10E9D400FB1FAF010895E0912D0CF0912E0C0895CA
:10E9E400E32FA0911E08EA0F0895ADE02A9FF001DD
:10E9F400E35FFC4F0895A8E0B0E00E94007C089516
:10EA0400F0E0FA93EA9308950E94A6420C947542AA
:10EA1400F0E00E94E57A08950E94E57B0E9490420E
:10EA24000C9475420E94A642E0EFF7E1CACB0E9423
:10EA340075420C94754220E030E0E12FE05DEA93EA
:10EA4400E3EFF7E196CBEAE0EA930C94FC62E3E4AB
:10EA5400FBE0FA93EA93089510915D0500915F0538
:10EA640008950E9435433E2F0C941A46EAE0F0E0E4
:10EA74000E942E7B0895DF01EE27A30FBE1F089589
:10EA8400EF81F885FA93EA930895F0E0EA0FFB1F0B
:10EA94000895E02FACE2B2E0BBCFEA0FFB1F329641
:10EAA400E4910895FA93EA93E0911B0CEA930E948F
:10EAB4009238E1320895EA930E943838E132089599
:10EAC400E6E0F0E00C94D06CEAE3EA930C9471462F
:10EAD4000E94D746AAE9BBE0EE27A10FBE1FEC9126
:10EAE400E1700895EE0FFF1F0C94A06DEA930E944D
:10EAF4009238E13208950E94110D0C94A46C0E9486
:10EB0400E57B0C947E41E4E7F7E07EC8EA23EA93D0
:10EB14000E94A541B7C8EA930E94A541B3C8DF018A
:10EB2400329676C80E94E37AEE52FF4F0895E2EEE1
:10EB3400F7E0E0933C0CF0933D0C08950E940E1A0C
:10EB4400E0E0E09320080E943C150E94110DE1E0F2
:10EB5400E0931B0808950E94FE460E94B30F0E9492
:10EB640035430E2F0D330895EE81FF81FA93EA9316
:10EB74000895E5E0F0E0FA93EA930895E0E0EA937B
:10EB84000C94A46CEAE2EA93E5E0F8E10895EA93D0
:10EB94000E948C150C94110DE093C105F093C205ED
:10EBA4000895FE01FA93EA930895E6E1F8E1FA93F1
:10EBB400EA93EE85FF8568897989F5CEEAE1F8E183
:10EBC400FA93EA93AE85BF85888999896ACE0E94B3
:10EBD400E57BAA89BB898C899D89E4E6F0E060E045
:10EBE40070E00E949D7B0E94E57B88E00E94D26BCE
:10EBF4002C960895E3E2F8E1FA93EA93EE85FF8513
:10EC04007ECE84E00E94D26B2896CBCFFA93EA930F
:10EC1400EE85FF8508950E9401640C94E66884E003
:10EC24000E94D26B28960895EE27A10FBE1FEC9187
:10EC34000895EA930E9410421F5F0895E091C4056D
:10EC4400A7ECB5E0F0E00895AF5FEAE00E94887BAE
:10EC54000895E091C305A7ECB5E0F0E0C6CBA0E0D1
:10EC6400A083E981ADE0EA9FF0010895EF73A5E187
:10EC7400EA9FF001E051FB4F0895EF73ABE0EA9F88
:10EC8400F001EC5EFB4F0895AC81BD81EE27A30F2C
:10EC9400BE1FAC91A0300895ABE00A9FF001EC5E7A
:10ECA400FB4F0895EA0FFB1F0F01AC81BD8182CE9B
:10ECB400A5E10A9FF001E051FB4F0895EE81FF8129
:10ECC40001801280AE81BF8115960E94D27BD00153
:10ECD4000895FE013896FA93EA930895EAA5FBA5F0
:10ECE400FA93EA930895FA93EA93FE013A96FA9313
:10ECF400EA930E94906930E0E02F0895E091C10505
:10ED0400F091C2050895A1ECB5E0ED91FD91329624
:10ED1400FE93EE930895AE81BF81EA17FB07089531
:10ED2400E0E0E0936505E093660508951A930A937D
:10ED34003A932A930895FA93EA93E0910E0408957E
:10ED4400A0910003B09101030895E0910003F091B4
:10ED54000103FA93EA93E0910203F0910303FA9317
:10ED6400EA930895E0930003F09301030895A981C1
:10ED7400BA815ACFF801AA81BB81EA0FFB1FE49143
:10ED84000895AE0FBF1FAC91A0300895D801F0E0F4
:10ED9400AE17BF070895AE0FBF1FEC91EA93089515
:10EDA400EFEEF0E0EA1BFB0B0895A0910E04E4E102
:10EDB400EA9FF0012E2F3327C8CFE0E0EA930E94A8
:10EDC4006D4B0E94BD7D0895ECE0EA9FF001A09197
:10EDD4000D04EA9FF00108951A93E1E0E0930E0414
:10EDE400E0930D0410E00895ED81FE81FA93EA9317
:10EDF4000895EF81F885EA1BFB0B0895EA9FF00163
:10EE0400F0E008953A932A935A934A930895EAA511
:10EE1400FBA5E20FF31FFA93EA930895ECA1EA939A
:10EE24000C94D04B3A932A93EEA1FFA1E40FF51F63
:10EE34000895FA93EA93EBCFEAA5FBA5E40FF51F37
:10EE4400FA93EA93EBCFE20FF31FFA93EA93089550
:10EE5400FA93EA935A934A930895EA9FF001AEA174
:10EE6400BFA1F0E00895E2E0E0930E04E0E2F0E0F8
:10EE7400EAA3FBA30895AE1BBF0BA0CAEE8DF0E07E
:10EE84000895E20FF31F3196FA93EA93ECA1FDA1E2
:10EE9400E40FF51F31960C94E66EECA1FDA1E40F8E
:10EEA400F51F0C94E66EE9A1F0E0DE0116960895D4
:10EEB400ED8DEA930E942746E9A1EF5FE9A3089547
:10EEC400EFE3F1E0EA1BFB0B0895EB81FC81AF81DA
:10EED400B8850895E00DF11DFA93EA930E94E24982
:10EEE400E5E3EA930895E09365000C94826F0E9431
:10EEF400B47DEE81EA930E94114A8F010895E98559
:10EF0400FA85AD85BE8508950E942B4AEB85FC8564
:10EF1400FA93EA930C94434AED85FE85A985BA8554
:10EF2400AE17BF070895EB85FC85AF81B885AE1792
:10EF3400BF070895AD85BE85E985FA85EA1BFB0BFD
:10EF44000895FA93EA930C947D6CAB85BC8551CFFC
:10EF5400AF81B885EB85FC85EA1BFB0B0895D901CD
:10EF64000E942E7B0F010895D0010E94597BAF01AE
:10EF7400FA01AD85BE850C94A06DED85FE85E21B7E
:10EF8400F30BFA93EA930895AD85BE850C94A06DB6
:10EF9400A985BA85ED85FE85EA1BFB0B0895E881FA
:10EFA400F981FA93EA9308955A934A93EE85FF857B
:10EFB4002DCEFA93EA93EC85FD85FA93EA930E94A9
:10EFC400B14CE0910E04AA85BB855FCDE15CF54FA1
:10EFD400C2CAE091380CA091370CEA170895E09169
:10EFE4001108ABE0EA9FF001E655F84F0895F0965A
:10EFF400EA930E94E663E2E7EA930C941B63EA93C4
:10F004000E941B63EEE0EA930C941B63E6E3F8E1D1
:10F014005DCBE0911108ABE0EA9FF0010895FA930B
:10F02400EA930C944E63EBE3EA930C941B63EC5564
:10F03400F84FDF014BCCE0E3EA930C941B63E091BF
:10F044001008A0911108EA170895E1E1F8E0FA9395
:10F05400EA930C94BE33EA930E941B63E2E0E093CC
:10F064003408D7CFED55F84FA2E0A0830C94A24DFD
:10F07400E3E0EA930E948763CCCFA091260CB09181
:10F08400270C0895E2E5EA930E941B630C94A24DB9
:10F094001A93E985FA85FA93EA930895E552F84FAD
:10F0A400A885B985A083B1834DCCE2E5EA930C949D
:10F0B4001B631A93E0913808E0531E2FECE3F8E049
:10F0C4001FCBE0911208A0911308EA170895E3E119
:10F0D400F8E0FA93EA930C94BE33E0911308ABE0A2
:10F0E400EA9FF0010895A091740BAECDE093740BE8
:10F0F400EAE2EA930E94E663D8CFE091740BE05A07
:10F104007ECFD9011696EC917BCC0E944E638BCFB7
:10F11400F901A281B381BA93AA9308950E944E6320
:10F12400EAE3EA930C941B63D9011196E0E0EC93B3
:10F134000E940164CCCFD901EC9162CCE05DEA93EA
:10F144000C941B63E05DEA930E94E663AECFEB5838
:10F15400F44FE081E05D53CFEAE3EA930E941B633E
:10F16400F9010895E093620CF093630CE2E0E093FC
:10F174003508D9011196EC930895EA930E94E66349
:10F1840094CF0E944E6347CDE091190CDBCFE09100
:10F19400190CF0E0DCCF0E944E63ECE2EA930E948B
:10F1A4001B63FDCEA1DAAC91A0330895A0915D0B51
:10F1B400B0915E0B0895EE81FF81E093280CF093EB
:10F1C400290C1093250C0E94E71BE1E3089541E00C
:10F1D40050E00E944E62E887F987EAE3EA930E94CE
:10F1E400C161E13008951A93E985FA8531CEE2E2EE
:10F1F400EA930E94C161E030089576DAAC91A032BE
:10F20400089572DAAC91AB3308956EDAEC91EA9317
:10F214000895EAE3EA930C94C1610E944E62319727
:10F22400E887F987E88508950E94D27BE40FF51FEB
:10F23400D001ED93FC930895E0913F0BF0E0ED5580
:10F24400F94F0895E0E0E093690CE0936A0C0895A7
:10F254000E944E623197E0933F0BE091580BA091CE
:10F264003F0BEA1708950E94FF56E0913F0BEA9383
:10F274000895ECE2EA930E94C161E0300895ED5BE9
:10F28400F44F0F0131DAEC91D001EC931F5F23CBE3
:10F29400ED5BF44FA0E0A0830895EA930E94C1615E
:10F2A400E1300895E091400BF0CBE091400BEF5F2B
:10F2B400E093400B0895A3EABBE0E091400BF0E03B
:10F2C40094C8AAE9BBE0E091400B0C946770E0910C
:10F2D400400BF0E00895E2E2EA930C941B63FA9386
:10F2E400EA930C947153E0913F0BF0E01BCC0E9425
:10F2F4004E63ECE2EA930C941B63ECE2EA930C9405
:10F304001B630E946653E0E0E093400B0895E09194
:10F31400400B0C946770E0915F0BF091600B0895C3
:10F32400ADE5BBE00C940F6F41DFEC93F9CFE0E067
:10F33400EA930E94CA53E09334080895EA930E9422
:10F344001B630E948F53E1300895AA81BB81EC9125
:10F35400E295E07FAE2FEC810895EA0FAA81BB818C
:10F36400EC93F6CAE0910A0DA091090DEA170895ED
:10F37400E0913A09F0E0E15CF64F08951083E091E2
:10F384003A09EF5FE0933A09E12FA0913C0908950F
:10F39400E0933C09E0913B09E150E0933B09E03004
:10F3A4000895E15CF64FA0E0A0830895E091D50DA7
:10F3B400F091D60D0895A091D30DB091D40DEA1714
:10F3C400FB070895E12FA091DA0DEA0FE093DA0D1F
:10F3D400E091DC0D0895F0E0E95CF74F10830895A7
:10F3E400E091E10EF0E0E052F24FE081E0939C0006
:10F3F400E091E10EEF5FE093E10E089575D9AC91D1
:10F40400AA3308950F0170D9EC91E05388C8EA93A8
:10F414000E941B631F5F0895E4EEF8E1FA93EA93F8
:10F424000895FE013196FA93EA930895E881EA93E8
:10F434000C941B63E881F9816A817B810E94E57BDE
:10F444000895E15CF54FE081E0300895EA930E946D
:10F45400D568EA930C94B35EEA930E945565EAE595
:10F46400E0933D090895EA930E942267E0300895ED
:10F47400E0E0EA930C944767EA930E946467E03003
:10F484000895E0917100E87F1E2F0895E0937300C2
:10F49400E4E8F2CF0A930E943B67E0300895FF2727
:10F4A400662777270E948B7C0895EE8DAE85BF85F5
:10F4B40088899989F4DF0E94137DA9A1BAA18827BC
:10F4C40099270E94EC7B0E94EF7B0E94BE7C0895EA
:10F4D4000E94EF7B0E94BE7C0895FA93EA93E2E1D6
:10F4E400F0E0FA93EA9308952A93ED89FE89FA935A
:10F4F400EA93FE017596FA93EA930C94E969EE890E
:10F50400FF893497EE8BFF8B0895ED89FE89FA937A
:10F51400EA93FE017596FA93EA930C94E969AE892D
:10F52400BF8914960E94D27BEE83FF831DCBE885AE
:10F53400F9856A857B85AC85BD858E859F85089513
:10F544000E94F96BE883F9836A837B830895E881D9
:10F55400F9816A817B810895EA81FB816C817D81D7
:10F564000895E991F991309639F080EA9FE0019786
:10F57400F1F7A8953197C9F708950024AF0DB01D90
:10F584000895EA0FFB1F681F791F0895EA1BFB0B00
:10F59400680B790B0895F195E195F0400895F09585
:10F5A40060957095E195FF4F6F4F7F4F0895EE235F
:10F5B4000E2EEA2F19F0EE0F0A94E9F70895EE0FD4
:10F5C400FF1FEE0FFF1FEE0FFF1FEE0FFF1F08952B
:10F5D400FE2FFF0FFF0B6F2F7F2F08956F2F660FE6
:10F5E400660B762F0895BA2FBB0FBB0B8B2F9B2F67
:10F5F40008958B2F880F880B982F0895EA17FB071F
:10F60400E1E00CF0EE270895FA9FF02DEB9FF00D4A
:10F61400EA9FE02DF10D08957A9F702D6B9F700D78
:10F62400F89F700DE99F700D6A9F602D710DFB9F0F
:10F63400600D711DE89F600D711D8827FA9FF02DE4
:10F64400610D781FEB9FF00D611D781FEA9FE02D7F
:10F65400F10D681F781F089582D0D6DF0EF49BDF6A
:10F6640008958BD0D9DF0EF49ADF0895002498E032
:10F67400AA0F001C0E1A10F40E0E01C0A1609A9578
:10F68400B9F7EA2FA02D08950024112490E1AA0FC0
:10F69400BB1F001C111C0E1A1F0A18F40E0E1F1E8D
:10F6A40001C0A1609A9599F7FD01D001089557D042
:10F6B400EBDF0EF470DF08953F934F935F930024C4
:10F6C40011244427552730E2AA0FBB1F881F991F16
:10F6D400001C111C441F551F0E1A1F0A460B570B02
:10F6E40028F40E0E1F1E461F571F01C0A1603A9535
:10F6F40059F7FD01BC01D001CA015F914F913F91BF
:10F7040008953BD0D9DF0EF44ADF0895AFDFEA2F26
:10F714000895E894B7FF04C0A095B0951196689435
:10F72400F7FD39DFB1DFFD010EF435DF0895C4DFE5
:10F73400FD01BC010895E89497FF09C0A095B09518
:10F7440080959095AF5FBF4F8F4F9F4F689477FD23
:10F7540026DFB2DFFD01BC010EF421DF0895E89439
:10F76400F7FF02C018DF6894B7FF06C0A095B095F4
:10F77400119600F8039400FA0895E89477FF02C004
:10F784000EDF689497FF0BC00024A095B095809578
:10F7940090951196801D901D00F8039400FA089529
:10F7A400ED91FC9111970895ED91FD916D917C91EE
:10F7B40013970895ED93FD936D937C9308950590AD
:10F7C400F491E02D08957A936A93FA93EA93089555
:10F7D400689401C0E89401D09DD0182E862F612D25
:10F7E400192E972F712D1B2EBF2FF12D1A2EAE2FF0
:10F7F400E12D0895119602D0FE2F1197E199FECFC5
:10F80400FF93FFB7F894AEBBBFBBE09AEDB3FFBF65
:10F81400FF91089507D01196EF93EF2F03D0EF9146
:10F8240011970895E19B02C0A895FCCF9FB7F89467
:10F83400AEBBBFBBE09A8DB3E81719F0EDBBE29AFB
:10F84400E19A9FBF0895552342F4503811F4E0FF24
:10F8540004C03196691F791F6BF050E8572711F4E3
:10F864005F93CDC05F3F31F0660F000C57956795ED
:10F87400752F08955F9300200AF0CDC0C6C050E8EC
:10F88400192E1522880F991F9527550F879550E833
:10F89400072E0522660F771F7527550F6795089564
:10F8A400689401C0E8945F93F2DF703818F07F3FEA
:10F8B40008F4A5C056E1571BAAF4519558300EF42C
:10F8C400593030F0EFEFFFEF6FEF7FE777F91AC0B1
:10F8D40077275523B9F0EE0FFF1F661F771F5A9540
:10F8E400D1F710C07727583028F0EF2FF62F672F65
:10F8F4005850F9CF552331F076956795F795E795EC
:10F904005A95D1F700200AF44ADE5F91089568946D
:10F9140001C0E894309760407040B1F0002426F0B4
:10F92400772312F400943BDE172E7EE1112032F08F
:10F934007A95EE0FFF1F661F111CF9CFEF2FF62FDC
:10F94400612D5F938ADF5F9108954F93AF01FD01AD
:10F95400DA01AB01BC01CA01402D012C142E4F91D8
:10F964000895EA0FFB1F681F0895E095F0956095D0
:10F97400EF5FFF4F6F4F08955F9381DF903871F110
:10F9840050E8152604C05F937ADF903839F1703857
:10F9940021F1572F591B13F112F4D7DFFACF583145
:10F9A40018F0AA27BB278827583028F0AB2FB82F88
:10F9B40088275850F9CF552329F08695B795A795F0
:10F9C4005A95D9F7502D512562F0CBDF38F467955D
:10F9D400F795E795739513F41EC0B7DF3EDF5F918B
:10F9E4000895EA1BFB0B680B51F010F40094BDDF83
:10F9F4006623A2F3EE0FFF1F661F7A95CBF7EE275F
:10FA0400FF27662777275F910895EFEFFFEF6FE7F2
:10FA14007FEF5F910895EFEFFFEF6FE77FE75F916F
:10FA240008955F932CDF703851F3903841F301242B
:10FA34000894791F23F41CF300203AF3ECCF0F92BF
:10FA44001F932F933F934F93112722279927689F42
:10FA5400A0018F9F302D410D591F6B9F300D411D0B
:10FA6400591F8E9F27D0BF9F25D06A9F23D0BE9F4A
:10FA74001DD0AF9F1BD0AE9F110D291F391F491FE9
:10FA8400591FE32FF42F652F522F4F913F912F9140
:10FA94001F910F9066232AF0550FEE1FFF1F661F5C
:10FAA40002C073954BF2CFDE5F910895100D211DB6
:10FAB400391F02C0200D311D491F591F08955F933E
:10FAC400DEDE703821F411200AF49FCFA4CF9038E1
:10FAD40009F495CF01240894970B1BF4D4F3002068
:10FAE400F3CF792F1F932F933F934F931124112713
:10FAF400222733274427552790E2AE17BF078607EE
:10FB0400410730F0AE1BBF0B860B410B089401C0BC
:10FB14008894551F221F331F111CAA1FBB1F881F47
:10FB2400441F9A9551F7F901612D4F913F912F91FF
:10FB34001F91662332F0550FEE1FFF1F661F7A9543
:10FB440043F281DE5F9108953097604070400895DC
:10FB540000240A160B06089500240A160B0608064C
:10FB6400090608955A934A933A932A931A930A9347
:10FB740008955D814C813B812A8119810881089512
:00000001FF
